:020000040800F2
:1000000000200010111B030851A7020851C300086B
:100010004FA702084DA702084BA7020800000000E6
:1000200000000000000000000000000049A70208D6
:1000300047A702080000000045A70208F9DB0008F6
:10004000791B0308791B0308791B0308791B030834
:10005000791B0308791B0308211701084D180108B3
:1000600011180108D517010899170108351F000854
:10007000251F0008151F0008051F0008F51E0008B1
:10008000E11E0008CD1E0008791B0308791B030838
:100090006DA80208791B0308791B03085D17010886
:1000A00071D30008A1D3000861D30008B1D30008C0
:1000B00091D3000881D30008791B0308791B03083A
:1000C000791B0308791B0308791B0308791B0308B4
:1000D000791B0308C104010845040108C90301088C
:1000E000E5160108791B030835A70208791B0308E8
:1000F000791B0308791B0308791B0308791B030884
:10010000000000000000000000000000791B030850
:10011000791B0308791B0308693501084D3501086F
:10012000B91E0008A51E0008911E00087D1E0008CB
:10013000691E0008791B0308000000000000000091
:10014000791B0308791B0308791B030800000000D2
:10015000000000000000000000000000000000009F
:100160000000000000000000791B0308791B030851
:10017000791B0308000000000000000000000000E0
:0801800000000000791B0308D8
:10018800002870B51EDB0928044620DD012303EB97
:1001980083035B00B0FBF3F2092AF8D87BB10E4E5B
:1001A800B4FBF3F00928CCBF57223022A6FB03E5A5
:1001B800024403FB1044EB0801F8012BF0D10023A3
:1001C8000B7070BD2D230B7040420131DBE73030DE
:1001D80001F8010BF3E700BFCDCCCCCC884230B49A
:1001E8004FF001042ED301FB04F4B0FBF4F58D426B
:1001F800F9D284B1AAB901E0B0FBF4F5092DCCBF5E
:10020800572230222A4404FB150003F8012BB4FBC3
:10021800F1F4002CF0D100221A7030BC7047B0FB0A
:10022800F4F5092DCCBF372230222A4404FB1500EF
:1002380003F8012BB4FBF1F4002CF0D100221A7062
:1002480030BC70470546002AEBD1D7E703685A1C33
:1002580002601970704700BF2DE9F047089C2578A7
:10026800002B804689460CBF4FF0200A4FF0300A19
:10027800661C35B3002A29DD334601E0024698B1F1
:1002880013F8011B501E0029F8D1971E60B13D4696
:10029800013D51464046C8476B1C002BF8DC2578C9
:1002A80027EAE770013055B1041B29464046C84784
:1002B800301916F8015B002DF7D1BDE8F087BDE8CD
:1002C800F087002A04DC2846BDE8F0870020EBE729
:1002D800571EDCE783684268D0ED037A00EB8301A0
:1002E8000133934281ED040A836004BF00238360D5
:1002F80000EB830393ED047A036870EE277A9A4241
:10030800C0ED037A77EEC77AC0ED037A0CDA0133D1
:1003180007EE103AF8EEC76AB7EE007A87EEA60A3B
:10032800036030EE070A704707EE102AB8EEC77A66
:1003380087EE870A704700BF90ED057A90ED004A76
:10034800D0ED066AD0ED014AD0ED047A90ED035A5B
:10035800D0ED025AA4EE007AB0EE406AB0EE470A39
:10036800B0EE667AA6EE247A67EEC07AA0EE457AF9
:10037800E6EE257A80ED057AC0ED067A704700BF73
:10038800D0ED057A90ED013AD0ED003AD0ED064A6D
:1003980090ED024A90ED077A90ED035A90ED086AC5
:1003A800D0ED045AC0ED067AF0EE406A27EE830AD3
:1003B800C0ED056AA3EEA60A80ED087AA4EE240A29
:1003C800A5EE470AA5EEC60A80ED070A704700BFEA
:1003D800D0ED007A90ED017A30EE670AE7EE007A08
:1003E800B0EE670AC0ED007A704700BF704700BFE3
:1003F8000A44914214D030B40139551E41F2210209
:1004080011F8014F082380EA042004044CBF82EA53
:1004180040004000013B80B2F7D18D42F0D130BCA2
:10042800704700BF4FF4805383827047012380F8E0
:100438004530704790F8203033B1012B03D14FF489
:1004480000638382704770474FF4806383827047EC
:1004580070B40468037B2268022101FA03F31A428C
:1004680013D042690A495C2000FB02124FF6FE765F
:1004780050685289C5680068296831402960C16898
:10048800D24392B20A40C260636070BC704700BF3A
:10049800844E002030B40A4B1D7875B1094B0020FA
:1004A80003EBC5051A6899885062D4682143D16066
:1004B800083323F8040CAB42F4D130BC704700BFBA
:1004C800645100206851002010B40268047B116850
:1004D8000223A340194209D00649406800240C7041
:1004E80001684FF6FE742140016053605DF8044BCB
:1004F800704700BF09370020014B186810F08AB810
:1005080034210020F0B5836983B0054613B11A6819
:100518009B8813856869264F8389C3244FF47A73AF
:100528004FF0060E6E464FF6FF71013703E0013BB0
:100538009BB28B421DD002899207F8D504734FF401
:100548007A7302E0A3B28B4213D00289D20703F177
:10055800FF34F7D5027BD2B20EB132700136BEF14C
:10056800000F08D00EF1FF3EFF24002FE3D03C78A7
:10057800DBE711F0CFF9AB6913B11A689B88936177
:100588009DF805009DF801609DF802109DF8034054
:100598009DF804209DF8063041EA062143EA00232D
:1005A80042EA0422012029876A87AB8703B0F0BD9D
:1005B800C82F030810B490E80600047B40690223A2
:1005C800A3404B6013685DF8044B4FF6FE710B4077
:1005D80013600FF0AFBFF8B5174D2B78A52B28D1B6
:1005E8006B78BE2B25D1022229464FF6FF70FFF704
:1005F800FFFE124FAC1C22884AB1A618BE4218D280
:10060800052A16D92146FFF7F3FE3446F3E72146BB
:100618000222FFF7EDFE0222A118FFF7E9FE0634D9
:10062800074B641B1C8041F60F53C31A58425841AC
:10063800F8BD0020F8BD00BF00F003080000040862
:10064800863200202DE9F04FDFF848914C4F8BB0EF
:100658000326A7EB09071822002104A832F041FC61
:10066800484BCDF8109005971A69120604D5464AEA
:100678005A6002F188325A6001228DF8242034220F
:10068800DA60424B424C1B88ADF8003002226946C2
:1006980004A811F073FA022269464FF6FF70FFF7BB
:1006A800A7FEDFF8F4A080464FF0000B544536D380
:1006B8000AAC002524F8245D0222214604A811F082
:1006C8005DFA022221464046FFF792FE40BAC04337
:1006D800ADF80800022202A904A811F04FFA079801
:1006E80060B106ABC0F104022946184432F0F9FBA8
:1006F800069904A811F0E8F9079508909DF82430A8
:10070800089A23B11F490B6943F080030B61013E2E
:100718002DD0002A9FD1FFF75EFF50B32CE06588EB
:100728008DF80DB0C5F30B05AB1DADF80830238867
:10073800C3F30B02ADF80A201B0B062202A904A87A
:100748008DF80C3011F01AFA062202A94046FFF77C
:100758004FFE616880462A4604A811F00FFA6168C6
:1007680040462A46FFF744FE143480469EE7002A96
:10077800D1D005200BF028FE0BB0BDE8F08F00BFEC
:10078800000004080020024023016745CF2F03081A
:10079800708D030800F00308D09103080378202B1C
:1007A800024600F10100F9D0092BF7D02D2B2CD0EF
:1007B8002B2B03BF5378B7EE000A0246B7EE000AA8
:1007C800A3F13001C8B209289FED467A10D8F2EE9D
:1007D800046A07EE901AF8EEE77A12F8013FE7EE9E
:1007E800267AA3F13001C8B20928B0EE677AF0D9A9
:1007F8002E2B4CD003F0DF03452B0BD0F7EE007AFD
:1008080067EE276A20EE260A70475378BFEE000A83
:100818000246D5E710B451782D2959D02B290ABFA3
:100828009178501C901C0024A1F13003092B53D857
:10083800002303EB830301EB430310F8011FA1F12D
:100848003002092AA3F13003F3D9B3F59A7F28BF00
:100858004FF49A73072B42D9DFED236A1A46F7EE55
:10086800007A083A072A67EEA67AFAD803F007034F
:100878002BB1F2EE046A013B67EEA67AFBD124B3F2
:10088800C7EE276A5DF8044B20EE260A70475378B6
:10089800A3F13001C8B2092802F10102AAD8F2EE88
:1008A800046AF0EE665A07EE901AF8EEE77A12F844
:1008B800013F87EEA66AA3F13001C8B2092866EEA7
:1008C800A56A37EE067AEED994E767EE276AD9E784
:1008D800901C91780124A7E7F7EE007ACFE7F7EEAE
:1008E800007AC5E70000000020BCBE4CB5EEC00A87
:1008F800DFED317AF1EE10FACCBF30EE270A30EE98
:10090800670ADFED2E7A20EE270A30B5FDEEC07AB1
:1009180087B017EE904A054684EAE470002303A9DD
:10092800A0EBE4700193009302932FF0A3FB002C3B
:10093800ACBF20232D2303A88DF8003030F066FAD1
:10094800012803A924D002282DD0032805BF30236D
:10095800684668468DF8013032F0CBFA684630F0C8
:1009680055FA0338C4B222466946284632F0F8FAE6
:1009780000232B55284630F049FA2E22431C2A54CE
:100988000DEB0401E81832F0D1FA284607B030BD63
:10099800302368468DF801308DF802308DF8033029
:1009A80032F0A7FADAE7302368468DF801308DF87F
:1009B800023032F09EFAD1E76F12033A00007A440F
:1009C8002DE9F041064615460846B6FBF2F43CB957
:1009D80005FB1464124B1B5D00F8013BBDE8F08178
:1009E800B4FBF2F767B90E4B05FB174705FB146418
:1009F800DA5D00F8012B1B5D00F8013BBDE8F081D2
:100A0800B7FBF2F8B8F1000F02D04046FFF7D8FF65
:100A180005FB1878024B13F8082000F8012BE3E7D0
:100A28006C5D03082DE9F04714461D460646002371
:100A38004FF47A722046294630F092FEDFF848815A
:100A48004B4A4C4F88FB00310144C31782FB002EF0
:100A5800C3EB611188FB012887FB00278644464ABF
:100A6800C3EBEE2EC1EB011C82FB0E29A0EB8C0C14
:100A78000744424A86F806C0C3EB27474FEAEE7C94
:100A880008EB010ACCEBA90C82FB07824FEAE1785C
:100A98000CEB4C0CC8EB6A18AEEBCC0EC8EB081884
:100AA800DFF8E8C086F804E0A1EB880171718CFBDF
:100AB8000010F917C1EBE21240F2B55101FB1272B6
:100AC800C3EBE050B2F5896F4FEA80073FDA40F296
:100AD800DA239A4243DCB2F5B77FB4BF4FF0000C7B
:100AE8004FF0010C4FEA4C08254B08EB0C0103EBC7
:100AF800C1031FFA8CFE588C224908EB0C0301EB4A
:100B0800C30116310B2301E031F8020D82421BDAD2
:100B1800013BF9D11A4BC44403EBCC0C0123BCF8BC
:100B28000C00B37007F2B2770132121ABE44F270A9
:100B3800A6F800E0204629464FF47A72002330F0E8
:100B48000FFE3281BDE8F0870133DBB2E9E74FF0F1
:100B5800030EF44640F296504FF00608CCE74FF0EB
:100B6800020EF44640F229404FF00408C4E700BFE3
:100B7800C5B3A29107452EC2ABAAAA2A73B06D16B7
:100B8800C82F0308D42F030889888888792D031172
:100B9800104B2DE93048D3E9004554EA05020BD142
:100BA8000346012200201871587198719A70DA7002
:100BB80018801881BDE83088074B1A6814EB020BBF
:100BC80045F1000C5A466346FFF72CFF0120BDE8AB
:100BD800308800BFF81D002054650020F0B402885A
:100BE8008578164FC37804794179A2F2B27202F07F
:100BF800030606EB4606013D05EB860507EB4505B2
:100C0800013BAE898579008940F2B557920807FB08
:100C18000232931903EB430304EBC303C3EB03133F
:100C280001EB8303C3EB031305EB830300214FF4AC
:100C38007A72C2FB0301F0BC704700BFC82F0308DB
:100C4800FAB170B48E18044603E0101A14D1B142F8
:100C580014D014F8012BA2F14103192B11F8013B10
:100C6800A3F1410598BF2032192D03F12000ECD9DA
:100C7800D01A01D1002BEAD170BC7047002070BC9B
:100C880070471046704700BF4FF0FF32FFF7D8BFDC
:100C9800A0F16103192B98BF20387047A0F14103D8
:100CA800192B98BF20307047202805D00938042810
:100CB8008CBF002001207047012070476138192837
:100CC8008CBF002001207047413819288CBF0020B4
:100CD80001207047303809288CBF00200120704758
:100CE800A0F13003092B07D920F02000413819283A
:100CF8008CBF0020012070470120704730B4026883
:100D08001146531C036011F8024B0160D31C517843
:100D180003609378151D05601B0443EA0123D0780E
:100D2800234343EA006030BC704700BF0368591C86
:100D38001A46016012F8021B0260587841EA002046
:100D4800704700BF03685A1C02601878704700BFDC
:100D580038B504460068154630F0C6FF22682A44B4
:100D6800226038BD036810B40A0A5C1C04601A705B
:100D780003685A1C026019705DF8044B704700BF85
:100D880003685A1C026010B4197003680A0A5C1CD4
:100D980004601A7003680A0C5C1C04601A7003680B
:100DA800090E5A1C026019705DF8044B704700BFA9
:100DB80003685A1C026019700368090A5A1C026009
:100DC800197070472DE9F047002488B080460F4617
:100DD8001E46A14605AD531C0393117839B3252946
:100DE80033D1931CCDF810900393507830284ED00F
:100DF8004FF0000AA0F13003DBB2092B42D96C286E
:100E080019D0642800F0938024D825281CD063D9F1
:100E1800582876D063281BD131784046B847039AC2
:100E2800531C03931178043601340029D7D1204686
:100E380008B0BDE8F087039B5A1C03921B78642B0B
:100E48007CD02AD8252B54D1252140460134B847D7
:100E5800039AC0E7732833D044D975284FD106F1D7
:100E6800040E30682B4600220A217646FFF7B6F9B1
:100E7800049A0095534639464046FFF7EDF9039A20
:100E88000444A8E704AA03A92FF03CF8B7E7D31C49
:100E9800039390784FF0010AACE7732B10D05BD91D
:100EA800752B3AD0782B96D1A3F15802B2FA82F278
:100EB800306852092B4610210436FFF78FF9D7E71F
:100EC8003368049A0093394600234046FFF7C4F973
:100ED80004360444039A7EE70028B9D1204608B0B6
:100EE800BDE8F0876E28B3D1039A336804361C60D6
:100EF80071E72AD9582BD7D0632B8DD06BE7782888
:100F0800A6D1A0F15802B2FA82F2306852092B46F3
:100F18001021FFF763F90436AAE706F1040E3068DA
:100F28002B4600220A217646FFF758F9A0E7331D21
:100F3800306829461E46FFF723F999E7331D3068C4
:100F480029461E46FFF71CF992E7002B7FF443AFB2
:100F5800204608B0BDE8F0876E2BC6D03BE700BF3F
:100F68000EB400B584B005AB019053F8042B0649C4
:100F7800039301A8FFF726FF019B00221A7004B013
:100F88005DF804EB03B07047550200080FB430B5A4
:100F980083B006AB0A490B4853F8042B096800686C
:100FA8000193FFF70FFF084C054620680FF022FB5E
:100FB8000028FAD0284603B0BDE8304004B0704796
:100FC8009C2C0020A02C002034210020DFED2B7A5F
:100FD800B4EEE70AF1EE10FA4ADDDFED296A9FED7B
:100FE800297A01E0B0EE670AB4EEC70AF1EE10FA0A
:100FF80070EE667AF6DC9FED247AF4EEC77AF1EEAD
:1010080010FA38D5DFED1E6A9FED207A01E0F0EE88
:10101800407AF4EEC77AF1EE10FA37EEA60AF6D463
:10102800DFED1B7AB4EEE70AF1EE10FA14DDDFED1E
:10103800137A37EEC00A60EE006A9FED166A9FEDDC
:10104800167ADFED167AA6EE867A20EE266AE6EEA6
:10105800877AA6EE270A7047DFED117AB4EEE70A21
:10106800F1EE10FA44BFDFED087A37EEC00AE2E786
:10107800F0EE407ABFE7B0EE670AD1E7DB0F4940F0
:10108800DB0FC940E4CB1641DB0F49C0E4CB16C1E6
:10109800DB0FC93F92E741B99730083C15A82ABE33
:1010A800DB0FC9BF09B909E0194690FBF1F301FB51
:1010B80013030846002BF7D1084670470146FBE7A3
:1010C80007EE901AF8EE677A9FED837A27EE800A8A
:1010D80020EE070AFDEEC07A17EE903A2033402B37
:1010E80000F28C80DFED7D7AB4EEE70AF1EE10FABB
:1010F80040F3E880B0EE407A9FED796ADFED796AD7
:1011080001E0B0EE677AB4EEE67AF1EE10FA77EE27
:10111800467AF6DC9FED747AF4EEC77AF1EE10FAAF
:1011280040F1CD809FED6E6ADFED706A01E0F0EE70
:10113800477AF4EEE67AF1EE10FA37EE867AF6D4CC
:10114800DFED6B7AB4EEE77AF1EE10FA51DCDFED01
:10115800697AB4EEE77AF1EE10FA44BFDFED627A0D
:1011680037EEC77A27EE076ADFED635ADFED637A59
:10117800DFED636A9FED635AE6EE257A67EE065A5D
:10118800E6EE276AF7EE007AA5EEA67AF0EE675A41
:10119800E7EE055AE7EE457A87EEA55ADFED547A71
:1011A80030EE277AFDEEC76A16EE903A2033402BD0
:1011B80029D99FED557AF6EE006AB7EE006AF7EE88
:1011C800004AC4EEA57A0023836143610362C361C8
:1011D80080ED045A67EEA66A27EE866A27EE877ABC
:1011E800C0ED006AC0ED026A80ED016A80ED037A05
:1011F8007047DFED3A7A37EEC77AB3E7B7EE005AB1
:10120800F0EE455ACAE7B4EEE70AF1EE10FA5FDDF0
:101218009FED336ADFED336A01E0B0EE677AB4EE32
:10122800E67AF1EE10FA77EE467AF6DC9FED2E7A42
:10123800F4EEC77AF1EE10FA47D59FED296ADFED93
:101248002B6A01E0F0EE477AF4EEE67AF1EE10FA56
:1012580037EE867AF6D4DFED267AB4EEE77AF1EE49
:1012680010FA27DCDFED237AB4EEE77AF1EE10FA14
:1012780044BFDFED1D7A37EEC77A27EE076ADFED48
:101288001E4ADFED1E6ADFED1E7AE6EE246A67EE7F
:10129800064AE6EE267AB7EE006AA4EEA77AF6EEDC
:1012A800006A36EE476AF8EE007A27EE277A66EE8D
:1012B800266A84E7DFED097A37EEC77ADDE7B0EE14
:1012C800677A3DE7F0EE407A24E7B0EE677AC2E746
:1012D800F0EE477AAAE700BF27D4D236DB0F4940A1
:1012E800DB0FC940E4CB1641DB0F49C0E4CB16C184
:1012F800DB0FC93FDB0FC9BF92E741B99730083C04
:1013080015A82ABEF304353F0000008070B40668B3
:101318008E4217D90139751E002311F8014F082292
:10132800634013F0800F4FEA430318BF83F0D503DF
:10133800013ADBB2F5D18D42EFD1721C02603370F5
:1013480070BC70470023F8E710B44C09012250F82C
:10135800243001F01F0102FA01F10B4340F8243058
:101368005DF8044B704700BF4B0901F01F0150F8AE
:101378002320012303FA01F1114214BF184600206B
:10138800704700BF074A084B10781B78074A83420A
:1013980096BFC31AC3F18003002012681844104492
:1013A800704700BF705F0020EC5E0020585200209C
:1013B800064A074B10781B7883428ABFC3F1800323
:1013C800C01AC018C0F17F00704700BF705F0020CE
:1013D800EC5E0020F8B584894FF6FF764FF47A74F6
:1013E8002BB311B30F78013101E0B44217D005894E
:1013F800013CAD07A4B2F8D507734FF47A7402E044
:10140800BCB2B4420BD00589ED0704F1FF37F7D51C
:10141800057BEDB20AB115700132013BE0E710F02F
:1014280079FA003018BF0120F8BDFF27DFE7012057
:10143800F8BD00BF30B5134C237883B01BB9012029
:10144800237003B030BD1049052200230D688DF8C4
:1014580004208DF8053000BFA86810F0DBF86A4654
:1014680001A902236868FFF7B5FFA86810F0D8F84B
:1014780000BF9DF8013003F0010383F001002370E1
:1014880003B030BD0F590020FC58002070B5064C41
:101498000646256803E023685B1BB34203D8FFF7C1
:1014A800C9FF0028F7D070BD54650020F0B51F4C67
:1014B80083B0277800234FF0030E00930E4615469D
:1014C8008DF804308DF800E06FB3030E8DF801300D
:1014D8000DF10203010C020A9870197006205A7067
:1014E800FFF7D4FFE8B100BF114F3B68986810F0D0
:1014F80091F823783A68002B14BF05230423694622
:1015080050680022FFF766FF3B68324600215868A2
:101518002B46FFF75FFF3B68986810F081F800BF23
:10152800284603B0F0BD0DF10103D3E70E590020A2
:10153800FC58002008B540F2E93300E09BB102896D
:10154800013B12F0020F9BB2F8D0017340F2E9336D
:1015580000E043B10289013B12F0010F9BB2F8D0C1
:10156800007BC0B208BD10F0D5F9C0B208BD00BFFD
:1015780038B504460D4600BF806810F04BF8294680
:101588006068FFF7D7FFA06810F04AF800BF38BDC1
:101598002DE9F04F89B0B2F1000A0290049103934B
:1015A80040F3C5800B46002201EB8A0153F8040B77
:1015B8008B420244FAD1039B0592002B00F0AF80C6
:1015C800059B002B7CD05E4B059A1B68DFF8889141
:1015D80000920099DAB25118B1F5807F8CBFC2F53C
:1015E8008072009A0192574A92689A4240F2828029
:1015F800554A1178002206928DF81C2002228DF897
:101608001820002960D01A0E8DF819200DF11A0241
:101618001C0C190A9370147051700620FFF736FFDE
:101628000621D9F80000FFF7A3FF484A01231370E9
:1016380000BFD9F8003098680FF0ECFF424BD9F89A
:1016480000201B785068002B06A90CBF0423052333
:101658000022FFF7BFFE0024049D029E019FA346BF
:1016680029684FEA840800220B46013471B1B94257
:101678002DD2D9F8000031684068FFF7ABFE2A6820
:10168800336813443360BF1AC5F800B0A24505F1AA
:10169800040506F10406E3D1D9F8003098680FF084
:1016A800BFFF00BF264B019900981B68421A0092A1
:1016B800234A0B441360039A4AB3009A002A88D13C
:1016C800059809B0BDE8F08F0DF11902A0E7029C5A
:1016D800D9F8003054F80810586800223B46FFF744
:1016E80079FE54F808202B683A44DF1B44F8082098
:1016F8002F60D1E70598009C1549164A001B0590F4
:10170800059800230B70137009B0BDE8F08F059B96
:10171800009A9B1A0593059809B0BDE8F08FFFF76A
:1017280089FE00287FF44CAF039B0593C8E7039C10
:101738001CB9FFF77FFE0594C2E700230593BFE7B6
:1017480058520020901900200E5900200F590020EF
:10175800705F0020EC5E0020FC58002070B5104D32
:10176800104E2B7831788B4284B016D00E4A0392F3
:101778001A4402928CBF0C46CA1A04A98CBFC3F142
:1017880080020024012341F8102D02A802220194AE
:10179800FFF7FEFE002333702B7004B070BD00BF4E
:1017A800EC5E0020705F0020F05E0020F0B5124B68
:1017B8009D6885B00DB905B0F0BDED0A14D00027BD
:1017C80004AE7C196410E00210226946FFF76EFE31
:1017D8000F2809DD6B4653F8042B01320AD1B342B6
:1017E800F9D12546AF42ECDBFFF7B8FF034BED021A
:1017F8001D60E0E7671CF5E79019002058520020AB
:1018080070B5194C194D23782978994284B027D09E
:10181800174A03921A44029234BF0E46CA1A04A900
:1018280034BFC3F180020026002341F8102D02A81E
:1018380002220196FFF7ACFE23781844C0B20306D3
:101848002B7848BF80F080008342207002D00020AF
:1018580004B070BD002301202B70237004B070BD4C
:10186800012004B070BD00BFEC5E0020705F002056
:10187800F05E002010B50C4C45F20820FFF706FE7C
:1018880020680621FFF774FE084B20680122C72153
:101898001A70FFF76DFE06480649074A00230370D1
:1018A8000B70136010BD00BFFC5800200F590020BA
:1018B800705F0020EC5E002058520020F0B55B4BB2
:1018C8005B4A97B01968914200AF00F0A38059496C
:1018D800594A00234FF47000C1F888003B607B60D0
:1018E800136843F48033136003E03B68B3F5A04FFB
:1018F80009D0136803F400337B603B6801333B6015
:101908007B68002BF1D04C4B1B6813F4003318BFD5
:1019180001237B607B68012B52D0464C464B474ADB
:10192800E260474A596A11605A6A42F080725A6204
:101938005A6942F4FC025A610025032207F10801A2
:10194800012341F6FF764FF09040FD60BE603A7388
:10195800BB731AF0CFFF4FF6FF7307F10801394840
:10196800BB601AF0C7FF07F108013748374E1AF075
:10197800C1FF07F1080136481AF0BCFF07F108015A
:1019880034481AF0B7FF07F1080133481AF0B2FFDC
:1019980007F108001BF008F8BB683049304AA1FB82
:1019A800031330499B0CF0204FF0070E5C370B6097
:1019B800566084F823009560C2F800E0BD46F0BD8B
:1019C800294A1D4B122111605A685A605A685A6098
:1019D8005A6842F480625A605A6822F47C125A604B
:1019E8005A6842F4E8125A601A6842F080721A6023
:1019F8001A689201FCD559680F4A21F00301596011
:101A0800596841F002015960536803F00C03082B30
:101A1800FAD182E700221A6062B6144B1B6883F37E
:101A28000888134B1B689847FEE700BFFC9F0020FF
:101A3800EFBEADDE00ED00E0001002400005FA0543
:101A48006866002000040048000800483F190100AB
:101A5800000C0048001000480014004883DE1B43B7
:101A680010E000E0586500200020024000D8FF1F69
:101A780004D8FF1F70B50F4C0F4DC0EBC00004EB2E
:101A88008004686926693043686182B09209667B80
:101A9800A1600025012101A863618DF804608DF81B
:101AA80005208DF806508DF807101AF0EDFE02B0EB
:101AB80070BD00BF341A002000100240074BC0EB75
:101AC800C00030B403EB8000054C056963692B4303
:101AD80063610176427630BC704700BF341A00203B
:101AE800001002402DE9F04F5E4C54F8204083B0BE
:101AF800002C71D0A66D984691465B4B72682265A2
:101B0800A160236004F15E014FF4807304F5AF72A5
:101B18006161A261E36023610746307E2CF078F8AA
:101B2800F068A8B1514B00215A68904203F11C0398
:101B380000F0928001310C29F6D100207A1CD2B233
:101B48000C21FFF7BBFF236DF26862632433E36463
:101B5800B068D8B1454B00215A68904203F11C0384
:101B680078D001310C29F7D100257A1CD2B20B218B
:101B78002846FFF7A3FF2346F27E3D492846FFF794
:101B880079FF236DB268A2632833A36494F85D00DB
:101B98000FF0D8F8054694F85C000FF0D3F818F069
:101BA800080F824696F819B01AD0CDB118F0110F67
:101BB8004FF00B0307F1010714BF4E213E21EF71CF
:101BC8005A46AB7128460FF097F918F0010F45D027
:101BD800636B5BB3A36B4BB3204603B0BDE8F08FD8
:101BE80018F0010F0CBF4FF02E084FF04E0819F0F7
:101BF800020F09D045B10B227B1CAA71EB71284654
:101C08005A4641460FF078F919F0010FE0D0BAF1C1
:101C1800000FDDD001370C238AF807705A46414679
:101C28008AF8063050460FF067F9D1E7337FB27E65
:101C38008DF804209B090021012201A88DF80530A8
:101C48008DF806108DF807201AF01EFE204603B006
:101C5800BDE8F08FCDB288E7C8B26FE728460FF02D
:101C6800D9FCB5E7A82C002034300308341A00202A
:101C7800BD05000800B97047F0B595B005462CF0D1
:101C880065FB6E4EC368026832600446002B00F0A4
:101C9800C38028460FF056F8694B186018B12922FE
:101CA80000238271C371227A664D2E210FF024F928
:101CB80030680BF0E9FC2BF0ABFF3068624A038810
:101CC80023F001031B041B0C038014A91E232B8083
:101CD80001270F230025138021F84C7D2D23029323
:101CE800ADF80C50ADF80650ADF80E502CF0DCFAFB
:101CF800E379ADF8145060229907ADF816500695AF
:101D0800ADF81C50ADF81E50ADF82050ADF822507B
:101D1800049200F1838013F0010F14BF0222002205
:101D28004FF48073ADF81470ADF81C20ADF8203076
:101D3800002304AA6179306806930BF013F9306820
:101D480061792CF091FA3068436C43F400434364A2
:101D580003889BB243F080030380E3799B0768D52F
:101D68006179026A04238B4022EA03020262026A52
:101D7800134303623268354F13889BB243F0010363
:101D88001380207C00222921FFF798FE3049207C0F
:101D980000236022FFF76EFEE06838601AF0E0FC6E
:101DA800386803684FF6FE72134003601AF0D8FCD7
:101DB80009A81AF0A7FC33686279264938680A919D
:101DC80034331344099380221023002509A940F2D3
:101DD8002A3E0E920B934FF400724FF400530D9568
:101DE8001095139511950F921293ADF830E01AF0F3
:101DF80097FC627933680C2A98BF1749D86898BF4E
:101E080031F812503A6815490543DD60136801201E
:101E180043F002031360087015B0F0BD13F0010F12
:101E280014BF08222A460423ADF81E20ADF8163048
:101E38007EE7012261791AF0A3FB9BE7BC470020EB
:101E4800A81D0020B2470020B0470020B847002056
:101E5800D1040008B4380020B0540308B447002067
:101E68000348D0F83C3113B100F59A701847704711
:101E7800341A00200348D0F8203113B100F58C70D3
:101E880018477047341A00200348D0F804310BB1C2
:101E9800FC301847704700BF341A00200348D0F8B8
:101EA800E8300BB1E0301847704700BF341A002003
:101EB8000348D0F8CC300BB1C4301847704700BF86
:101EC800341A00200348D0F8B0300BB1A8301847B6
:101ED800704700BF341A00200348D0F894300BB183
:101EE8008C301847704700BF341A00200248836FAF
:101EF8000BB1703018477047341A00200248C36D80
:101F08000BB1543018477047341A00200248036C4C
:101F18000BB1383018477047341A00200248436A1A
:101F28000BB11C3018477047341A002002488368E8
:101F380003B11847704700BF341A0020F0B53E4C73
:101F4800059D00EB800004EB80046468002C71D0D0
:101F58003A4E49004FF42040CFB27060A16909049D
:101F680054D46068DFF8E0E047F4903100EA0E00EE
:101F780001434FF420406160706003E0411E002877
:101F880048D00846A1698907F8D54FF42040A262D5
:101F9800706003E0421E00283CD01046A269520639
:101FA800F8D5274A6168DFF8A0E0706042EA03428A
:101FB800174301EA0E0217436760C3B1013BDBB266
:101FC80001332B44A0694FF4204210F0040002F1C1
:101FD800FF3207D1511C26D0A06910F0040002F18D
:101FE800FF32F7D0626A05F8012B9D42EAD14FF41F
:101FF8002040706002E0431E60B11846A3699B064A
:10200800F9D520237060E3610120F0BD411E08B1BD
:102018000846A3E70B4A138801339BB24FF0FF3100
:1020280013807160F0BD074972600B8801339BB261
:102038000B80F0BD2046F0BDC4640020A81D002020
:102048000024000284320020009800FC2DE9F04FA3
:1020580089B090F855300490002B40F06782534BBC
:102068001B7A002B00F0A480049B103305931846BC
:1020780004994A69138823F040031B041B0C13803E
:1020880013889BB223F0380343F038031380138876
:102098009BB243F04003138091F84E201A210FF0B1
:1020A8004BFC0BF061FC04460BF05EFC8442FBD059
:1020B800049A5069038823F040031B041B0C038017
:1020C800038823F038031B041B0C038003889BB28E
:1020D80043F040030380137C012B4CD0022B1346A2
:1020E8005BD1936913B11A689B88138540F2E93371
:1020F80002E0002B00F0C3820289013B12F0020FBC
:102108009BB2F6D0C323037340F2E93302E0002BFD
:1021180000F0B5820289013B12F0010F9BB2F6D0A4
:10212800037B049B58690627838906AD4FF47A73AD
:102138004FF6FF714FF0FF0E04E0013B9BB28B425C
:1021480000F07D8202899207F7D580F80CE04FF401
:102158007A7303E0A3B28B4200F071820289D6073A
:1021680003F1FF34F6D5027BD2B20DB12A700135E6
:10217800013FE7D165E292F914001346421C0CD0E6
:1021880002280ADC597D06AB009343220623FFF799
:10219800D5FE002840F05B82049BB3F93A305BB26D
:1021A800013300F01A8209B0BDE8F08FA81D0020A5
:1021B8000499BC4C4A69BC4F1388DFF8F8A223F095
:1021C80040031B041B0C138013889BB223F03803B5
:1021D80043F03803138013889BB243F04003103157
:1021E80013800591084680226B210FF0A5FB9623EA
:1021F800AE48DFF8C4C24FF010084FF47A759E4617
:10220800DAF80430C3F30803002B40F07381EFF3CE
:102218001183002B40F06E812168826800BF23681B
:102228009942F9D13E6805FB06F39B1AB3FBF6F316
:1022380005FB013101260391DAF80430C3F30803E2
:10224800002B40F01181EFF31183002B40F00C813B
:102258002368816800BF22689342F9D1D7F800B09B
:1022680005FB0BF2521AB2FBFBF205FB0323039AA0
:102278009B1AB3F57A7FDFD3BEF1010EC0D10322DA
:1022880068210598DFF82CA20FF056FB96238748A3
:10229800DFF824C24FF010084FF47A759E46DAF83A
:1022A8000430C3F30803002B40F00881EFF31183D7
:1022B800002B40F003812168826800BF236899429F
:1022C800F9D13E6805FB06F39B1AB3FBF6F305FB51
:1022D800013101260391DAF80430C3F30803002B17
:1022E80040F0A580EFF31183002B40F0A080236815
:1022F800816800BF22689342F9D1D7F800B005FB86
:102308000BF2521AB2FBFBF205FB0323039A9B1A4A
:10231800B3F57A7FDFD3BEF1010EC0D103226B2162
:1023280005980FF009FB0BF01FFB04460BF01CFB94
:10233800001B0E28FAD910226A2105980FF0FCFA22
:102348000BF012FB04460BF00FFB001B0E28FAD90A
:1023580000226C2105980FF0EFFA0BF005FB0446FC
:102368000BF002FB001B0E28FAD9049B059893F882
:10237800502019210FF0E0FA0BF0F6FA04460BF0A2
:10238800F3FA001B0E28FAD918221B2105980FF022
:10239800D3FA0BF0E9FA04460BF0E6FA001B0E2814
:1023A800FAD910221C2105980FF0C6FA0BF0DCFAB6
:1023B80004460BF0D9FA001B0E28FAD9102237214F
:1023C80005980FF0B9FA0BF0CFFA04460BF0CCFAE7
:1023D800001B0E28FAD90122382105980FF0ACFA13
:1023E8000BF0C2FA04460BF0BFFA001B0E28FAD90C
:1023F800049B5A69138823F040031B041B0C1380A9
:10240800138823F038031B041B0C138013889BB21A
:1024180043F0400313800BF0A7FA04460BF0A4FA2C
:102428008442FBD0224A05980123137220E6EFF379
:10243800118988F3128881680368DB0344BFCCF8EC
:10244800006081682368DCF800205FFA89F989F365
:102458001188D7F800901A4405FB09F35B1AB3FBFF
:10246800F9F305FB023351E7EFF3118988F312887A
:1024780081680368DB0344BFCCF800608168236887
:10248800DCF800205FFA89F989F31188D7F8009001
:102498001A4405FB09F35B1AB3FBF9F305FB023396
:1024A800E5E600BF546500205865002010E000E014
:1024B800A81D002000ED00E050650020EFF3118218
:1024C80088F3128886680368D90303D50123CCF8FA
:1024D800003086682368DCF80010D2B282F31188D5
:1024E8003A68194405FB02F39B1BB3FBF2F305FBA7
:1024F8000131EEE6EFF3118288F3128886680368EB
:10250800D90303D50123CCF8003086682368DCF8AA
:102518000010D2B282F311883A68194405FB02F31D
:102528009B1BB3FBF2F305FB013183E61D09013D5B
:10253800022D03F00F0300F2AA805E4A32F815005C
:1025480040FA03F2D40740F1A280012404FA03F30D
:10255800013B18402FF054F9574B584A5B5D18441B
:1025680012EBC00500F0938052F83000AF88038A60
:102578003B407FF474AD00F138425149EB71920A47
:102588008A5C02F01F0352092021022A04FA03F38D
:10259800A97100F08580032A74D0012A00F0858093
:1025A800002306A9079306971AF0A4F90499454B46
:1025B80041F80C3F284623F021FBAB88B3FA83F39C
:1025C800C3F11F03581C3FF44AAD012202FA03F37A
:1025D8003D490A6813430B6041E5049B93F9383081
:1025E80001337FF4E0AD0A26322022F0D5FF4FF404
:1025F800FA750BF0B9F904460BF0B6F9001BB0F503
:102608007A7FF9D3013DF4D107202BF0FFFE4FF478
:102618007A750BF0A9F904460BF0A6F9001BB0F582
:102628007A7FF9D3013DF4D1013EDDD12749284B0A
:102638002848294A0860DA6009B0BDE8F08F0FF031
:1026480069F9049B9B6913B11A689B8893619DF88B
:1026580018409DF81A509DF81B309DF819109DF8E8
:102668001C009DF81D2041EA042143EA0523049C2F
:102678001BB242EA002263872187A2878FE50FF009
:1026880049F94EE5154AD1690B43D36188E70499A6
:102698000C4B41F80C3F002023F0B0FA012397E7D8
:1026A8000E4A91690B4393617AE70C4A51690B43CF
:1026B800536175E7945403089C540308A848002004
:1026C8006C5903083504000800040140FC9F0020F1
:1026D80000ED00E0EFBEADDE0400FA050010024098
:1026E800F0B5037C012B85B0044663D0022B67D17B
:1026F800836913B11A689B881385606940F2E933CE
:1027080001E0002B6CD00289013B12F0020F9BB252
:10271800F7D0C323037340F2E93301E0002B5FD005
:102728000289013B12F0010F9BB2F7D0037B60696D
:102738004FF0060E838902AE4FF47A734FF6FF719D
:10274800FF2703E0013B9BB28B423CD002899507EF
:10275800F8D507734FF47A7302E0ABB28B4232D0EC
:102768000289D20703F1FF35F7D5027BD2B20EB149
:1027780032700136BEF1010EE8D1A36913B11A68AF
:102788009B8893619DF80C009DF808609DF80910DE
:102798009DF80A509DF80B209DF80D3041EA06215E
:1027A80043EA002342EA0522012021876287A387A2
:1027B80005B0F0BD90F91400431C01D0022805DDD6
:1027C800002005B0F0BD0FF0A5F8D6E702AB617D9B
:1027D800009343220623FFF7B1FB0028D2D1EFE78D
:1027E8000FF098F8A3E700BFF0B5037A012B85B086
:1027F800044663D0022B67D1036913B11A689B881A
:102808001385E06840F2E93301E0002B6CD00289BF
:10281800013B12F0020F9BB2F7D0BB23037340F2C7
:10282800E93301E0002B5FD00289013B12F0010F70
:102838009BB2F7D0037BE0684FF0060E838902AEA7
:102848004FF47A734FF6FF71FF2703E0013B9BB209
:102858008B423CD002899507F8D507734FF47A73F9
:1028680002E0ABB28B4232D00289D20703F1FF35C6
:10287800F7D5027BD2B20EB132700136BEF1010E2D
:10288800E8D1236913B11A689B8893619DF80C00FD
:102898009DF808609DF809109DF80A509DF80B20D6
:1028A8009DF80D3041EA062143EA002342EA052259
:1028B8000120E1822283638305B0F0BD90F90C000A
:1028C800431C01D0022805DD002005B0F0BD0FF043
:1028D80021F8D6E702AB617B00933B220623FFF782
:1028E8002DFB0028D2D1EFE70FF014F8A3E700BFC3
:1028F800B0F1FF3F56D0022854DCF0B4324C00EB64
:10290800800004EB80004468002C5BD02F4E490007
:102918004FF42040CDB27060A169090444D46068C6
:102928002B4F45F08071384041F4903101434FF40A
:1029380020406160706003E0411E002838D00846DE
:10294800A1698F07F8D54FF42040A262706002E0B9
:10295800421E68B31046A2691106F9D562681C497F
:1029680045F0007545F480350A4015434FF4204082
:102978006560706002E0421ED0B11046A2699207FD
:10298800F9D54FF42040A362706002E0431E78B18D
:102998001846A3699B06F9D520237060E3610120DE
:1029A800F0BC704700207047411E08B10846B3E7E5
:1029B800084A138801339BB24FF0FF3113807160CE
:1029C800F0BC70472046FBE7C4640020A81D002027
:1029D800009800FC843200202DE9F04F87B090F871
:1029E80055300290002B40F0C281029A137C1032BD
:1029F800012B1046039200F01482022B00F0B281E2
:102A0800BD4CBE4EDFF8FC92BD48DFF8FCE24FF04B
:102A1800640A4FF0100C4FF47A75D9F80430C3F3F8
:102A28000803002B40F0F380EFF31183002B40F0F4
:102A3800EE802168826800BF23689942F9D137681F
:102A480005FB07F39B1AB3FBF7F305FB01310127DD
:102A58000191D9F80430C3F30803002B40F09D809E
:102A6800EFF31183002B40F098802368816800BF42
:102A780022689342F9D1D6F800B005FB0BF2521A3E
:102A8800B2FBFBF205FB0323019A9B1AB3F57A7F8D
:102A9800DFD3BAF1010AC0D1029D297C012900F0D7
:102AA800B781022900F04A81029B012993F850302E
:102AB80000F05081022900F03B81DFF848929048ED
:102AC800DFF844E24FF00F0A4FF0100C4FF47A751C
:102AD800D9F80430C3F30803002B40F0B480EFF3B7
:102AE8001183002B40F0AF802168826800BF236803
:102AF8009942F9D1376805FB07F39B1AB3FBF7F343
:102B080005FB013101270191D9F80430C3F308030B
:102B1800002B5FD1EFF31183002B5BD12368816811
:102B280000BF22689342F9D1D6F800B005FB0BF23A
:102B3800521AB2FBFBF205FB0323019A9B1AB3F569
:102B48007A7FE1D3BAF1010AC2D1029C237C94F8BE
:102B58004E20012B00F06E81022B00F0D780012B54
:102B680000F0DC80022B00F0B280012B00F0B9806D
:102B7800022B00F09880012B00F09F80022B7ED062
:102B8800012B00F08680022B04D103980122382102
:102B98000EF0D2FE07B0BDE8F08FEFF311888CF38A
:102BA800128881680368DB0344BFCEF8007081682F
:102BB8002368DEF800205FFA88F888F31188D6F8D1
:102BC80000801A4405FB08F35B1AB3FBF8F305FB16
:102BD800023359E7EFF311888CF312888168036890
:102BE800DB0344BFCEF8007081682368DEF800205C
:102BF8005FFA88F888F31188D6F800801A4405FB34
:102C080008F35B1AB3FBF8F305FB023395E7EFF320
:102C180011828CF3128887680368D90303D50123CE
:102C2800CEF8003087682368DEF80010D2B282F34D
:102C380011883268194405FB02F3DB1BB3FBF2F37E
:102C480005FB013103E7EFF311828CF312888768E3
:102C58000368D90303D50123CEF8003087682368B9
:102C6800DEF80010D2B282F311883268194405FBED
:102C780002F3DB1BB3FBF2F305FB013142E71A4613
:102C8800372103980EF058FE029B1B7C012B7FF422
:102C98007AAF02983822417D90F91400FFF728FE98
:102CA80007B0BDE8F08F18221C2103980EF044FEEF
:102CB800029B1B7C012B7FF461AF029C022337220D
:102CC800617D94F91400FFF713FE237C58E718225E
:102CD8001B2103980EF030FE029B1B7C012B7FF416
:102CE80047AF029C18231C22617D94F91400FFF75A
:102CF800FFFD237C3FE700BF546500205865002096
:102D080010E000E000ED00E0506500201A21039873
:102D18000EF012FE237C012B7FF424AF029C1823B3
:102D28001B22617D94F91400FFF7E2FD237C1CE768
:102D38001A46192103980EF0FFFDBEE66B21032207
:102D480003980EF0F9FD297C029B012993F8503075
:102D58007FF4B0AE02981922417D90F91400FFF774
:102D6800C7FDAAE680226B210EF0E6FD48E61D09A4
:102D7800013D022D03F00F0365D83F4A32F81500D4
:102D880040FA03F2D4075ED5012404FA03F3013BA9
:102D980018402EF035FD394B394A5B5D184412EB6B
:102DA800C00550D052F83000AE88038A33407FF413
:102DB8001CAE00F138423349EB71920A8A5C02F08A
:102DC8001F0352092021022A04FA03F3A9714DD0E6
:102DD800032A46D0012A3FD0002304A9059304966C
:102DE80019F088FD0299284B41F80C3F284622F03B
:102DF80005FFAB88B3FA83F3C3F11F02501C3FF4FD
:102E0800F4AD01239340214A11680B431360ECE5AC
:102E1800697D95F9140003236B22FFF769FD297C6E
:102E280042E602988023417D90F914006B22FFF757
:102E38005FFDE5E51346617D94F914001A22FFF75A
:102E480057FD237C8BE602990F4B41F80C3F00207D
:102E580022F0D4FE0123D6E70D4A51690B43536192
:102E6800BAE70B4AD1690B43D361B5E7084A9169C0
:102E78000B439361B0E700BF945403089C540308C4
:102E8800A84800206C5903083504000800040140D4
:102E9800001002401749184B184A194810B4D1F8C5
:102EA800884044F47004C1F888401C6844F0010468
:102EB8001C605C6822405A601A6822F0847222F40E
:102EC80080321A601A6822F480221A605A6822F442
:102ED800FE025A60DA6A22F00F02DA621A6B0024E4
:102EE80010404FF0006218639C608A605DF8044BE4
:102EF800704700BF00ED00E0001002400CC07FF8F2
:102F0800CCFC00FF2DE9F04F95B0B0F908500D81C9
:102F1800EDB2442D00AF0C46904600F042840646C0
:102F280043D9812D00F07B8300F29880542D00F066
:102F3800CC8040F2D6806E2D00F00184802D40F0C8
:102F4800D380764B93F800A00AF1020A1AF0FF0A20
:102F580000F09780724BDFF8F481724EDFF8F0B121
:102F68009A4403F101090A2516E0322D01F0218364
:102F7800A5F13C00C0B2132841F222830023226845
:102F8800511C216015702268D14502F101012160B0
:102F9800137076D019F8015B0A2DE6D1BBF8003022
:102FA800FF2BA8BFFF23DBB2E9E7052D00F0E7837D
:102FB80020D8022D00F0818040F21083032D00F00C
:102FC800B583042D40F09080574920462A46FDF7E6
:102FD800BFFE00212046FDF7EBFE22680021531CAE
:102FE8000125236028462B46543711706381BD465E
:102FF800BDE8F08F242D5ED040F2A682282D00F087
:103008005783382D70D10A68484B0125511C21601F
:1030180015702268052150192060117022680A2154
:103028005019206011702268002150192060117019
:10303800226819785019206011702268597850193F
:103048002060117022689978531923602B461170FB
:10305800284654376381BD46BDE8F08FA02D18D0AF
:1030680040F29182B82D00F05F83FE2D3CD1304DA7
:1030780005F1080635F8021B2046FDF799FEB54212
:10308800F8D101252B46284654376381BD46BDE853
:10309800F08F284B08461968FDF772FE264B20462C
:1030A8001968FDF76DFE254B196820460125FDF7C7
:1030B80067FE2B46E7E7224BF6E704222149204624
:1030C8000125FDF745FE2B46C2E70B6800215A1C77
:1030D8002260197022680125531923602B4611704C
:1030E800B6E7522D3FF479AF214628460EF0B4FDDD
:1030F80003460028C5D1742D00F08382772D29D18D
:103108003268716891421EBF531C336011780E4AB1
:1031180008BF1946204612F08BF9B2E76940002033
:103128005C30030894240020EA330020FB3C002094
:103138008C400020ACF7FF1FB0F7FF1FB4F7FF1F4C
:10314800443E0020945D0308D54201086766666620
:10315800BC240020F52D01F0F482472D00F04E83A9
:10316800292D326801F0B382392D01F09D82212D7D
:1031780001F07A8270680B3D811AEF2D00F29C8471
:103188000FF2040E5EF825F075440008C13A0008F5
:10319800C13A0008C13A0008C13A0008C13A00081B
:1031A800C13A0008C13A0008C13A0008C13A00080B
:1031B800C13A0008C13A0008C13A0008C13A0008FB
:1031C800C13A0008C13A0008C13A0008C13A0008EB
:1031D800C13A0008C13A0008C13A0008C13A0008DB
:1031E800C13A0008C13A000801440008C13A000881
:1031F800DF430008C13A0008B5430008C13A000897
:10320800C13A0008C13A00087B450008C13A0008E5
:1032180005450008C13A0008D3440008C13A00082F
:10322800AD440008C13A0008A3450008C13A0008A7
:103238005D430008C13A000809430008C13A000884
:10324800C13A0008C13A0008C13A00088B300008AA
:10325800C13A0008DD420008C13A0008C13A000836
:1032680077420008C13A00081D420008C13A000828
:10327800C13A0008C13A0008C13A000811420008E2
:10328800C13A0008C13A0008C13A0008D141000813
:10329800C13A000883410008C13A0008C13A000851
:1032A80043410008C13A0008C13A0008C13A000881
:1032B800C13A0008C13A0008C13A0008C13A0008FA
:1032C800D5400008C13A000853400008C13A000838
:1032D800713F0008C13A0008813E0008C13A000861
:1032E8002B400008633E0008473E0008C13A00082A
:1032F800C13A0008C13A0008C13A0008C13A0008BA
:10330800C13A0008C13A0008C13A0008C13A0008A9
:10331800C13A0008C13A0008C13A0008C13A000899
:10332800C13A0008C13A0008C13A0008C13A000889
:10333800C13A0008C13A0008C13A0008C13A000879
:10334800C13A0008C13A0008C13A0008C13A000869
:10335800C13A0008C13A0008C13A0008C13A000859
:10336800C13A0008C13A0008C13A0008C13A000849
:10337800C13A0008C13A0008C13A0008C13A000839
:10338800C13A0008C13A0008C13A0008C13A000829
:10339800C13A0008C13A0008C13A0008C13A000819
:1033A800C13A0008C13A0008C13A0008C13A000809
:1033B800C13A0008C13A0008C13A0008C13A0008F9
:1033C800C13A0008C13A0008C13A0008C13A0008E9
:1033D800C13A0008C13A0008C13A0008C13A0008D9
:1033E800C13A0008C13A0008C13A0008C13A0008C9
:1033F800C13A0008C13A0008C13A0008C13A0008B9
:10340800C13A0008C13A0008C13A0008C13A0008A8
:10341800C13A0008C13A0008C13A0008C13A000898
:10342800C13A0008C13A0008C13A0008C13A000888
:10343800C13A0008C13A00081D3E0008C13A000818
:10344800013E0008D73D0008C13A0008C13A00080B
:10345800C13A0008C13A0008C13A0008C13A000858
:10346800C13A0008C13A0008C13A0008C13A000848
:10347800C13A0008C13A0008C13A00085D3D000899
:10348800C13A0008253D0008C13A0008833C0008FD
:10349800693C0008BB3D0008C13A00084F3C0008E1
:1034A800C13A0008273C0008C13A0008C73B000899
:1034B800C13A0008973B0008C13A0008C13A000821
:1034C8006D3B0008073B0008F33A0008CB3A0008B8
:1034D800A33A0008793A0008C13A0008C13A00083E
:1034E800C13A0008C13A0008C13A0008C13A0008C8
:1034F800C13A0008C13A0008C13A0008C13A0008B8
:10350800C13A0008C13A0008C13A0008C13A0008A7
:10351800C13A0008C13A0008593A0008C13A0008FF
:10352800C13A0008013A0008C13A0008C13A000847
:10353800C13A00089D390008C13A0008C13A00089C
:10354800C13A000883390008202D7FF4CDAD0B68FF
:10355800984D591C6A7821601A7023682A78591C7A
:1035680021601A702368AA78591C21601A70298969
:103578002046FDF71DFC23686A79591C21601A70E2
:103588002268A9792BE5822D7FF4AEAD0B688A4AB3
:103598008A4D1178874A581C206019701189204675
:1035A800FDF706FC864B22681B88FF2B02F1010100
:1035B800A8BFFF2321601370A96881F3100189B2A5
:1035C8002046FDF7F5FB296801F30F0189B2204673
:1035D800FDF7EEFB7B4B2268197800E5012D7FF49F
:1035E80083AD0B680022591C21601A7023685A1C8D
:1035F80022601D7022682521531C23602B46117000
:1036080026E53268716891421EBF531C33601178F9
:103618006D4A08BF1946204611F00AFF31E56B4B89
:103628001E78033616F0FF063FF42BAD684BDFF823
:10363800C4811E4403F1010A4FF00A0920E0B9F1E0
:10364800500F00F0B387B9F1320F00F0CF87A9F11E
:103658003C00C0B2132840F2E787002529462368BA
:103668005A1C2260204683F80090FDF7A1FB2946EA
:103678002046FDF79DFB56453FF403AD1AF8019B24
:10368800B9F10A0FDBD1534B9D68196805EB850525
:103698004FF6FF736D009D42A8BF1D469942A8BF13
:1036A800194625EAE57521EAE171ADB289B2D6E796
:1036B8000B68DFF84491484E591C022221601A70A9
:1036C80023684FF006085A1C226083F8008023689C
:1036D8000A22591C21601A70236801255A19226090
:1036E8001D70B9F800102046FDF762FBB9F802100A
:1036F8002046FDF75DFB23685A19226083F8008095
:1037080023685022591921601A7023680022591918
:1037180021601A7031882046FDF74AFB71882046DF
:10372800FDF746FB2B4693E42C4BBDE40B685A1C73
:103738000A601D700B685A1C0A601D704DE4204B0E
:103748000A681B881D4DFF2BA8BFFF23511C216051
:103758001370A96881F3100189B22046FDF728FB90
:103768001F4B20461988FDF723FB296801F30F0139
:1037780089B220460125FDF71BFB2B4668E40B2286
:1037880018492046FDF7E4FA082217492046FDF7B4
:10379800DFFA0125072215492046FDF7D9FA2B46FD
:1037A80056E4002A3FF46DAC114B136001252B46FB
:1037B8004EE400BF604300209E410020704300207B
:1037C8008841002034370020354301086940002033
:1037D8006C300308482400207C240020B8450020D1
:1037E800303700209C5D0308A85D0308B45D03081A
:1037F800351C01088C24002024610020726835687B
:103808007B623046551BFDF779FA052D38627B6AD5
:1038180001F216808026B346012594E80600521A64
:10382800103AB242B8BF1FFA82FBC04A396A92689E
:103838003A61521A9345396A7B622046FA6088BF1A
:103848001FFA82FBFDF79CFA7B6A002B00F0D687F3
:10385800002D40F055872368C7F800D05D71C0B0CF
:103868000533C7F808D0FB61BBF1000F01F0D78022
:103878003B6A3A69934281F0CE80AA463E6A7D62ED
:103888007C6080255446FB681C1BA84BB4F5807FE0
:1038980028BF4FF480749B6832199A4288BF9C1BDA
:1038A800FDF75CFF2246BC6830462146FDF7FEFD69
:1038B800F969B86104EB000C0B787B61644530D280
:1038C800DFF898920CF1FF3C04F1FF3E1EF8013F2F
:1038D80009EB830219F823405688FCB100234FF402
:1038E800004204F1FF3816424FEA520202D008782B
:1038F800284308706D0806D10AF1010A4D701FFAB5
:103908008AFA01318025D34505D8E645C0F0A3865B
:103918004345C0F2A08601339C42E4D1F445D5D199
:10392800F9617B6ABA6913449BB2D3457B6206D9B5
:103938007B6A3A6A1C46D6183B699E42A3D37C68C8
:10394800802D1CBF0AF101031FFA83FA0AF1020154
:1039580089B22046FDF72CFA2368796A01255A199D
:10396800226020461D70FDF723FA23685344236024
:103978002B46D7F800D0FFF76BBB6D4B1B78DB07E6
:1039880000F19A80012508F015FD08F0EFFE2B469E
:10399800FFF75EBB3046FDF7C9F93368B8851A46AC
:1039A800591C316012F8021B326087F82E105A78C1
:1039B80087F82F20DA1C32609A7887F830201A1D91
:1039C8003260DA7887F831205A1D32601B7987F81F
:1039D800323007F12C000023BB86FDF7FFF8554A6B
:1039E800554B1268801A4FF0010561F10001C3E9D7
:1039F80004012B46FFF72CBB531C336013780F2BA5
:103A08005AD8911C3160C3EBC3034C495078C85451
:103A1800D01C30600B4491785970111D3160D178F9
:103A28009970511D31601179D970911D31605179AA
:103A38001971D11D31609179597102F10801316014
:103A4800D2799A71012520F065FB2B46FFF700BB60
:103A58003046FDF76BF9DFF8EC80A8F80E00304629
:103A6800FDF764F90125A8F80C002B46FFF7F0BA1A
:103A78003046FDF75BF9DFF8E880A8F8100030461B
:103A8800FDF754F9A8F812003046FDF74FF9012563
:103A9800A8F814002B46FFF7DBBA1346511C316017
:103AA80013F8020B3360D31C51783360927817F007
:103AB80083F800287FF4E5AA4FF0FF352B46FFF77F
:103AC800C7BA1346511C31601D4913F8020B087020
:103AD80033601C4953788B70D31C33601A4B92782F
:103AE8009A7001252B46FFF7B3BA184B1849186886
:103AF8004E2201252EF0F8F82B46FFF7A9BA1146F9
:103B0800531C3360134B11F8020B18703160517855
:103B18005970D11C316092789A703046FDF706F9D9
:103B28000D4B0125D8802B46FFF792BA901900203B
:103B38000340002054650020E81D0020CC440020EC
:103B4800C04900203461002044610020D443002093
:103B58001C5603082C610020905800207C30030874
:103B68005C4E00203046FDF7E1F8DFF8E483A8F862
:103B780000003046FDF7DAF8A8F802003046FDF7F5
:103B8800D5F80125A8F804002B46FFF761BADFF83D
:103B9800C49399F80030002B3FF473AADFF8B88378
:103BA80000253046FDF7C2F821F008F899F80030F2
:103BB800A8EC010A01359D42F3DBFFF762BA0D2933
:103BC8007FF47AAF531C33601578072D3FF674AF36
:103BD800DFF8889330464FF00C08FDF7A7F808FB8C
:103BE80005F809EB0805A8803046FDF79FF8E8803E
:103BF8003046FDF79BF8336828811A46591C316016
:103C080012F8021BA97232605B78EB723046FDF73E
:103C180075F8012549F808002B46FFF719BA531C17
:103C280033601078060600F1EB86BF4B1B78DD0782
:103C38003FF527AA032828BF0020012508F09EFB8E
:103C48002B46FFF705BAB84B1B78D8073FF519AADA
:103C5800012509F07BF908F089FD2B46FFF7F8B933
:103C6800B14B1B78D9073FF50CAAB04B4FF4C8727B
:103C780001251A802B46FFF7EBB909297FF71CAFFE
:103C8800DFF8DC821346511CD8F80050316013F875
:103C9800021B297033605378AB70D31C3360937860
:103CA800642B02F10401A8BF64236B713160D378DF
:103CB800642B02F10501A8BF6423AB71316013794D
:103CC800EB71931D33605379642B02F10701A8BF90
:103CD80064232B7231609379EB7002F1080333602F
:103CE800D3792B713046FDF721F872683368688103
:103CF800D11A00290CDD591CD8F800003160521A7D
:103D0800002A1978417203DD9A1C32605B7843708F
:103D180001252BF059FB2B46FFF79AB9844B1868FD
:103D2800D31C014621329D1E356013F8035C0D70CB
:103D38005D1E356013F8025C4D70336013F8015C4A
:103D48008D700333934201F10301ECD120F006FE9C
:103D5800FFF797B9C1F34705122D3FF6ADAEC5B1D0
:103D680007F1500307F12A0903EB450AC846AAF1EF
:103D7800260A3046FCF7DAFF28F8020FC245F8D1C8
:103D88006C4B39F8022F23F8022FC145F9D1112DB8
:103D980009D8694A6B00023B13440021223223F8F8
:103DA800021F9A42FBD1654A01231D461370FFF793
:103DB8004FB95D4B1B78DA073FF563A9604A137862
:103DC800012543F0040313702B46FFF741B9531C38
:103DD8005C48336001781378002940F0BE850422DE
:103DE8000270594A9B00138009F0BEFD574B01250C
:103DF80098612B46FFF72CB9DFF86881002330461D
:103E0800C8F80030FCF77AFF0125C8F800002B46F7
:103E1800FFF71EB91346511C316013F8025B33607B
:103E2800D31C507833609178002D00F02886012D3E
:103E38007FF427A90FF0A2FB2B46FFF709B9531C03
:103E480033601378002B00F08D854FF40040012576
:103E58000EF014FF2B46FFF7FBB8334B1B7813F01B
:103E680001017FF429AE531C3360107801250FF04F
:103E7800C7FA2B46FFF7ECB83046FCF757FF304639
:103E8800FCF754FF3046FCF751FF3046FCF75AFF69
:103E98003368274D1946581C2A68306011F8020B00
:103EA80082F82C003160597882F83610D91C3160BC
:103EB8009B7882F837303046FCF744FF3046FCF7F1
:103EC80041FF3046FCF73EFF3046D5F80080FCF74E
:103ED8002DFFA8F83A003046D5F80080FCF726FFF9
:103EE80033687268A8F83800D11A01290ADD591C0C
:103EF8002A6831601B7882F82E303046FCF722FFA2
:103F080033687268D31A032B0BDD3046D5F800806E
:103F1800FCF70CFFA8F8320030462E68FCF706FFC5
:103F2800B086286812E700BF03400020EE65002035
:103F3800D4430020A2610020A4610020C8610020B1
:103F48007C520020C25C002030370020E81D002091
:103F580090580020694000208C3200200C4400203A
:103F6800D8430020B8450020531C3360C64DDFF805
:103F78005483137888F805303046D5F80090FCF75C
:103F8800D5FEA9F820003046D5F80090FCF7CEFE03
:103F980072683368A9F81E00D11A072919DD30465E
:103FA800FCF7C4FEA8F80A003046FCF7BFFEA8F8E4
:103FB8000C003046D5F80090FCF7B8FEA9F82200AE
:103FC8003046D5F80090FCF7B1FE33687268A9F85E
:103FD8002400D11A03290BDD3046FCF7A7FEA8F808
:103FE8000E003046FCF7A2FE33687268A8F810008D
:103FF800D21A002A05DD591C2A6831601B7882F81C
:10400800263008F015FB1DF03FF8A04B1B68002B6D
:1040180000F0CC842868012520F008F92B46FFF72A
:1040280017B81346511C3160994913F8020BC87030
:104038003360984953784B71D31C3360964B927810
:10404800DA7001252B46FFF703B81346511C31607F
:10405800DFF8708213F8021B88F8021033608F496A
:1040680053780B70D31C33608D4D93782B71131DCF
:104078003360D378092BA8BF09233046AB70FCF70F
:1040880055FE336872682880D11A012905DD30464B
:10409800FCF74CFE33687268E8819A4207D05A1CD4
:1040A80032601B78003318BF012388F8073008F006
:1040B800BFFA336872689A423EF4E3AF5A1C326022
:1040C8001B78EB7001252B46FEF7C2BF754B1B68AA
:1040D800002B3EF4D6AF1CF075F9FF283EF4D1AFA3
:1040E8003046FCF723FE3F2840F29E84DFF8D88153
:1040F800002588F8005033687268A8F80400D21ABE
:10410800012A7EF7BEAF1A46591C316012F8021B0D
:1041180088F8021007F15000326000225D7800F83C
:10412800242D1CF021F997F82C30AB423EF4A9AFAE
:1041380028461CF03DF9FEF7A4BF5B4B1B78012B0A
:104148003EF69FAF531C11463360DFF8808111F8AB
:10415800023B88F80230D31CC01A3160012892F85B
:1041680001E0336040F370843046FCF7DFFD012541
:10417800A8F800002B46FEF76BBF531C336092F87B
:104188000080B8F1110F3FF697AC931C3360474D90
:10419800537805F818303046FCF7C8FD40F6CA03D6
:1041A8009842A8BF184640F2EE23984205EB480112
:1041B800B8BF18460125A0F2EE222B46192092FB23
:1041C800F0F24A70FEF744BF1346511C384D316077
:1041D80013F8021B2971336053786B713046FCF772
:1041E800A5FD336828805A1C32601B78AB713046B5
:1041F800FCF79CFD336868805A1C32601B78EB71B1
:1042080001252B46FEF724BF0125FDF733FB2B467E
:10421800FEF71EBF531C3360264B1278DFF8B080C0
:104228001A700023C8F800303046FCF767FD336881
:10423800D8F800202049214D10435A1CC8F8000026
:1042480032601B780B723046FCF770FD28603046F0
:10425800FCF76CFD68603046FCF768FDA8603046E6
:10426800FCF764FD3046FCF761FDFEF70ABF144B0E
:1042780002F108010132326012F8010C03F8010F53
:104288009142F7D1FEF7FDBED443002054520020DE
:1042980034610020E43C00204461002028610020B3
:1042A8005C4E0020084000202E3E0020286400209C
:1042B800CC65002070520020D8590020D42C002052
:1042C800D7590020C04900200C400020303E002073
:1042D800443E00201346511C3160C64913F8025B66
:1042E8008D70336055784D7083423EF4CAAED31C4E
:1042F8003360C14B92781A7201252B46FEF7A8BE8F
:104308000723B1FBF3F3C3EBC305491B7FF4D4AB1D
:10431800DBB203F1FF395FFA89F9002B3EF4B1AE45
:10432800DFF8D8A209F101090D46531C336092F950
:104338000010B24B4FF0000893F902208A4203F1B3
:10434800080300F09F8208F10108B8F1060FF3D1C5
:10435800FFF7B2BB531C336013780E2B3FF6ACABA0
:10436800911C31605578032D3FF6A6ABA448062171
:1043780001FB03F1431802F1030E5D71C6F800E07A
:1043880095784554111D3160D1785970511D3160AF
:1043980011799970911D31605179D970D11D3160B1
:1043A80092791A7101252B46FEF752BE3046FCF76A
:1043B800BDFCDFF86C82C8F800003046FCF7B6FC9C
:1043C800C8F804003046FCF7B1FC0125C8F808001D
:1043D8002B46FEF73DBEDFF84C820023C8F80030BC
:1043E8003046FCF78BFCD8F8003001250343C8F8A9
:1043F80000302B46FEF72CBE511C316015783B620D
:10440800132D3FF659AB911C316050787A6211F048
:1044180049F800283FF450AB7A6A7A49007801F8E5
:104428002500D01C306001EB850590786870101D60
:104438003060D078A870501D30601279EA7001F1B0
:1044480050003B6A02E00431884207D00A78002A0B
:10445800F9D18D78CA789542F5D201236A4A83F05A
:104468000103012513702B46FEF7F2BD674810299A
:104478004FF000020B4628BF1023026042608260A2
:10448800C2600274002B3EF4FCAD3268411E134436
:104498000132326012F8010C01F8010F9A42F7D18B
:1044A800FEF7EFBD531C336015781F2D3FF604ABA4
:1044B80005297FF401AB3046FCF720FC544B43F848
:1044C800250014F0CDFDFEF7DCBD514D05F1400887
:1044D8003046FCF72BFC3368A5F88000591C1A46B7
:1044E800316012F8021B85F8821032605B7885F81B
:1044F80083300435A845EBD1FEF7C3BD531C454DA9
:10450800336013782B723046FCF710FCA8833046D2
:10451800FCF70CFC28833046FCF708FC32686883FB
:10452800531C33601278EA747268D31A032B00F3B1
:1045380048823368D11A05290EDD5A1C32601B786F
:10454800EB723046FCF7DAFB3368E8605A1C3260DD
:104558001B782B7433687268D21A002A7EF791ADE3
:104568005A1C32601B7885F8213001252B46FEF74E
:104578006FBD531C3360284915780D70C01A002888
:104588007EF77FAD931C33605378003318BF012347
:1045980001254B702B46FEF75BBD531C33601D4B4A
:1045A80012785A7501252B46FEF752BD1B4BFFF7B3
:1045B8006BB83388FF2BA8BFFF23DBB2FEF7DFBC45
:1045C80019F098FA00283EF4D9AC03780A2B49D898
:1045D800B0F9023088FB0312DB17C3EBA2039BB2CE
:1045E800FF2BA8BFFF23DBB2FEF7C9BC98E8220067
:1045F800FFF74CB854610020E81D0020045A002041
:10460800C445002018630020CC1B00201061002046
:10461800F0340020D8590020705200208024002057
:10462800D42C0020443E002019F064FA00283FF4FE
:1046380014A803780A2B3FF610A8B0F90430B0F993
:10464800061003EB830383F3500521EAE171ADB251
:1046580089B2FFF704B8FB697C681A463B7D137082
:10466800FFF76EB90023BEE71346511C3160C24DF7
:1046780013F8021B6970336053782B70D31C3360B6
:104688009378AB703046FCF751FB33682881591C8E
:104698001A46316012F8021B697132605B78AB719F
:1046A80001252B46FEF7D4BC531C336013780A2B24
:1046B80000F0D9803046FCF745FB3046FCF742FB5A
:1046C80001253046FCF73EFB2B46FEF7C1BC531CC8
:1046D800336013780A2B00F0C080502B7FF4BFADF5
:1046E8003046FCF723FBDFF8B882A8F80000304614
:1046F800FCF71CFB0125A8F802002B46FEF7A8BC16
:104708009E4B3A6A9B68D4F800905A449342C0F092
:104718001181FDF723F85A464946386AFCF7C6FE68
:1047280023680344236086427EF7ABAC002100E097
:10473800236801305A1CB04222601970F8D1FEF784
:10474800A0BC336872689A4240F0CB808C4BFF2241
:104758001A704FF0000A8B4D12F014FE51462022B9
:10476800894885F800A02EF0BCFB87F82CA097F8A4
:104778002C30072B00F2EF80DFF82892824E524649
:1047880097F82C3003EB430309EBC3035B7CE3B1DD
:1047980097F82C3003EB430309EBC30320215B6933
:1047A8009BB197F82C3003EB430309EBC30358691B
:1047B80046F822000CF072FD2B7856F823000CF016
:1047C8002FFF2A780132D2B22A7097F82C300133A1
:1047D800DBB287F82C3097F82C30072BD0D9236818
:1047E800591C21601A70B8F1000F3EF44AAC674BAF
:1047F800C8F8003001252B46FEF72ABC002D7FF4AF
:104808007FAF59462046FCF7D3FA23685A1C22602A
:104818001D705A4B26689D683B6A0BEB0302954254
:1048280080F01F813B6AED1AFCF798FF2A46314653
:10483800386AFCF73BFE236803442360FEF721BC7B
:104848003046FCF773FA326871687B6A9142834696
:104858003DD106461D46FEF7E0BF3046FCF766FA36
:10486800DFF8448141E7931C3360494B5178197054
:10487800D11C316091785970111D3160D2789A70CD
:10488800FEF7FFBB0AEBC80B30468BF80210FCF7AB
:104898004DFA33682AF838001A46591C316012F864
:1048A800021B8BF8031032605A788BF80420DA1C4C
:1048B80032609A788BF806201A1D32600135DB7851
:1048C8008BF80530A9457FF430ADFEF7DABB511CF3
:1048D800316012781D46131C064618BF0123FEF7E7
:1048E8009CBF5A1C19463260254811F8022B0270E9
:1048F80031605B784370042A03D9FF2A7EF46DABDC
:1049080027E724490978994205D8022A7EF465AB3D
:10491800FF2B7EF462AB236801255A1922601D70B3
:10492800B8F1000F3EF4ADAB1B4BC8F800302B4676
:10493800FEF78EBB3A6AA3EB0208FCF70FFF42466C
:104948004946386AFCF7B2FD236803442360002D0A
:104958003EF497ABE7E6524641E704297EF491AB73
:10496800FFF73FBA0D4A1368012523F4004313608B
:104978002B46FEF76DBB00BF604300209019002056
:10498800E81D0020F3460020A0620020E1F00108A5
:10499800FB3C0020694000204D1C0108CC4300204E
:1049A8007C2400209C4D0020246100203748384991
:1049B800384A394B036001250B6013602B46FEF71C
:1049C80047BB3046FCF7B2F9A8843046FCF7AEF98D
:1049D80033687268E884D11A03297FF7ABAD1A46A9
:1049E800591C316012F8021BA97732605B7885F890
:1049F80020303046FCF79AF933687268688499E584
:104A080000F07F00032828BF002001250EF0D2FD0A
:104A18002B46FEF71DBB7D62AA46FEF797BFDA4616
:104A2800C7F824B0FEF792BFC50800F007030135A8
:104A38000133EDB2DFF868802846194688F801305E
:104A480018F0FEFFFFF755BB144B91781A88012523
:104A580012FB0EF22B4692FBF1F2A8F80020FEF7AB
:104A6800F7BAFCF77BFE5A463146386AFCF71EFD5A
:104A780023680125034423602B46FEF7E9BA012584
:104A88001FF0F8FD2B46FEF7E3BA00BFCC56002016
:104A98002057002088570020F5030008845F002075
:104AA8000C4000202DE9F04F2DED0E8BDFF8F4B00F
:104AB80097B0DBF80420079058469047002800F08C
:104AC8008E82BBF8A87000218BF85110002F6DD191
:104AD800BBF93A00DBF82450DBF82810BBF9386042
:104AE800DBF82040BBF93C20DFF8BCA0401B521A81
:104AF800CBF830009BF85210CBF83420341B0BF164
:104B08002C00CBF82C401EF015FDDAF8002091009F
:104B180041F17987DBED0C5A1F4CDBED0B7A1F490D
:104B280094ED406AD4ED416A94ED427AD4F80C21B0
:104B380009681B4B0593B8EEE58ADBED0D5AF8EED4
:104B4800E77AF8EEE58A013277EE867A38EE268A39
:104B580078EE878A8A42C4ED407A84ED418AC4EDB2
:104B6800428AC4F80C2101F04A8393F800E0BEF1B0
:104B7800140F02F09B870023D4F814510693062DD6
:104B880001F29784DFE815F004161617281529177F
:104B9800020CC6168A1500BF101E00208052002085
:104BA80088400020D44900205C4C0020DE4BDF48C0
:104BB8001A6808934FF47A76B6FBF2F2C2EB421603
:104BC80002EB8602D600DA4BDFF8C88344780593F7
:104BD800B6B2B7421D78B8F9060003F08980DBF851
:104BE8007C30BBF93810DBF8602003F1010E07EECA
:104BF800901A0A44BEF1010FCBF87CE0CBF8602094
:104C0800F8EEE77A03F08180DBED1B5ADBED1D6AD5
:104C180007EE10EA37EEE56AB8EEC75A012F86EEBE
:104C2800057A37EE257A77EEC77A8BED1C7AE7EEB0
:104C3800866A8BED1B7AF0EE667ACBED1E6ACBEDB9
:104C48001D6A03F00384DBF89030BBF93A10DBF8F7
:104C5800642003F1010E07EE901A0A44BEF1010F19
:104C6800CBF890E0CBF86420F8EEE77A03F06880A0
:104C7800DBED205ADBED226A07EE10EA37EEE56A33
:104C8800B8EEC75A012F86EE057A37EE257A77EE09
:104C9800C77A8BED217AE7EE866A8BED207AF0EE03
:104CA800667ACBED236ACBED226A03F0A783DBF8A3
:104CB800A430BBF93C10DBF8682003F1010E07EEC5
:104CC800901A0A44BEF1010FCBF8A4E0CBF8682093
:104CD800F8EEE77A03F04F80DBED255ADBED276A23
:104CE80007EE10EA37EEE56AB8EEC75A012F86EEEE
:104CF800057A37EE257A77EEC77A8BED267AE6EED7
:104D0800276A8BED257AF0EE667ACBED286ACBED33
:104D1800276A03F06683874CA8F80600BBF8A8202A
:104D2800059B013A1D78ABF8A82008990022072DA9
:104D38004A608A60CA6040F0598108F015FE059BF8
:104D4800DFF850821D78079BC01A94F82831A8F81C
:104D580000000993002B40F04F81744A5279002AD1
:104D680001F07A81744A1278013AD2B2072D84F898
:104D7800282102F01A8200230A93704BD4F83421B8
:104D8800D3F800A0684B0893079B9FED6D6AD4ED9C
:104D98004C9A6C49C4F834319A1A07EE902AF8EE06
:104DA800677AB7EE007AC6EE278A0025664BDFF8E9
:104DB800E891DFF8E881654F06932E46D1ED006A49
:104DC80094ED4BDA9FED629ADFED62AA9FED62CA1D
:104DD8009FED62AADFED62BA9FED62BA77EE69CA0B
:104DE8006CEEA6CAF4EEC7CAF1EE10FA88BFF0EE70
:104DF80047CA5D4B99ED008A2B44D3ED007AF5EE56
:104E0800407AF1EE10FA17D0584B2B4493ED007A04
:104E180078EE476AB0EEE66AF4EEC67AF1EE10FA7A
:104E280008D5F5EEC06AF1EE10FACCBF37EE878AE6
:104E380037EE678A83ED008A4D4B1A88930739D07D
:104E4800022E37D09AF82E104A4B07EE901A2B44B0
:104E580093ED007A4B42F8EEE76A07EE903A26EEB9
:104E6800877AF8EEE77AB4EEE77AF1EE10FA0AD428
:104E780007EE901AF8EE677AF4EEC77AF1EE10FAB8
:104E880088BFF0EE477A3C4B3C4903EB460331F9C7
:104E98001600B3F90C30C31A07EE103AB8EEC77A09
:104EA800D007E7EE497A41F17380354B93ED008ADC
:104EB80027EE888A089B94F868212B4493ED01EA31
:104EC80078EE4EDA002A00F0F7802E4BD4F86C21E9
:104ED80007991B688A1A9A4240F3EE809AF848307C
:104EE800022B02F0A181022E04F04584264B1B6898
:104EF800990700F19780254B87ED00CA1B689342FC
:104F0800C0F2CA80F7EE007AF4EEE79AF1EE10FAF2
:104F180040F1D28008991E4BD1ED017A93ED007AC9
:104F2800F0EEE77A3CE000BF4C4C0020C04900207E
:104F380088400020101E002028610020D443002053
:104F480000247449DC570020FC510020085200203E
:104F5800CDCCCC3DAE47813F000000000000C842E8
:104F680000003443610BB63BD0570020541F00208B
:104F7800D0430020601F00203461002080430020BF
:104F8800B8570020E45700207C430020E057002059
:104F9800EC5700208C400020481F002014520020AD
:104FA800F4EEC77AF1EE10FA40F18680D1ED027A7C
:104FB800F0EEE77AB4EEE77AF1EE10FA7CDDD1EDA7
:104FC800037AF0EEE77AB4EEE77AF1EE10FA73DDE1
:104FD8000F4B1B689B075FD50E490F4B43E00F4BE8
:104FE8000F4C1D780593072D3FF4A7AE94F8283190
:104FF8000993002B3FF4B1AE013B84F82831012D11
:1050080001F0A88217B0BDEC0E8BBDE8F08F00BF91
:105018007C43002080430020346100208840002029
:10502800101E0020D34BD449DFF8C8E331F916C06D
:105038009EED008ADFF8C0E387ED00CA03EB460067
:1050480028EE098AB0F90C00A0EB0C0007EE900AD4
:10505800F8EEE77ADEF8000027EE888A904278EECC
:105068004EDABFF64FAFB3F90C20B1F900E0C348F0
:10507800AEEB020E00688EEAEE72A2EBEE7282428E
:105088001ADAB3F90E30B1F90220D21A82EAE273C1
:10509800A3EBE27398420FDDB94B1A88002384F81A
:1050A8006831002A43F06A85B64AB74B1178186808
:1050B80081F001010CF0BAFAB44B2B4493ED000ACD
:1050C800069B2DEE000A022E20EE2D0AA3EC010A03
:1050D800069304F00D83AE4BD7ED006A93ED007A8A
:1050E800AC4BD3ED007AAC4B93ED006AAB4B67EE5B
:1050F800277A2B4427EEAC7AD3ED007A67EE277A2D
:10510800F0EE665AEDEEA75AB1EE467AB4EEE57ABD
:10511800F1EE10FA08DCB4EEE56AF1EE10FA8CBF95
:10512800B0EE657AB0EE467A94ED4C6AF7EE007A06
:10513800B4EEE76AF1EE10FAACBF0123002343B1E5
:10514800F0EEE66AF0EEC77AF4EEE67AF1EE10FADF
:1051580001D587ED007A022E04F0AC82904A914B7B
:1051680052F826001B68B0EE4E0A98478E4A8F4BBD
:1051780052F826001B6898479AF8373023B18C4BB1
:105188001B88002B00F06B87B0EE4C8A894B38EEF9
:10519800400A2B4493ED008A83ED000A9AF84830C0
:1051A80030EE480A20EE288A002B33D0824B1B7839
:1051B80013F0010300F0B886F7EE007AF4EEE79AF0
:1051C800F1EE10FA94F86831C1F2E684002B00F091
:1051D800EB87D4F86C31079AD31A784A12689A4246
:1051E80018DD774BD3ED007AF0EEEDDAF4EEE7DA7E
:1051F800F1EE10FA42F12980614B1A88002384F8F5
:105208006831002A00F09C866E494A6912B10A6822
:1052180013604B746C4B94F878212B4493ED000A7F
:105228002DEE000A20EE088A88ED008A32B9069B26
:1052380087ED00CA03ED01CA88ED00CA0136032EC6
:1052480009F1040908F1040807F1040705F1040548
:105258007FF4CFAD059B1A78072A01F0B384012AA1
:1052680001F090870023069394F88021002A41F0EA
:105278007E81DFF888A1554BDAF800201968D6043A
:1052880091F82C0000F10687DFF87491504AB9F8BC
:105298001A3092ED006A4F4A4F4DD2ED005AD5EDC3
:1052A800036A4E4A84ED646A07EE103A4C4B92ED5D
:1052B800005AD3ED007AD3ED013AD3ED024A84EDDA
:1052C800626AB8EEC77A35EEC64A012236EEC77A68
:1052D80084ED614AC4ED655A84F89821C7EE055AF1
:1052E8000A8D534206EE103A3E4BDFED3F6A93EDCE
:1052F800005A3E4B93ED004AB7EE007AF4EEC75AD7
:1053080035EE045AF1EE10FA88BFF0EE475A35EE42
:10531800275AB8EEC66AF4EEE65AF1EE10FA07EE2E
:10532800902AB4EEC65AB8BFF0EE665AF1EE10FAFB
:10533800C4ED685AB8EE677A01F10483B4EEC75A2F
:10534800F1EE10FA88BFB0EE475A264BDFED286A17
:10535800D3ED017A254B93ED014A77EE847A25EE59
:10536800265A77EEA37AB4EEE76AF1EE10FA52DC29
:1053780048E000BF3461002080430020E857002047
:105388002C6500202E650020306500208C570020F9
:10539800C856002000000020005800209857002020
:1053A800D0560020CC56002024570020205700203B
:1053B800D0430020801F002003400020E457002035
:1053C800F057002034650020A4570020D443002063
:1053D800A05F002000610020A04100209858002014
:1053E80008520020FC510020000000001452002048
:1053F8006F12833AB8570020E05700205C4C002019
:10540800D8590020B4EEE77AF1EE10FA8CBFB0EE6E
:10541800676AB0EE476AEC4B4A8DD3ED027A9FED8E
:10542800EB7A534204EE103A74EEA77AB8EEC44A07
:1054380026EE076AF4EEC47AF1EE10FA0AD407EE03
:10544800102AB8EE474AB4EEE74AF1EE10FA88BFE0
:10545800B0EE674ADE4ADFEDDD7A527824EE274A5D
:105468000AB9B1EE444A002841F0D085B7EE003AB7
:10547800D84E3278002A02F04B86D749DFEDD77A2A
:10548800D1ED024AD1ED016A91ED037A66EE244A24
:10549800E5EE264AE4EE074A63EE244AF4EEE74ACC
:1054A800F1EE10FAB4BFF0EE673AF0EE643A98BF46
:1054B800F0EE647A012ACDED0E4A02F04E8691EDA7
:1054C800067AD1ED052AD1ED076A26EE077AA5EE10
:1054D800227AA4EE267A23EE077AB4EEE77AF1EE82
:1054E80010FAB4EEE37A8CBFF0EE676AF0EE476A22
:1054F800F1EE10FA88BFF0EE676AB4BFF0EE637A97
:10550800F0EE477A022A8DED0F7A00F0DE8091EDF9
:105518000A7AD1ED092AD1ED0B3A26EE077AA5EEE3
:10552800227AA4EE237A23EE077AB4EEE67AF1EE35
:1055380010FAB4EEE77A8CBFF0EE663AF0EE473A2E
:10554800F1EE10FA98BFF0EE636AA8BFF0EE477A62
:10555800032A8DED107A00F0B88091ED0E7AD1ED26
:105568000D2AD1ED0F3A26EE077AA5EE227AA4EE9F
:10557800237A23EE077AB4EEE67AF1EE10FAB4EE67
:10558800E77A8CBFF0EE663AF0EE473AF1EE10FAA1
:1055980098BFF0EE636AA8BFF0EE477A042A8DED53
:1055A800117A00F09280D1ED123AD1ED112A91EDE5
:1055B800137A66EE233AE5EE223AE4EE073A63EE12
:1055C800233AF4EEE63AF1EE10FAF4EEE73A8CBF3D
:1055D800B0EE667AB0EE637AF1EE10FA98BFF0EEAC
:1055E800476AA8BFF0EE637A052ACDED123A6CD06F
:1055F800D1ED163AD1ED152A91ED177A66EE233AD8
:10560800E5EE223AE4EE073A63EE233AF4EEE63AA0
:10561800F1EE10FAF4EEE73A8CBFB0EE667AB0EE2F
:10562800637AF1EE10FA98BFF0EE476AA8BFF0EE81
:10563800637A062ACDED133A47D0D1ED1A3AD1ED67
:10564800192A91ED1B7A66EE233AE5EE223AE4EE4A
:10565800073A63EE233AF4EEE63AF1EE10FAF4EE86
:10566800E73A8CBFB0EE667AB0EE637AF1EE10FAE4
:1056780098BFF0EE476AA8BFF0EE637A072ACDED2F
:10568800143A22D091ED1E7AD1ED1D2AD1ED1F3AA0
:1056980026EE077AA5EE227AA3EE847A27EE037A1D
:1056A800B4EEE67AF1EE10FAB4EEE77A8CBFB0EE1B
:1056B800666AB0EE476AF1EE10FA8DED157A98BF7A
:1056C800F0EE466AA8BFF0EE477A77EEE67AF7EE94
:1056D800006AF4EEE67AF1EE10FAC4ED4C7A43F380
:1056E800D78586EEA77A022ADDED0F7A67EE244A7F
:1056F80067EE877ACDED0E4ACDED0F7A2DD0DDED30
:10570800107A67EE877A032ACDED107A25D0DDED81
:10571800117A67EE877A042ACDED117A1DD0DDED76
:10572800127A67EE877A052ACDED127A15D0DDED6B
:10573800137A67EE877A062ACDED137A0DD0DDED60
:10574800147A67EE877A072ACDED147A05D0DDED55
:10575800157A27EE877A8DED157A2149096811F0B7
:1057680080530A9301F0CB81F6EE005AC4ED685AD3
:10577800002A02F09D8494F998311A4994ED656ADB
:10578800C87894ED645ADAF80010DFF868E0164F2C
:10579800DEED004AB7F906E0B9F81A700B9707EE84
:1057A800103A124BD4ED616A1D78114BD4ED627A30
:1057B8001B780893BDEEC66A01F4805316EE10CA32
:1057C800BDEEC56A0D9317E0FC5100206F12833AB5
:1057D8007052002069400020085800200000000096
:1057E800F860002020340020FA71002003400020D7
:1057F800804E00200458002001F4800301F01007B7
:10580800B8EEC77A0C9305F0010816EE101A0028B6
:1058180040F06487002F41F0D582D34D9DED0E5A9C
:1058280095ED006AD14825EE866AA5EE076AB0EEC6
:10583800675AA6EE265ABDEEC56A16EE10EA16EEAF
:10584800107AE645A8BF67467145C8BF0F4606EE01
:10585800107AB8EEC66A012A80ED006A00F0DC8092
:1058680095ED046A9DED0F5A25EE866AA5EE076A46
:10587800B0EE675AA6EE265ABDEEC56A16EE10EAD5
:1058880016EE107AE645A8BF67467145C8BF0F46B1
:1058980006EE107AB8EEC66A022A80ED016A00F0B8
:1058A800BB8095ED086A9DED105A25EE866AA5EE37
:1058B800076AB0EE675AA6EE265ABDEEC56A16EE1E
:1058C80010EA16EE107AE645A8BF67467145C8BFCC
:1058D8000F4606EE107AB8EEC66A032A80ED026A11
:1058E80000F09A8095ED0C6A9DED115A25EE866AB6
:1058F800A5EE076AB0EE675AA6EE265ABDEEC56A4F
:1059080016EE10EA16EE107AE645A8BF674671450E
:10591800C8BF0F4606EE107AB8EEC66A042A80EDB4
:10592800036A79D095ED106A9DED125A25EE866AC4
:10593800A5EE076AB0EE675AA6EE265ABDEEC56A0E
:1059480016EE10EA16EE107AE645A8BF67467145CE
:10595800C8BF0F4606EE107AB8EEC66A052A80ED73
:10596800046A59D095ED146A9DED135A25EE866A9E
:10597800A5EE076AB0EE675AA6EE265ABDEEC56ACE
:1059880016EE10EA16EE107AE645A8BF674671458E
:10599800C8BF0F4606EE107AB8EEC66A062A80ED32
:1059A800056A39D095ED186A9DED145A25EE866A78
:1059B800A5EE076AB0EE675AA6EE265ABDEEC56A8E
:1059C80016EE10EA16EE107AE645A8BF674671454E
:1059D800C8BF0F4606EE107AB8EEC66A072A80EDF1
:1059E800066A19D095ED1C6A9DED155A65EE865A22
:1059F800E7EE055AE6EEA57AFDEEE77A17EE905A3D
:105A0800AC45A8BFAC46A942D8BF614607EE901A7C
:105A1800F8EEE77AC0ED077AB8F1000F00F06C876E
:105A2800534A1268002A40F07487524A127892B199
:105A3800307868B14D4FDFF85C810025E8B2D8F8BE
:105A48000030B7EC010A9847307801358542F5DB1C
:105A5800494A12689047059B1A78072A01F0A180E5
:105A68000026DAF80020530500F1D187434B1B7854
:105A7800BBB1434AB9F81A30B2F906209A4210DC91
:105A8800404B1B78012B01F09583192B01F0928371
:105A98000E2B06D0082B04D03B4D0023AB60C4F876
:105AA800403194F8AA5125B1384B1B889F0741F023
:105AB8002F8394F8B021002A40F0488799F81E7087
:105AC800002F00F02984022F01F0D582032F41F026
:105AD800CE8299F82030C3EB431103EB8101C90052
:105AE80089B299F81F300233DBB2002A00F05585DD
:105AF800002900F0528526480768B1FBF7F10FB27C
:105B0800A4F8E071002B03F0438007EE907AF8EEDA
:105B1800E77AF7EE006A86EEA77A1B4D012BD4EDE3
:105B28007D6AD5ED007A77EEE67A67EE877AC4ED7E
:105B3800797A3BD0D5ED017AD4ED7E6A77EEE67AB4
:105B4800022B67EE877AC4ED7A7A2FD0D5ED027AE8
:105B5800D4ED7F6A77EEE67A032B67EE877AC4ED99
:105B68007B7A23D018E000BF08580020305200206C
:105B7800C4560020A85100207C4E0020CC1B0020D9
:105B8800FA71002070520020A0410020D04300206C
:105B980054520020744E0020D5ED037AD4ED806A6B
:105BA80077EEE67A67EE877AC4ED7C7A059909780C
:105BB800092903F0ED81002F40F3B4839BB394EDE2
:105BC8007D7AD4ED797A77EE877A012BC4ED7D7AE8
:105BD800C5ED007A21D094ED7E7AD4ED7A7A77EE0D
:105BE800877A022BC4ED7E7AC5ED017A15D094ED43
:105BF8007F7AD4ED7B7A77EE877A032BC4ED7F7AB0
:105C0800C5ED027A09D0D4ED807A94ED7C7A77EEEE
:105C1800877AC4ED807AC5ED037A013B022BB8BFC1
:105C28000223DBB20993099B002A18BF02239E4670
:105C3800C84BDFEDC96A1A68059B91781878137804
:105C480007EE903AF8EEE77AB0EE007A67EEA67AB9
:105C5800F4EEC77AF1EE10FA40F35F86DFEDBF6A23
:105C680037EEC77AB0EE676AA7EE266AF0EE466AA4
:105C780095ED007A9FEDBA6A27EE066AF0EEC65AED
:105C880084ED546AC4ED575A99B107EE101AB8EE6C
:105C9800C75A9FEDB17A66EE064A25EE075AB7EE67
:105CA800007A37EE457A64EEA54AA4EE857A26EEA8
:105CB800076A9FEDAC7A537926EE877A27EE067A43
:105CC800CBB1DFEDA56A9FEDA86A65EEA65A06EE90
:105CD800903AF8EEE66A65EEA65AF4EEC65AF1EE88
:105CE80010FA01F38981B7EE006A76EE655AC6EEBE
:105CF800256A27EE267A0C289FED9C8ADFED9C6AA0
:105D080000F02487B4EEC87AF1EE10FA98BFB0EE2E
:105D1800478AB4EEE68AF1EE10FAB8BFB0EE668AAA
:105D280084ED4E8ABEF1000F00F0DD80B0EE007AFF
:105D3800F4EEC77AF1EE10FA05DD37EEC77ADFED3B
:105D4800876AE7EE267A95ED017ADFED856A27EE18
:105D5800267AF0EEC75A84ED557AC4ED585A99B1AF
:105D680006EE901A9FED7C6AF8EEE66A27EE075A6F
:105D780066EE866AB7EE006A36EE666A25EE255A42
:105D8800A5EE266A27EE067ADFED766A937967EE46
:105D9800A67A67EE877AABB107EE103AB8EEC77A03
:105DA8009FED6D6ADFED706A27EE257A27EE067A99
:105DB800B4EEE67AF1EE10FA41F31081DFED6D6A88
:105DC80067EEA67A0C2800F0A186DFED686A9FEDE1
:105DD800687AF4EEE67AF1EE10FA88BFF0EE667AA9
:105DE800F4EEC77AF1EE10FAB8BFF0EE477ABEF1DA
:105DF800010FC4ED4F7A76DD5378DFED576A07EE71
:105E0800903AF8EEE77AB0EE007A67EEA67A537A1F
:105E1800F4EEC77AF1EE10FA05DD37EEC77ADFED5A
:105E28004F6AE7EE267A95ED027ADFED4D6A27EEA6
:105E3800267AF0EEC75A84ED567AC4ED595A9BB1CA
:105E480006EE903A9FED446AF8EEE66A27EE075AA6
:105E580066EE866AB7EE006A36EE666A25EE255A61
:105E6800A5EE266A27EE067ADFED3E6AD37967EE5D
:105E7800A67A67EE877AFBB107EE103AB8EEC77AD2
:105E88009FED356ADFED386A27EE257A27EE067A28
:105E9800B4EEE67AF1EE10FA01F39C80B5EEC07A22
:105EA800F1EE10FA02F1FE82B7EE006A36EE477A9A
:105EB800C6EE076A67EEA67A0C2800F06586DFED65
:105EC8002B6A9FED2B7AF4EEE67AF1EE10FA88BF92
:105ED800F0EE667AF4EEC77AF1EE10FAB8BFF0EE9B
:105EE800477AC4ED507A092800F0FC8599F82150CA
:105EF800002D40F0B185002384F8B0311E4B1B788B
:105F080023B91E4DAA78002A41F0C180059B1D784F
:105F1800072D7FF474A807F027FD194B059A801BFD
:105F28001578D880FFF76BB894F86821002A3FF4F9
:105F380071A9144A84F868311288002A7FF464A988
:105F4800114A124B1178186881F001010BF06EFBB1
:105F5800FFF760B9D84300200AD7233CD7A368418C
:105F68006F12033B00004843A4707D3F00C0F94412
:105F780000C0F9C40000C842C9330020303E0020E8
:105F88008C4000202C6500202E6500203065002004
:105F980094ED577AB1F90000D4ED586AB1F902E0EE
:105FA800E24AF4EEC76A80EAE0738EEAEE71A3EB88
:105FB800E073F1EE10FAA1EBEE71B8BFF0EE476AAC
:105FC8008B42B8BF0B4607EE103A1378B8EEC77A83
:105FD80027EE097A002B40F0B880D54B93ED006A84
:105FE800B4EEEA6AF1EE10FA41F14C80F7EE005A8D
:105FF80075EEC65A3BEEC77A65EE8B5ACD4BA7EEC7
:10600800256A93ED007A26EE076AB5EEC06AF1EECE
:1060180010FA40F27085CAEE065AB7EE007AB0EE72
:10602800476AA6EEE56AF0EE466AF4EEC76AF1EE54
:1060380010FA88BFF0EE476AF5EEC06AF1EE10FA82
:10604800B8BFF0EE4C6ABC4B93ED007A67EE877AE6
:10605800A7EEA68AFEF72EBF0122FEF787BEB74B32
:10606800B74A2B4493ED007AD2ED007AB54B67EE30
:10607800277AF7EE006AF4EEE67AF1EE10FA93ED7D
:10608800007A88BFF0EE667A67EE877A27EE888A0C
:10609800FFF77CB8AC4BDFF8EC921A78D5075CBFF9
:1060A800B9F81820A4F88C21A84AA94D1288D5ED72
:1060B800037A07EE102AB8EEC77AF4EEC77AF1EE43
:1060C80010FA41F2C587A34D2B8807EE103AB8EEB7
:1060D800C77AF4EEC77AF1EE10FAC1F277809E4AD9
:1060E8009E4D92ED006AD5ED006A94F99821C4EDB1
:1060F800646A76EE665A012AC4ED626AC4ED615A92
:1061080084ED656A01F0EE85079BC4F89C31002593
:1061180037EEC77AFCEEE77A914E84ED687A17EE8F
:10612800902AA4F88C21012296ED005A84F898212F
:106138008C4A954241F279878B4BD3ED007AD3EDA7
:10614800013AD3ED024AFFF7C9B87A4B93ED005AEA
:10615800B5EEC05AF1EE10FA40F3CD84834BD3ED7F
:10616800004AF5EEC04AF1EE10FA40F3C48434EE6A
:10617800C77A66EECA5A87EE246AC5EE856AB7EE14
:10618800007AB4EEC76AF1EE10FA88BFB0EE476A3B
:10619800B5EEC06AF1EE10FA76EE876AB8BFB0EED7
:1061A8004C6A66EE266A40E7714AD2ED007AB0EE94
:1061B800C87AB4EEE77AF1EE10FA7FF72BA86D4AA9
:1061C800D2ED007AB0EEED7AB4EEE77AF1EE10FA9D
:1061D8007FF720A8684AD9ED007A92ED007AF0EEB0
:1061E800E77AF4EEC77AF1EE10FA7FF513A80122E8
:1061F8000799C4F86C1184F86821FEF7EEBF07EE22
:10620800102A1978DFF88081C4F80C71B8EEC77AC3
:10621800F7EE006A132986EE879AB8F90400B4F8F5
:1062280010619BED070A01F0E984544A544992ED44
:10623800001AD2ED053A92ED122A92ED173AD2EDF4
:10624800091AD2ED0E4A92ED016A92ED064A92EDD4
:106258000A7AD2ED0F5AD2ED132AD2ED186A92EDCE
:10626800045AD2ED030A67EE897A69EE288A29EE84
:10627800088AE1EE273A01EB86070025A2EE283AC4
:10628800C4F80051C4F80451E1EE884AA6EE274A42
:10629800E7EE085A92ED167A92ED0D6A92ED021A1F
:1062A800D2ED0C1AC7ED003AE2EEA86A25EE635A61
:1062B80027EE437A92ED0B2AD2ED152AC7ED204A34
:1062C800A0EEE34A26EE646AD2ED143A82ED054A5E
:1062D800A1EE275AF0EE477AE1EEE45AA2EE086AF8
:1062E800E2EEC36AE3EEA87A82ED065AC2ED0E5AD0
:1062F80082ED0F6A87ED403AC2ED176AC2ED187A4F
:10630800C4F80851721C02F01F02A4F81021A8F862
:106318000400059BFEF729BCA4F8E071002A3FF4AD
:10632800EDAD0B4D4FF0020E82E400BFC4570020C4
:10633800CC570020C0570020BC5700206C1F0020FD
:10634800B4570020B0570020034000209C5800207C
:10635800A04100209E58002000610020885800209D
:10636800A45800208FD0030008520020C8570020EE
:10637800F4570020F0570020F8570020105500204F
:10638800A4520020D85900208C400020BC4A117823
:10639800D4F81871BB4B9FEDBC7AFE009A1982EDB8
:1063A800007A002979D0B948B0EE476AF0EE476A1A
:1063B8000022F0EC017A013267EEA77A05EE902A06
:1063C800B4EEE77AF1EE10FAF8EEE55AB8BFB0EE9F
:1063D800677A8A4276EEA76AA7EEA56AE9D1F5EE52
:1063E800C06A9A19F1EE10FA82ED007A55DDC6EE10
:1063F800265AA74AA7490988F7EE007A75EEE75AA0
:10640800D2ED007A65EEA77AFDEEE77A17EE902ACC
:10641800812A42F353808A42A8BF0A4607EE902A8F
:10642800F8EEE77A9C4AF01902EB800292ED057AC1
:10643800D2ED003A92ED066A92ED014AD2ED046A75
:10644800D2ED034A92ED025AA3EEA77AA4EE276A88
:1064580066EEC76AA7EE646ABDEEC77AE5EE276AFC
:1064680017EE100A812882ED056AC2ED066A42F32A
:1064780022808142A8BF014607EE901AF8EEE77A1B
:10648800FCEEE77ACDED087ABDF8202099198A80CC
:106498001FB9BEF1130F02F0E786BEF1150F41F0E8
:1064A800ED801E44DFF81082B28828F81720D4F84F
:1064B80014517A4A013582FB05325119EA17C2EBA9
:1064C800A102C2EBC202AD1AC4F814517448D4F840
:1064D8001C11079B734D02682D78C4F81C31591A9A
:1064E8000A440260002D64D107EE901A6E4EDFF860
:1064F800E0916E4FB8EEE78A06F5F07506F5137869
:10650800F6EC017A9BED070ADBF80832F8EEE77A39
:10651800284627EE800A9847A5F1E000DBF82831E5
:106528009847A5F17000DBF898319847D6F8EC0049
:10653800DBF8AC309847D7ED007AA9EC010AE0EE19
:10654800087A2435A845E7EC017AD9D1059B1D784E
:10655800FEF749BD564B574A19681288564BC96908
:1065680019805A8017B0BDEC0E8BBDE8F08F534BE5
:10657800534E1A7812F0010F327840F03983002A0E
:1065880000F03E8592004F494F48DFF848A1DFF8F8
:1065980048912BF0A9FBFFF743BAB4F8E071013F2B
:1065A8003FB2002FA4F8E0717FF7B8AE474DFFF770
:1065B80005BB07EE901A3C4D454BDFF8FC80DFF831
:1065C800EC900694F8EEE78A05F5B87600271C46A5
:1065D800CDF82480059BDBED077A1B78172B00F09C
:1065E800A08195ED007AB8EEC78A082B28EE278A95
:1065F80007D1B0EE480A08932BF0B6FC089BA8F820
:106608000000DAF8002092000BD5002F03F0028179
:10661800B0EE480ADBF8083206F170009847B0EE91
:10662800408AB0EE480ADBF82831A6F17000984796
:10663800DBF8983130469847059B1B78032BB0EE62
:10664800408A00F07A81D5F8F000DBF8AC30B0EE83
:10665800480A9847D9ED007AA4EC010AE0EE287AB6
:106668000137032F06F1240608F1020805F1040595
:10667800E9EC017AAED1059B069C1D78FEF7B3BC08
:10668800865200207C55002000000000101E0020CB
:106698008852002084520020A45400209324499258
:1066A800906500207D520020004A0020946500205B
:1066B800F43C0020883200208C4000200340002059
:1066C800694000208C32002030520020A041002078
:1066D800504C00205C4C0020D8590020002F00F0BE
:1066E8009186B8F1000F42F0A982089BCD4D002B8E
:1066F80042F0F68095ED006A9DED0E5ACA4825EEE7
:10670800866AFDEEE44AA5EE076AB0EE675AA6EE81
:10671800265A14EE901ABDEEC56A16EE10EA16EE69
:10672800107AE645A8BF67467145C8BF0F4606EE12
:10673800107AB8EEC66A012A80ED006A00F0DF80A0
:1067480095ED046A9DED0F5A25EE866AA5EE076A57
:10675800B0EE675AA6EE265ABDEEC56A16EE10EAE6
:1067680016EE107AE645A8BF67468E45B8BF0F46B5
:1067780006EE107AB8EEC66A022A80ED016A00F0C9
:10678800BE8095ED086A9DED105A25EE866AA5EE45
:10679800076AB0EE675AA6EE265ABDEEC56A16EE2F
:1067A80010EA16EE107AE645A8BF67468E45B8BFD0
:1067B8000F4606EE107AB8EEC66A032A80ED026A22
:1067C80000F09D8095ED0C6A9DED115A25EE866AC4
:1067D800A5EE076AB0EE675AA6EE265ABDEEC56A60
:1067E80016EE10EA16EE107AE645A8BF67468E4503
:1067F800B8BF0F4606EE107AB8EEC66A042A80EDD6
:10680800036A7CD095ED106A9DED125A25EE866AD2
:10681800A5EE076AB0EE675AA6EE265ABDEEC56A1F
:1068280016EE10EA16EE107AE645A8BF67468E45C2
:10683800B8BF0F4606EE107AB8EEC66A052A80ED94
:10684800046A5CD095ED146A9DED135A25EE866AAC
:10685800A5EE076AB0EE675AA6EE265ABDEEC56ADF
:1068680016EE10EA16EE107AE645A8BF67468E4582
:10687800B8BF0F4606EE107AB8EEC66A062A80ED53
:10688800056A3CD095ED186A9DED145A25EE866A86
:10689800A5EE076AB0EE675AA6EE265ABDEEC56A9F
:1068A80016EE10EA16EE107AE645A8BF67468E4542
:1068B800B8BF0F4606EE107AB8EEC66A072A80ED12
:1068C800066A1CD095ED1C6A9DED155A65EE865A30
:1068D800E7EE055AE6EEA57AFDEEE77A17EE905A4E
:1068E800AC45A8BFAC46A942D8BF614607EE901A8E
:1068F800F8EEE77AC0ED077A002A3FF491A89200F3
:106908004A4949482BF0F0F9494A1268002A3FF4ED
:106918008CA81DF033F8FFF788B8F0EE676AFFF728
:10692800A7B995ED007A0BEB4702B8EEC78A128F2C
:10693800A8F8002028EE278A63E62BF015FBA8F8B4
:10694800000080E6B0EE465AFEF7FFBC39493A4BE4
:10695800D1F8EC101B6844F620608142A8BF0146BC
:10696800B1F57A7FB8BF4FF47A7189B213F0100F7E
:10697800A4F8B211DAF8003000F02384DB0441F106
:10698800A1852E4BD3F800E0BEF832707F082C4D5D
:106998002C48D4F8B431D5ED037AA0FB010188095D
:1069A800642191FBF0F11429BDEEE77A04EB43056D
:1069B800A8BF142101338B42C4F8B43117EE10CAB2
:1069C800A4BF0023C4F8B43104EB4303A5F8B8C14D
:1069D800B3F9B83107EE103AB8EEC77A77EEC77A4E
:1069E800FDEEE77ACDED067ABDF9181081EAE1737C
:1069F800A3EBE173BB4201F32D8713494FF07E539C
:106A08000B60FFF75BB8114B0593114C5EE5DBF8A3
:106A18000830002B3FF42AA80E49A1F14C009847F2
:106A2800FFF724B808580020305200208C3200208C
:106A3800C4560020F8000020F8600020D44300204D
:106A4800A0410020D34D62100000002088400020A3
:106A5800101E0020204A00201E21CE48FAF784FC90
:106A680000283FF448AACC4B1B8858063FF543AA98
:106A780094F80432AB4242F01C82C84BD4ED827ABF
:106A8800D3ED016A94ED505ADFEDC55A9FEDC56A02
:106A980027EEC57A68EE277AA8EE267AE5EE267AFA
:106AA800B4EEE57AF1EE10FA88BFB0EE657AB4EE8E
:106AB800C67AF1EE10FAF4EEE57AB8BFB0EE467A8F
:106AC800F1EE10FA88BFF0EE657AF4EEC67AF1EED0
:106AD80010FAB8BFF0EE467A84ED4E7AC4ED507ADB
:106AE800FFF709BAFDEEC87AAF4A17EE903A9780D9
:106AF800D380FFF7FBB9DFEDAD6AFFF7A4BADAF888
:106B0800001049023EF530AEFEF732BE9FEDA47A82
:106B1800DFEDA46AA449F4EEC77AF1EE10FA98BF43
:106B2800B0EE677AFDEEE77AB4EEE67AF1EE10FAA7
:106B380017EE903AB8BFB0EE667ABEF1010F84ED59
:106B48004F7A4B803FF758A9FFF7D0B9B4EEC87A0F
:106B5800F1EE10FA98BFB0EE478ABDEEC77AB4EEF0
:106B6800E68ADFF844C2F1EE10FA17EE103AB8BF21
:106B7800B0EE668A84ED4E8AACF80030BEF1000FA4
:106B88007FF4D4A8FFF7B2B9BDEEE77A864B17EECB
:106B9800102A9A80FFF793B9002B3EF43BABFEF71F
:106BA80018BB06F0E1FE059B7F491A78069B072A69
:106BB800A0EB030088807EF453AF06F0D5FE0646AE
:106BC800FEF74FBF06F0D0FE059BDFF8DC811A7890
:106BD8000A9B012AA0EB0300A8F8020000F0D48267
:106BE800072A7EF43FAB06F0BFFE0690FEF73CBBDB
:106BF800002A00F00582D4ED583A94ED574AD4EDB6
:106C0800627A6B4994ED617A91ED005AD4ED555A48
:106C180094ED546A674D6848F4EEC43AF3EE046A9A
:106C2800F1EE10FA77EEA64A00F11E8395ED026A9E
:106C380026EE656AB0EE674AA6EE074AB4EEE44A65
:106C480034EE666AF1EE10FA48BFB0EE456A012AE2
:106C580080ED006A00F0D48195ED066A26EE656A3B
:106C6800B0EE674AA6EE074AB4EEE44A34EE666A26
:106C7800F1EE10FA48BFB0EE456A022A80ED016ACB
:106C880000F0BE8195ED0A6A26EE656AB0EE674AA5
:106C9800A6EE074AB4EEE44A34EE666AF1EE10FA5C
:106CA80048BFB0EE456A032A80ED026A00F0A88169
:106CB80095ED0E6A26EE656AB0EE674AA6EE074ABB
:106CC800B4EEE44A34EE666AF1EE10FA48BFB0EE6C
:106CD800456A042A80ED036A00F0928195ED126AF4
:106CE80026EE656AB0EE674AA6EE074AB4EEE44AB5
:106CF80034EE666AF1EE10FA48BFB0EE456A052A2E
:106D080080ED046A00F07C8195ED166A26EE656ACE
:106D1800B0EE674AA6EE074AB4EEE44A74EE666A35
:106D2800F1EE10FA48BFF0EE456A062AC0ED056A92
:106D380000F06681D5ED1A6A66EEE56AB0EE674A3C
:106D4800A6EE874AB3EE046AB4EEE44A74EE466AE5
:106D5800F1EE10FA48BFF0EE456A072AC0ED066A60
:106D680000F04E81D5ED1E6ADFF850A0DFF8509094
:106D780066EEE55AE5EE877AF4EEE74A77EEC67AEC
:106D8800F1EE10FAC8BFF0EE457AC0ED077AFEF7CB
:106D980047BE00BFF8600020D0430020000000205C
:106DA80000C0F94400C0F9C48C4000200000000075
:106DB8000458002008580020305200205C4C002065
:106DC800D8590020B8F1000F41F00282DB4D9DED4B
:106DD8000E5A95ED006ADA4825EE866AA5EE076A2E
:106DE800B0EE675AA6EE265ABDEEC56A16EE10EA50
:106DF80016EE107AE645A8BF67467145C8BF0F462C
:106E080006EE107AB8EEC66A012A80ED006A3FF4F1
:106E180076AD95ED046A9DED0F5A25EE866AA5EECE
:106E2800076AB0EE675AA6EE265ABDEEC56A16EE98
:106E380010EA16EE107AE645A8BF67467145C8BF46
:106E48000F4606EE107AB8EEC66A022A80ED016A8D
:106E58003FF455AD95ED086A9DED105A25EE866A0A
:106E6800A5EE076AB0EE675AA6EE265ABDEEC56AC9
:106E780016EE10EA16EE107AE645A8BF6746714589
:106E8800C8BF0F4606EE107AB8EEC66A032A80ED30
:106E9800026A3FF434AD95ED0C6A9DED115A25EE6A
:106EA800866AA5EE076AB0EE675AA6EE265ABDEEC8
:106EB800C56A16EE10EA16EE107AE645A8BF6746D0
:106EC8007145C8BF0F4606EE107AB8EEC66A042AA6
:106ED80080ED036A3FF413AD95ED106A9DED125AEB
:106EE80025EE866AA5EE076AB0EE675AA6EE265A20
:106EF800BDEEC56A16EE10EA16EE107AE645A8BF92
:106F080067467145C8BF0F4606EE107AB8EEC66AE6
:106F1800052A80ED046A3FF4F2AC95ED146A9DED04
:106F2800135A25EE866AA5EE076AB0EE675AA6EEF2
:106F3800265ABDEEC56A16EE10EA16EE107AE64538
:106F4800A8BF67467145C8BF0F4606EE107AB8EE6F
:106F5800C66A062A80ED056A3FF4D1AC95ED186A39
:106F68009DED145A25EE866AA5EE076AB0EE675ABB
:106F7800A6EE265ABDEEC56A16EE10EA16EE107A8F
:106F8800E645A8BF67467145C8BF0F4606EE107AAA
:106F9800B8EEC66A072A80ED066A3FF4B0AC95EDF4
:106FA8001C6A9DED155A65EE865AE7EE055AE6EE1F
:106FB800A57AFDEEE77A17EE905AAC45A8BFAC4625
:106FC800A942C8BF8C4607EE90CAF8EEE77AC0ED32
:106FD800077A91E4DFED5B6AFEF76CBFB5EEC07A25
:106FE800F1EE10FA01F15A82B7EE006A36EE477AEE
:106FF800C6EE076AFEF7E4BEDFED526AFEF779BE19
:10700800DFF878A1DFF87891FEF70ABD4E494A7992
:10701800002A3EF42BAA4D4A1278002A3EF426AAEA
:107028000B784B49DFED4B4A07EE903A0B88B8EEE8
:10703800677A07EE902A06EE903AF8EEE77AF8EECD
:10704800666A67EE277AB7EE007A87EEA63AB4EE5C
:10705800E43AF1EE10FA88BFB0EE643AB4EEC73AFB
:10706800F1EE10FAB8BFB0EE473AFEF701BA3A4B64
:107078005988FEF736BDB4F8B21101F57A7189B2B4
:10708800FEF72FBD354B93ED006AFEF7BEBF344FB8
:107098003B78013B0D2B24D8DFE813F0F506BB073E
:1070A800E606CB0623002300A4078F0734070E004B
:1070B80067075B07860702072A4B1B78002B02F03D
:1070C800F5801A2028F01EF9002842F0EF80264BA0
:1070D8001B78002B42F0EA8009233B7024F0B6FCB1
:1070E800AA78012A00F063852B79012B01F05985D4
:1070F800022B7EF40BAF3B78012B7EF407AF1A4BC3
:107108001B78002B7EF402AF24F06AF9FEF7FEBE6E
:10711800164B9FED177AD3ED087AF4EEC77AF1EEA5
:1071280010FA00F2F9849FED137A134DD5ED037A26
:1071380077EE877AC5ED037AFEF7BBBC08580020C6
:10714800305200200000C842604300209E410020C9
:1071580088410020713DAA3FC0470020C057002049
:107168002E3E002072520020715F002068650020CA
:107178008FC2753C00000000A04100205C4C00203C
:10718800D8590020DFF8708206F0EEFB9049D4F859
:107198007C2109680690821A511AC4F87C01A8F863
:1071A8000420A8F80610FEF75FB806F0DDFB0A9089
:1071B800FDF7E3BD874B9B7B002B3EF46DACFEF7E0
:1071C80070BCDD003FF5DAABFEF778BCB4F88C5143
:1071D800954240F2028594F8A451002D40F06E8744
:1071E8007D4A7E4E92ED007AD6ED007A94F9982188
:1071F800C4ED647A77EE676A012AC4ED627AC4ED59
:10720800616A84ED657A02F03D80079BC4F89C3181
:10721800734A9FED747A92ED005A84ED687A0122E0
:1072280084F89821FEF784BF6F4B1B88002B40F031
:10723800E8856E4A6E4B117818680AF0F7F9D4F8A9
:107248006C21079B9A1AFDF74EBE6A4BD9ED007A5E
:1072580093ED007AF0EEE77AF4EEC77AF1EE10FAE1
:107268007DF7D8AFFDF7C8BFD5ED015A65EEC65A10
:10727800B0EE674AA5EE874AB4EEE44A74EE665A61
:10728800F1EE10FA48BFF0EE455A012AC0ED005A57
:107298003FF4B6AED5ED055A65EEC65AB0EE674A6C
:1072A800A5EE874AB4EEE44A74EE665AF1EE10FA97
:1072B80048BFF0EE455A022AC0ED015A3FF4A0AE8D
:1072C800D5ED095A65EEC65AB0EE674AA5EE874A6B
:1072D800B4EEE44A74EE665AF1EE10FA48BFF0EEE6
:1072E800455A032AC0ED025A3FF48AAED5ED0D5A2D
:1072F80065EEC65AB0EE674AA5EE874AB4EEE44A90
:1073080074EE665AF1EE10FA48BFF0EE455A042AB8
:10731800C0ED035A3FF474AED5ED115A65EEC65A66
:10732800B0EE674AA5EE874AB4EEE44A74EE665AB0
:10733800F1EE10FA48BFF0EE455A052AC0ED045A9E
:107348003FF45EAED5ED155A65EEC65AB0EE674A03
:10735800A5EE874AB4EEE44A74EE666AF1EE10FAD6
:1073680048BFF0EE456A062AC0ED056A3FF448AE0C
:10737800D5ED196A66EEC66AB0EE674AA6EE874A88
:10738800F3EE045AB4EEE44A74EE656AF1EE10FACC
:1073980048BFF0EE456A072AC0ED066A3FF430AEF2
:1073A800D5ED1D6ADFF854A0DFF8549026EEC66AC2
:1073B800E6EE077AF4EEE47A77EEE57AF1EE10FA83
:1073C800B8BFF0EE457AC0ED077AFEF729BB00BFDB
:1073D80054520020D847002000610020885800201F
:1073E800A4580020000000002C6500202E65002015
:1073F80030650020F85700208C4000205C4C0020AD
:10740800D8590020089BD94D002B41F08D8095ED6F
:10741800006A9DED0E5AD64825EE866AFDEEE44ACE
:10742800A5EE076AB0EE675AA6EE265A14EE901A31
:10743800BDEEC56A16EE10EA16EE107AE645A8BF4C
:1074480067467145C8BF0F4606EE107AB8EEC66AA1
:10745800012A80ED006A3EF4DFAA95ED046A9DEDED
:107468000F5A25EE866AA5EE076AB0EE675AA6EEB1
:10747800265ABDEEC56A16EE10EA16EE107AE645F3
:10748800A8BF67468E45B8BF0F4606EE107AB8EE1D
:10749800C66A022A80ED016A3EF4BEAA95ED086A22
:1074A8009DED105A25EE866AA5EE076AB0EE675A7A
:1074B800A6EE265ABDEEC56A16EE10EA16EE107A4A
:1074C800E645A8BF67468E45B8BF0F4606EE107A58
:1074D800B8EEC66A032A80ED026A3EF49DAA95EDCD
:1074E8000C6A9DED115A25EE866AA5EE076AB0EE84
:1074F800675AA6EE265ABDEEC56A16EE10EA16EED3
:10750800107AE645A8BF67468E45B8BF0F4606EE17
:10751800107AB8EEC66A042A80ED036A3EF47CAAA3
:1075280095ED106A9DED125A25EE866AA5EE076A5A
:10753800B0EE675AA6EE265ABDEEC56A16EE10EAF8
:1075480016EE107AE645A8BF67468E45B8BF0F46C7
:1075580006EE107AB8EEC66A052A80ED046A3EF493
:107568005BAA95ED146A9DED135A25EE866AA5EE81
:10757800076AB0EE675AA6EE265ABDEEC56A16EE41
:1075880010EA16EE107AE645A8BF67468E45B8BFE2
:107598000F4606EE107AB8EEC66A062A80ED056A2E
:1075A8003EF43AAA95ED186A9DED145A25EE866ABE
:1075B800A5EE076AB0EE675AA6EE265ABDEEC56A72
:1075C80016EE10EA16EE107AE645A8BF67468E4515
:1075D800B8BF0F46FEF7FEB9664ED4ED017A94EDBA
:1075E800006A3188726977EEA77AF0EE006AB0EE29
:1075F800677AA6EE267A4E1E04EBC601D6EE267AE8
:1076080008391032F6EE003A27EE237A67EEA37AAD
:1076180084ED207AC4ED217A574C274604F1800086
:1076280091ED027A91ED036AD7ED036AD7ED027AFC
:1076380052ED014A12ED025A37EE674A76EEC65A03
:1076480077EE277AE4EE845A013EA1F10801E5EECF
:10765800047A07F1080702F1080236EE267A00F1EB
:107668000800E4EE877AE5EE475A67EEA37A25EE3E
:10767800A37AC0ED007A80ED017AD1D1BEF1140F62
:107688007EF417AF06F070F9069BDFF80081C01A88
:10769800A8F80200D4F81451FEF70BBFD4F818313B
:1076A800B4F810C1354ACCF120095FFA89F90CEB1E
:1076B800431702EB87075FEA990201F0F28501326E
:1076C80016012F482F4907EB060807F1100212EDA3
:1076D800024A12ED035A12ED016A12ED047A50EDD6
:1076E800024A50ED035A50ED016A50ED047A64EEF7
:1076F800244A65EE255A66EE266A67EE277A103226
:10770800904541ED024A41ED035A41ED016A41EDD0
:10771800047A00F1100001F11001D8D11A48A6F13D
:1077280010010F4400EB0108214419F0030209D0AD
:10773800B7EC017AF8EC017A67EE277A013AE1ECC6
:10774800017AF5D1BCF1000F41F03180BEF1140F80
:107758007EF4AFAE06F008F9069BDFF83080D4F867
:107768001451C01AA8F80200FEF7A3BE085800205A
:10777800305200208C520020101E0020A4520020FD
:1077880034540020201E0020245400208C40002067
:10779800D04E318873684FEA51094FEA89005FEA91
:1077A800D10C04EB000204EB810500F0A18000F18C
:1077B80010010CF1010CC84F02EB0C1C29441032CB
:1077C80003F1100E05F1100050ED032A50ED043AB4
:1077D80017ED043A17ED032A50ED026A10ED016A1D
:1077E80017ED021A57ED010A11ED044A11ED035A7B
:1077F80052ED044A52ED035A12ED027A52ED017A23
:1078080051ED021A11ED010A73EE238A32EE228A33
:1078180047ED048A07ED038A71EE268A30EE868AE0
:1078280047ED028A07ED018A74EE848A35EE858A6F
:1078380042ED048A02ED038A77EE218A37EE808AC8
:1078480042ED028A02ED018A73EE633A75EE655ADB
:107858001EED035A32EE623A74EE644A25EE638AEC
:107868001EED044A23EE052A64EE652AA3EE048A77
:107878001032944524EE843AA3EE842A07F11007C7
:107888000EF1100EA5EE853A00F1100001F110017D
:10789800E4EE852A00ED078A00ED082A01ED073A93
:1078A80041ED082A5EED055A1EED065A71EE666A2C
:1078B80030EEC66A31EEC77A70EE677A26EE253A60
:1078C80065EEE63A25EE674A67EE054AE6EE053AC2
:1078D800A6EE853AA7EE254AE7EEA54A00ED063A58
:1078E80040ED053A01ED064A41ED054A7FF46CAFDB
:1078F8001FFA89F91A46494678481EF0BFFA726895
:10790800494628461EF0BAFA059B1A78142A7FF4CD
:10791800C1AEB7E6D4F8185171497248724BEA0003
:10792800114415448A88196800EE102A643AC82A56
:10793800A8BFC822782AB8BF782207EE902AB8EEE6
:10794800C07AF8EEE77A00EB850577EE670A77EEFE
:10795800876A67EE877A20EEA67AB8EE400AC7EE05
:10796800870A2846D5F81490D5F81880EF692E6A4A
:107978001EF072FE059BC5F8149093F800E0C5F858
:107988001880BEF1140FEF612E6201F0A484D4F8C0
:107998001821564BD4F81451013283FB0213A3EB80
:1079A800E27303EB4303D31A0135C4F81831C4F862
:1079B800145175E6474E4948B268B18929F0C6F9AD
:1079C800059B93F800E0BEF1140F01F09184D4F800
:1079D80014510135C4F81451FFE5454E31785FEA7A
:1079E800910C01F0AC85434F0CF101094FEA49199C
:1079F80007EB090807F12002A7F1700012ED076AEA
:107A080052ED056A12ED037A52ED017A52ED025AEF
:107A180012ED084A52ED064A12ED045A26EE066A9D
:107A280066EEA66A27EE077A67EEA77AA4EE046ADE
:107A380020329045E4EEA46A00F11000A5EE057A24
:107A4800E5EEA57AF1EEC65AB1EEE66AF1EEC76A3E
:107A5800B1EEE77A40ED085A00ED076A40ED066A94
:107A680000ED057ACAD1A9F120023A4404EB0C17BB
:107A780011F0030018BF08320FD052ED017A12ED51
:107A8800027A67EEA77A0138E7EE077A02F1080270
:107A9800B1EEE77AA7EC017AEFD1BEF1140F01F04D
:107AA8000A840135C4F81451FEF772BC05F05CFF76
:107AB800059B069093F800E0BEF1140F05BFDFF8B0
:107AC8003880D4F81451D4F81451A8F80050FDF7B0
:107AD80056B800BF8C520020201E0020101E002027
:107AE8007C550020E04B00204C4C00205655555545
:107AF80086520020901E00208C400020306E99BCD9
:107B08002716983DA40DC93F843459BEDB0F494060
:107B1800D06D393A00000000F0EEE76AB7EE005A7F
:107B280035EE665A1FED0B4A5FED0B5A1FED0A6AD8
:107B38001FED0C7A94ED6B0AF1EEC54AE6EE845A15
:107B4800F5EEC07AA6EEA56AF1EE10FAA6EE867AF0
:107B580048BF5FED127A27EE247A48BF37EEC77A1E
:107B680027EE000A2AF000FAB0F5617F00F38D864F
:107B780007EE900AF8EEE76A5FED1B7A66EEA76AF1
:107B880007EE905ABDEEE67AF8EEE77A17EE103A6D
:107B98002033402B41F281841FED220A2AF0E4F9B8
:107BA80000B207EE900AB8EEE77AFFF7BEBAC2490C
:107BB800C24B89681B6899423FF696AA3B780C3BF2
:107BC800022B7EF6A3A9BE4C3A702378002B3EF414
:107BD8009DA900232370FEF799B9BA4A02F150050E
:107BE80003E00432954200F069821378262BF8D11D
:107BF8009678D3789E42F4D2FFF7EDBAB24DB34FE0
:107C080095ED004A95ED057AD5ED014A95ED066AA0
:107C1800D5ED046A95ED035AD5ED025A67EE897AD7
:107C280007EB8602A4EE277AA4EEA76A66EEC76A77
:107C3800A5EE476AE5EEA76A20EE070A85ED056A14
:107C4800C5ED066A82ED007A29EE088A2AF08CF9D9
:107C580069EE288AD5ED0E5AD5ED176A95ED091A01
:107C6800D5ED121A95ED0F5A95ED187A95ED0A2A69
:107C7800D5ED132A95ED0D6AD5ED167A95ED0C3AEA
:107C8800D5ED0B3A95ED154AD5ED144AE1EE085AB3
:107C9800002207EB8601E8EEA16A00B2C4F80021D1
:107CA800A2EE085AC4F80421C4F80821A8EEA27A62
:107CB80026EE656A67EEE67AA3EE655AA3EE886A51
:107CC800A6EEC47AE8EEA47A85ED0E5AC1ED205AE4
:107CD80085ED0F6AC1ED406A85ED177AC5ED187A12
:107CE800FEF710BBD4F89C51079B5D1BFEF710BA3A
:107CF800BBF93820CBF8201007EE902A0121F8EEC6
:107D0800E77ACBF86020CBF87C100022012FCBED6E
:107D18001C7ACBED1B7ACBF8742001F09D82B74218
:107D28007CF491AFBBF93A20CBF8642007EE902A97
:107D380000210122F8EEE77ACBF82410CBF8902046
:107D48000022012FCBED217ACBED207ACBF88820C9
:107D580001F08682B7427CF4AAAFBBF93C20CBF88D
:107D6800682007EE902A00210122F8EEE77ACBF886
:107D78002810CBF8A4200022012FCBED267ACBEDDA
:107D8800257ACBF89C207CF4C6AF9FED518A032D51
:107D980049D04CB107EE904AF8EEE77AF4EEC87A8B
:107DA800F1EE10FA01F1D0834A4A4B4C1168DBF826
:107DB8006820A8F8060094F8200102EB560292FB0E
:107DC800F6F60022CBF828608A620A63CA6228B1F4
:107DD800424A126832F480637CF4A0AF404A1268C9
:107DE80012F4003241F030823E481146835C012B88
:107DF80002F10C0200F0778301311829F6D1FCF763
:107E08008DBF39494B69002B3DF46DA83748384B75
:107E1800008893FBF0F00B684FF0010E186081F8B2
:107E280011E0FDF760B8B0EE480A2AF09DF800B2FC
:107E3800AFE714F00BF92F4A0292A2F10C032521A7
:107E480001930091A2F10A035021163A49201AF031
:107E580035FBA8B9284BAA7818604FF0FF31596054
:107E680007233B70FFF73DB9DFF88C8014F0EEF87C
:107E7800224AD8F80430126864339342C1F07C83F4
:107E8800AA78FFF72EB91E4B1B78D90701F16A8330
:107E98001F2027F037FA0028F2D00C233B70EFE7B9
:107EA8001F20069227F02EFA069A00287FF419A9B7
:107EB80001233B70FFF715B9901900205852002094
:107EC800715F00201863002010550020A452002084
:107ED80000000000F43C0020101E0020CC430020CD
:107EE800B8450020884F0308346500204C65002001
:107EF80020A10700E634030804610020546500202F
:107F0800034000201A2027F0FDF900283FF4E6A8D6
:107F18009B4B1B88002B7FF4E1A89A4B4520D3F894
:107F2800008023F031F90E2023F02EF9404623F08B
:107F380021FADDF81C80404623F01CFA924A934B44
:107F480012681A6040460A233B7023F0BDFAFFF717
:107F5800C5B8012A01D1F9F78DFC0D2313203B7018
:107F68000DF0D2F8AA78FFF7BCB8894B89495B684D
:107F78000968C8338B4205D314F08CF8AA78002816
:107F88003FF4AFA8032A93D1DFF84082D8F8000065
:107F98000CF0BCFB804B1B780022022BC8F8002099
:107FA80001F00384AA7883E7012A01F0D4820E2322
:107FB80013203B700DF0A8F862E714F047F823F09F
:107FC8007BFD00283FF45CAF14F064F800283FF410
:107FD80057AF6D4A6D4B12681A600A233B70AA7836
:107FE800FFF77FB814F032F86C4B002105208DE8BC
:107FF8000300A3F10802029153201AF05FFA002847
:108008007FF43EAF624BAA78186008233B70FFF7F5
:1080180068B8604B5E491B684B60614800230B6081
:10802800032103603970FFF75CB8DFED5E7A5E4BC1
:1080380094ED687AC3ED007AC3ED017AC3ED027A54
:108048005A4BF0EE674AF0EE673A1968FDF746B901
:10805800574A584DD2ED006A574A95ED006A127892
:10806800C4ED646A84ED656A002A00F01F8276EE2A
:10807800665A94F99821C4ED615A0132C4ED626AD6
:1080880000F08985079BC4F89C31002537EE677A94
:10809800FCEEE77A494E84ED687A17EE902AA4F848
:1080A8008C21FF2296ED005A84F89821FEF740B8FB
:1080B800434B1D7805F00108FDF7AEBC3C4A3D4D29
:1080C800D2ED007A3C4A95ED007A1278C4ED647AD4
:1080D80084ED657A002A00F0658377EE676A94F983
:1080E8009821C4ED616A0132C4ED627A00F0DB8642
:1080F800079BC4F89C3100259FED2A7A2F4E84ED0A
:10810800687AFF2296ED005A84F89821FEF710B895
:108118002C49DFED2D7A0968C4ED4C7A11F08053B3
:108128000A9340F0A683DAF8001011F480030A934A
:1081380000F0CF8100230A93B6EE007A67EE877AC3
:10814800F4EEE57AF1EE10FAC8BFF0EE675A40F3A4
:108158009083C4ED685AFDF70BBB73EEE77AB7EE70
:10816800007AF4EEC77AF1EE10FAC4ED4C7A41F3D6
:108178008F8084EEA77A8DED0E7AFDF7EEBA00BFF8
:10818800785F0020745F0020885F0020805F0020F7
:1081980004610020546500205052002094360308E2
:1081A800EC3E00200000000008520020D4430020CC
:1081B800A05F00208C580020804E0020A05800208E
:1081C80003400020F860002000000080F03E0020FE
:1081D800D14D0D9B9DED0E5A95ED006A002B00F0D8
:1081E8001B8725EE866ACD48A5EE076AB0EE675A6A
:1081F800A6EE265ABDEEC56A16EE10EA16EE107AFD
:10820800E645A8BF67467145C8BF0F4606EE107A17
:10821800B8EEC66A012A80ED006A3DF401AC95ED1E
:10822800046A9DED0F5A25EE866AA5EE076AB0EE40
:10823800675AA6EE265ABDEEC56A16EE10EA16EE85
:10824800107AE645A8BF67467145C8BF0F4606EED7
:10825800107AB8EEC66A022A80ED016A3DF4E0ABF6
:1082680095ED086A9DED105A25EE866AA5EE076A17
:10827800B0EE675AA6EE265ABDEEC56A16EE10EAAB
:1082880016EE107AE645A8BF67467145C8BF0F4687
:1082980006EE107AB8EEC66A032A80ED026A3DF44B
:1082A800BFAB95ED0C6A9DED115A25EE866AA5EED9
:1082B800076AB0EE675AA6EE265ABDEEC56A16EEF4
:1082C80010EA16EE107AE645A8BF67467145C8BFA2
:1082D8000F4606EE107AB8EEC66A042A80ED036AE5
:1082E8003DF49EAB95ED106A9DED125A25EE866A17
:1082F800A5EE076AB0EE675AA6EE265ABDEEC56A25
:1083080016EE10EA16EE107AE645A8BF67467145E4
:10831800C8BF0F4606EE107AB8EEC66A052A80ED89
:10832800046A3DF47DAB95ED146A9DED135A25EE74
:10833800866AA5EE076AB0EE675AA6EE265ABDEE23
:10834800C56A16EE10EA16EE107AE645A8BF67462B
:108358007145C8BF0F4606EE107AB8EEC66A062AFF
:1083680080ED056A3DF45CAB95ED186A9DED145AF5
:1083780025EE866AA5EE076AB0EE675AA6EE265A7B
:10838800BDEEC56A16EE10EA16EE107AE645A8BFED
:1083980067467145C8BF0F4606EE107AB8EEC66A42
:1083A800072A80ED066A3DF43BAB95ED1C6A9DED0E
:1083B800155A65EE865AE5EE075AE6EEA57AFDEE01
:1083C800E77A17EE902A9445A8BF94468A42A8BF38
:1083D800614607EE901AF8EEE77AC0ED077AFDF7E6
:1083E8001FBBBEF1010F7FF7D0AC07EE103AB8EE15
:1083F800C77AC7EE876AB1EEE68AC8E4BEF1010F14
:1084080040F32E8707EE103AB8EEC77AC7EE876AB0
:10841800B1EEE68A032D13D04CB107EE904AF8EE80
:10842800E77AF4EEC87AF1EE10FA01F18D80DBF804
:10843800642002EB560292FBF6F2CBF8242089E482
:10844800B0EE480A29F090FD00B2E5E7BEF1010F51
:1084580040F3028707EE103AB8EEC77AC7EE876A8C
:10846800B1EEE68A032D13D04CB107EE904AF8EE30
:10847800E77AF4EEC87AF1EE10FA01F16580DBF8DC
:10848800602002EB560292FBF6F2CBF8202046E47D
:10849800B0EE480A29F068FD00B2E5E7F7EE006A99
:1084A800FDF78EBCF7EE006AFDF704BD76EEC65AFE
:1084B800F0EE466ADDE58222FDF7E8BFDFED187AC7
:1084C800FDF7B0BF174BD3F800E0BEF93270FEF7E6
:1084D8005EBAB6EE007AF4EEC75AF1EE10FA3FF73C
:1084E8002BAEFDF745B9D4F824614A003EB15518C2
:1084F80000EB850576786D78B542BCF40FAC0A447C
:1085080000EB82000022C4F82401A4F81022C4F869
:108518001422FCF703BC00BF08580020305200208A
:1085280000000243D443002095ED006A9DED0E4AF9
:10853800E34825EE866AFDEEE43AA4EE076AB0EE5B
:10854800674AA6EE264A13EE901AB4EEC45AF1EE24
:1085580010FAB0EE446A88BFB0EE646ABDEEC66A2F
:1085680016EE10EA16EE107AE645A8BF6746714582
:10857800C8BF0F4606EE107AB8EEC66A012A80ED2B
:10858800006A3DF449AA95ED046A9DED0F4A25EE6F
:10859800866AA4EE076AB0EE674AA6EE264AB4EEEB
:1085A800C45AF1EE10FAB0EE446A88BFB0EE646ABD
:1085B800BDEEC66A16EE10EA16EE107AE645A8BFBA
:1085C80067468E45B8BF0F4606EE107AB8EEC66A03
:1085D800022A80ED016A3DF41FAA95ED086A9DED17
:1085E800104A25EE866AA4EE076AB0EE674AA6EE40
:1085F800264AB4EEC45AF1EE10FAB0EE446A88BFC7
:10860800B0EE646ABDEEC66A16EE10EA16EE107A8F
:10861800E645A8BF67468E45B8BF0F4606EE107AF6
:10862800B8EEC66A032A80ED026A3DF4F5A995ED15
:108638000C6A9DED114A25EE866AA4EE076AB0EE33
:10864800674AA6EE264AB4EEC45AF1EE10FAB0EE26
:10865800446A88BFB0EE646ABDEEC66A16EE10EAD8
:1086680016EE107AE645A8BF67468E45B8BF0F4696
:1086780006EE107AB8EEC66A042A80ED036A3DF465
:10868800CBA995ED106A9DED124A25EE866AA4EEF7
:10869800076AB0EE674AA6EE264AB4EEC45AF1EE6F
:1086A80010FAB0EE446A88BFB0EE646ABDEEC66ADE
:1086B80016EE10EA16EE107AE645A8BF67468E4514
:1086C800B8BF0F4606EE107AB8EEC66A052A80EDE6
:1086D800046A3DF4A1A995ED146A9DED134A25EEAF
:1086E800866AA4EE076AB0EE674AA6EE264AB4EE9A
:1086F800C45AF1EE10FAB0EE446A88BFB0EE646A6C
:10870800BDEEC66A16EE10EA16EE107AE645A8BF68
:1087180067468E45B8BF0F4606EE107AB8EEC66AB1
:10872800062A80ED056A3DF477A995ED186A9DED56
:10873800144A25EE866AA4EE076AB0EE674AA6EEEA
:10874800264AB4EEC45AF1EE10FAB0EE446A88BF75
:10875800B0EE646ABDEEC66A16EE10EA16EE107A3E
:10876800E645A8BF67468E45B8BF0F4606EE107AA5
:10877800B8EEC66A072A80ED066A3DF44DA995ED64
:108788001C6A9DED154A65EE865AE7EE045AE6EE38
:10879800A57AB4EEE75AF1EE10FAC8BFF0EE647AA3
:1087A800FDF72AB977EEC76AF0EE477A97E4454AAB
:1087B8004FEA89075FEA9C09384402EBC313274450
:1087C80037D009F101094FEA091903EB090803F148
:1087D800100200F1100607F1100112ED024A12ED25
:1087E800035A12ED016A12ED047A56ED024A56ED6B
:1087F800035A56ED016A56ED047A64EE244A65EE92
:10880800255A66EE266A67EE277A1032904541EDC2
:10881800024A41ED035A41ED016A41ED047A06F13D
:10882800100601F11001D8D1A9F110094B444844B0
:108838004F441CF0030C3EF489AFB3EC017AF0EC22
:10884800017A67EE277ABCF1010CE7EC017AF4D1E2
:10885800FEF77CBFBEF834309FED1B7A07EE903AE6
:10886800F8EEE77A194B67EE877AC3ED007AFDF7E1
:1088780025B9B7EE007A77EE677AF4EEE75AF1EEAB
:1088880010FA88BFF0EE675A63E407EE905ADFEDFE
:10889800106AF8EEE77A66EEA65A9FED0E5A9FED3B
:1088A8000E6A9FED0E7AA5EE856A26EEA55AA5EE0C
:1088B800867AE5EE076A26EEA70AFFF76FB900BFCA
:1088C80030520020A45200206F12833A000000208A
:1088D80084F9223F92E741B99730083C15A82ABE8F
:1088E80095ED006A9DED0E4ACC4825EE866AFDEEB0
:1088F800E43AA4EE076AB0EE674AA6EE264A13EEFB
:10890800907AB4EEC45AF1EE10FAB0EE446A88BF19
:10891800B0EE646ABDEEC66A16EE10EA16EE101ADC
:10892800E645A8BF61467745C8BF394606EE101A26
:10893800B8EEC66A012A80ED006A3DF4E0AF95ED15
:10894800046A9DED0F4A25EE866AA4EE076AB0EE2A
:10895800674AA6EE264AB4EEC45AF1EE10FAB0EE13
:10896800446A88BFB0EE646ABDEEC66A16EE10EAC5
:1089780016EE101AE645A8BF6146BE45B8BF39468F
:1089880006EE101AB8EEC66A022A80ED016A3DF4B6
:10899800B6AF95ED086A9DED104A25EE866AA4EEFD
:1089A800076AB0EE674AA6EE264AB4EEC45AF1EE5C
:1089B80010FAB0EE446A88BFB0EE646ABDEEC66ACB
:1089C80016EE10EA16EE101AE645A8BF6146BE4537
:1089D800B8BF394606EE101AB8EEC66A032A80ED0B
:1089E800026A3DF48CAF95ED0C6A9DED114A25EEB7
:1089F800866AA4EE076AB0EE674AA6EE264AB4EE87
:108A0800C45AF1EE10FAB0EE446A88BFB0EE646A58
:108A1800BDEEC66A16EE10EA16EE101AE645A8BFB5
:108A28006146BE45B8BF394606EE101AB8EEC66AAA
:108A3800042A80ED036A3DF462AF95ED106A9DED5E
:108A4800124A25EE866AA4EE076AB0EE674AA6EED9
:108A5800264AB4EEC45AF1EE10FAB0EE446A88BF62
:108A6800B0EE646ABDEEC66A16EE10EA16EE101A8B
:108A7800E645A8BF6146BE45B8BF394606EE101A9E
:108A8800B8EEC66A052A80ED046A3DF438AF95ED64
:108A9800146A9DED134A25EE866AA4EE076AB0EEC5
:108AA800674AA6EE264AB4EEC45AF1EE10FAB0EEC2
:108AB800446A88BFB0EE646ABDEEC66A16EE10EA74
:108AC80016EE101AE645A8BF6146BE45B8BF39463E
:108AD80006EE101AB8EEC66A062A80ED056A3DF45D
:108AE8000EAF95ED186A9DED144A25EE866AA4EE40
:108AF800076AB0EE674AA6EE264AB4EEC45AF1EE0B
:108B080010FAB0EE446A88BFB0EE646ABDEEC66A79
:108B180016EE10EA16EE101AE645A8BF6146BE45E5
:108B2800B8BF394606EE101AB8EEC66A072A80EDB5
:108B3800066A3DF4E4AE95ED1C6A9DED154A65EEB6
:108B4800865AE7EE045AE6EEA57AB4EEE75AF1EE55
:108B580010FAC8BFF0EE647AFDEEE77A17EE901AC5
:108B68008C45A8BF8C468F42D8BF674607EE907ADF
:108B7800F8EEE77AC0ED077AFDF7BEBE28494A69E4
:108B8800002A3CF499AA0A6813604B74FCF794BA5B
:108B9800244DFDF70BB8D4F89C51079B5D1BFFF7DC
:108BA80075BA214B1B78DA0704D41CF093FC002813
:108BB80040F068851D4DD4F80C222B689A423EF689
:108BC8009AAA3B78012B3DF4A1A9194C2278002AD6
:108BD8003DF49CA90B2B19D801229A4040F60301B9
:108BE80012EA01087EF4F5AF12F4C06F0ED0093B0B
:108BF800012B0BD8452022F0C7FAFF2022F0C4FA37
:108C08000C4822F037FA404622F0BEFA0A4B2A688E
:108C18005A600B233B70FEF7DCBF00BF30520020C8
:108C280034650020A0410020034000205465002046
:108C3800715F0020C05D0308046100200D9B002BBC
:108C480000F07183E34D9DED0E4A95ED006A089B97
:108C580025EE866AA4EE076AB0EE674AA6EE264AB3
:108C6800B0EE446A33B1B4EE445AF1EE10FAC8BF1C
:108C7800B0EE646AFDEEE44ABDEEC66A14EE907A80
:108C880016EE101A8F4214EE90EA00F3F384614551
:108C9800A8BF614606EE101ACF48B8EEC66A012A88
:108CA80080ED006A3CF4BCAE95ED046ADDED0F4A38
:108CB800089B25EE866AA4EE876AF0EE674AE6EE20
:108CC800264AB0EE646A002B00F0CA84B4EEE45A77
:108CD800F1EE10FA40F3C48439466145A8BF6146F5
:108CE80006EE101AB8EEC66A022A80ED016A3CF454
:108CF80097AE95ED086ADDED104A089B25EE866A69
:108D0800A4EE876AF0EE674AE6EE264AB0EE646A99
:108D1800002B00F09B84B4EEE45AF1EE10FA40F315
:108D2800958439466145A8BF614606EE101AB8EE2B
:108D3800C66A032A80ED026A3CF472AE95ED0C6AAD
:108D4800DDED114A089B25EE866AA4EE876AF0EEEF
:108D5800674AE6EE264AB0EE646A002B00F06C849F
:108D6800B4EEE45AF1EE10FA40F3668439466145F0
:108D7800A8BF614606EE101AB8EEC66A042A80ED4E
:108D8800036A3CF44DAE95ED106ADDED124A089B7E
:108D980025EE866AA4EE876AF0EE674AE6EE264A72
:108DA800B0EE646A002B00F03D84B4EEE45AF1EEB4
:108DB80010FA40F3378439466145A8BF614606EE8C
:108DC800101AB8EEC66A052A80ED046A3CF428AE8B
:108DD80095ED146ADDED134A089B25EE866AA4EE2C
:108DE800876AF0EE674AE6EE264AB0EE646A002B20
:108DF80000F00E84B4EEE45AF1EE10FA40F3088461
:108E080039466145A8BF614606EE101AB8EEC66A33
:108E1800062A80ED056A3CF403AE95ED186ADDED8F
:108E2800144A089B25EE866AA4EE876AF0EE674A24
:108E3800E6EE264AB0EE646A002B00F0E083B4EE5A
:108E4800E45AF1EE10FA40F3DA8339466145A8BFD7
:108E5800614606EE101AB8EEC66A072A80ED066A61
:108E68003CF4DEAD95ED1C6ADDED154A089B65EE18
:108E7800865AE4EE875AE5EEA67A002B00F0B7830F
:108E8800F4EEC57AF1EE10FA40F1B1833A46624544
:108E9800A8BF6246964607EE90EAF8EEE77AC0ED7C
:108EA800077AFCF7BDBDD4F89C51079B5D1BFFF703
:108EB80023B907EE905ADFED496A9FED497A84F8A5
:108EC8000452F8EEE77A67EEA67A77EE876ABDEE87
:108ED800E66A16EE103A2033402B40F29782DFED17
:108EE800416A414BBDEEE77AC3ED016A17EE103ACD
:108EF8002033402B00F260829FED3C7AF4EEC77A73
:108F0800F1EE10FA40F3CA83DFED395A9FED396A62
:108F180001E0F0EE477AF4EEC67AF1EE10FA37EE99
:108F2800E57AF6DCDFED347AB4EEE77AF1EE10FAA2
:108F380040F1B183DFED2E5A9FED306A01E0B0EECB
:108F4800677AB4EEC67AF1EE10FA77EE257AF6D49F
:108F58009FED237AF4EEC77AF1EE10FA40F3E3823C
:108F68009FED227A77EE677A67EEA75A9FED245A2B
:108F78009FED246A9FED247AA5EE856A27EEA55A0F
:108F8800A5EE867AE5EE077AC4ED827AFDF77ABD1A
:108F980095ED000A0893069228F0E6FF1B49DFF8D2
:108FA80070E0D1F8EC10DFF86CC0069AACF800005D
:108FB8008EFB013EC917C1EBAE1107EE901AF8EE11
:108FC800E77A089BFDEEE77A17EE901AACF80210E4
:108FD800FCF7F1BD085800203052002035FA8E3CCD
:108FE800DB0FC93F0000000000000020DB0F4940F4
:108FF800DB0FC940E4CB1641DB0F49C0E4CB16C1F7
:1090080092E741B99730083C15A82ABEF80000201D
:10901800D34D62108C40002025EE866AA5EE076AC3
:10902800B0EE675AA6EE265ABDEEC56A16EE100ACD
:10903800814200F36C816045A8BF604606EE100AC5
:109048000A9BB8EEC66A002B00F0FF83DC48012AB1
:1090580080ED006A3CF4E4AC95ED046A9DED0F5A8E
:1090680025EE866AA5EE076AB0EE675AA6EE265A7E
:10907800BDEEC56A16EE107AB94200F3468167451F
:10908800A8BF674606EE107A0A9BB8EEC66A002BA0
:1090980000F09883022A80ED016A3CF4C1AC95ED9A
:1090A800086A9DED105A25EE866AA5EE076AB0EEAD
:1090B800675AA6EE265ABDEEC56A16EE107AB94270
:1090C80000F32D816745A8BF674606EE107A0A9B14
:1090D800B8EEC66A002B00F09383032A80ED026A7B
:1090E8003CF49EAC95ED0C6A9DED115A25EE866A0E
:1090F800A5EE076AB0EE675AA6EE265ABDEEC56A17
:1091080016EE107AB94200F308816745A8BF674692
:1091180006EE107A0A9BB8EEC66A002B00F066834A
:10912800042A80ED036A3CF47BAC95ED106A9DED52
:10913800125A25EE866AA5EE076AB0EE675AA6EEC1
:10914800265ABDEEC56A16EE107AB94200F3E380DE
:109158006745A8BF674606EE107A0A9BB8EEC66A4E
:10916800002B00F0B182052A80ED046A3CF458AC6B
:1091780095ED146A9DED135A25EE866AA5EE076AE9
:10918800B0EE675AA6EE265ABDEEC56A16EE107AFC
:10919800B94200F3BE806745A8BF674606EE107A5D
:1091A8000A9BB8EEC66A002B00F01683062A80EDEB
:1091B800056A3CF435AC95ED186A9DED145A25EE18
:1091C800866AA5EE076AB0EE675AA6EE265ABDEE85
:1091D800C56A16EE107AB94200F3A3806745A8BFA6
:1091E800674606EE107A0A9BB8EEC66A002B00F0B6
:1091F8007582072A80ED066A3CF412AC95ED1C6A6C
:109208009DED155A65EE865AE7EE055AE5EEA67A03
:10921800FDEEE77A17EE902A914203DC6245A8BF7B
:109228006246114607EE901A0A9BF8EEE77A002B81
:109238007FF435AE0C9B002B7FF431AE0B9B9E4523
:10924800B8BFF0EE647A2AE65E4A1278032A00F084
:1092580015820022FEF7C8BD9FED5B8AFFF702B9B1
:109268009FED598AFFF7D6B89FED580ADFF870814D
:1092780025EE800A28F078FED4F81451A8F80600E4
:10928800FDF717B9D4F89C51079B5D1BFDF7C0BFCC
:109298004F49096811F080530A937EF44DAFFEF7E9
:1092A80042BF4C484C498046FEF73FBA079822F027
:1092B8000BF9FDF713BF04F057FB059BDFF820817E
:1092C80093F800E0069B3178D4F81451C01AA8F836
:1092D8000400FEF7E6BB04F047FB059BDFF80081BE
:1092E80093F800E0069BC01AA8F80200FEF74FBBEF
:1092F80004F03AFB059BDFF8E88093F800E0069B52
:10930800C01AA8F80200FEF762BB0F46BAE6084684
:1093180094E60F4642E70F461DE70F46F8E60F466C
:10932800D3E60F465DE70EA9BDEEE46A01EB8202C3
:1093380090462A48089A224D0A9B089416EE107AFD
:1093480005E04145A5EC016A00F1100031D090ED2F
:10935800006AB1EC014A25EE866AA7EE046AB0EE0F
:10936800674AA6EE864AB0EE446A32B1B4EE445A71
:10937800F1EE10FAC8BFB0EE646ABDEEC64A06EE5A
:10938800107A14EE104AA74206DC14EE104A64451F
:10939800A8BF644606EE104AB8EEC66A002BD0D1C4
:1093A8000C9C002CCDD10B9CA645B8BFB0EE646ACE
:1093B800C7E7089CFCF734BBDFED037AE4E500BFA0
:1093C8003052002034370020000000000000C8425E
:1093D800F860002024540020101E002008580020A7
:1093E8008C40002092E741B99730083C15A82ABE66
:1093F800E4CB1641DB0FC940E4CB16C1DB0FC93FF4
:10940800DB0F4940DB0FC9BFDB0F49C0F4EEC77A59
:10941800F1EE10FA40F355815FED0A5A1FED0C6A20
:1094280001E0F0EE476AF4EEC66AF1EE10FA36EEA5
:10943800E57AF6DC5FED0C6AB4EEE67AF1EE10FA46
:1094480040F12F815FED155A1FED156A01E0B0EE6E
:10945800667AB4EEC67AF1EE10FA77EE256AF6D49B
:109468001FED1A7AF4EEC76AF1EE10FA40F3B380F2
:109478001FED1D7A77EE666A66EEA65A1FED275A2B
:109488001FED276A1FED277AA5EE856A26EEA55AF5
:10949800A5EE867AE5EE076A23E51FED277AF4EE56
:1094A800C76AF1EE10FA40F38A815FED2E5A1FED7C
:1094B800306A01E0F0EE476AF4EEC66AF1EE10FA9F
:1094C80036EEE57AF6DC5FED306AB4EEE67AF1EE78
:1094D80010FA40F171815FED395A1FED396A01E0E8
:1094E800B0EE667AB4EEC67AF1EE10FA77EE256A37
:1094F800F6D41FED3E7AF4EEC76AF1EE10FA05DDF8
:109508001FED417A77EE666AFFF7C5B91FED437A1A
:10951800F4EEC76AF1EE10FA44BF1FED457A77EE14
:10952800666AFFF7B8B91FED497AF4EEC77AF1EE2B
:1095380010FA44BF1FED4C7A77EE677A14E5C84FEE
:1095480007F18002FEF794BAA8F80600ABF8A86005
:10955800C34CFBF7EABBF7F76DFF00283EF490AC6D
:10956800FEF725BD802026F019FF08B10BF0FAF8A8
:1095780019F0F8F8FEF78CBC402012F03FFD0028E7
:109588007EF47EACD8F80030DFF814A3DFF814B30B
:109598004FF040090EE021F0F7FDDBF80020D8F885
:1095A8000030013A0133B9F10109CBF80020C8F8BD
:1095B800003079D01AF803301846002BEBD100237D
:1095C8004FF0FF32C8F800300423C8F804203B707D
:1095D800AA78FDF786BD9FEDA37AF4EEC76AF1EE8F
:1095E80010FA44BF9FEDA07A77EE666A44E7FDEE75
:1095F800E77A17EE902ABA42FFF64DAC47E4BDEE83
:10960800C66A16EE101AB942BFF620AC394620E4F5
:10961800BDEEC66A16EE101AB942BFF6F2AB39466D
:10962800FFF7F2BBBDEEC66A16EE101AB942BFF6D6
:10963800C3AB3946FFF7C3BBBDEEC66A16EE101AB8
:10964800B942BFF694AB3946FFF794BBBDEEC66A84
:1096580016EE101AB942BFF665AB3946FFF765BB7F
:10966800BDEEC66A16EE101AB942BFF636AB3946D9
:10967800FFF736BB14EE901AFFF70CBB0BF028FD72
:10968800FBF74CBB794B1B6803F59C530833C4F8B4
:109698000C32FDF730BDF0EE477A59E4B0EE677A48
:1096A80040E4F0EE476ADBE61AF80330002B7EF45C
:1096B800E7AB84E794F87831002B7BF4CBADFBF76C
:1096C800B6BDB0EE667AB5E60C9B002B7FF44BADC9
:1096D8000B9B9E45B8BFB0EE646A44E50C9B002B1B
:1096E8007FF487AD0B9B9E45B8BFB0EE646A80E5FA
:1096F8005F4A604B10681B6898475F4BD7ED006A5C
:1097080093ED007A5D4BD3ED007A5D4B83ED020A51
:109718005C4B67EE277A2B4427EEAC7AD3ED007AC0
:10972800594B67EE277AF0EE665AEDEEA75A93ED9D
:10973800006AB1EE467AB4EEE57AF1EE10FA08DC8A
:10974800F4EEC65AF1EE10FA8CBFB0EE467AB0EEDF
:10975800657A4E4B1B78012B02D0192B7BF4E4ACB5
:10976800DFED4B7AF4EEE7DAF1EE10FACCBF012325
:109778000023FBF7E4BC474BD3ED007AB1EE677AE0
:10978800F4EEC7DAF1EE10FA13D4F4EEE7DAF1EEFC
:1097980010FA88BFF0EE67DA3F4B87ED00CA1B6806
:1097A8009342BBF6AFABFBF713BC0BF0EBFBFEF73A
:1097B800F9BBF0EE47DAEFE7F0EE476A99E6B0EE6C
:1097C800667A80E60C9B002B7FF464AC0B9B9E456D
:1097D800B8BFB0EE646A5DE40C9B002B7FF4E6AC86
:1097E8000B9B9E45B8BFB0EE646ADFE40C9B002B70
:1097F8007FF496AC0B9B9E45B8BFB0EE646A8FE4CD
:109808000C9B002B7FF469AC0B9B9E45B8BFB0EE58
:10981800646A62E4132B05D1B0EE480A28F0A4FB71
:10982800099B1880B0EE480ADBF808321B489847B5
:10983800059B1B78132BB0EE408A7CF4F2AE28F01F
:1098480093FB099B5880FCF7ECBE0C9B002B7FF424
:10985800FDAB0B9B9E45B8BFB0EE646AFFF7F6BB45
:10986800101E0020DB0FC9BFDB0F49C05465002064
:10987800745700208857002000000020C856002098
:10988800FC51002098570020005800202C5600203A
:1098980000009642FC570020E0570020E04B0020D3
:1098A80080340308EC3E00202DE9F04F2DED068BA7
:1098B800A04BA14A1C7897B000F59C412031814605
:1098C8000B911160002C00F0EA869C4A12689042C5
:1098D80040F283809A4A069216689A499A4A0591F4
:1098E800013C1C70994B049206F480560893002E94
:1098F80040F08180964B1B78022B01F09481042B59
:1099080001F08381012B01F03781924B9945089B27
:109918009B7800F29685002B40F097858E4B079335
:10992800069B1E6816F4805740F08786DFF860A211
:10993800049BB3F90610059B5D8BA942B4BF0025B3
:109948000125864B1B6813F080535ED0079A127866
:1099580012F001025FD00598408C884241F3B8822A
:10996800002D5ED17E4C94F88C10002959D17D4889
:109978007D49006890F82D0000240C604C608C60D4
:109988007A4900284ED10870002A4FD0F0064DD5EC
:10999800774A1278D10649D4002F47D1002B45D1F8
:1099A800720243D4734B1B78002B02F01982724B5E
:1099B8009B78002D42F081823BB1704A704B12684F
:1099C8001B689B1A002BC2F26D821020644C0BF0AE
:1099D8009BFB012384F88D3028E0594B06931E68C1
:1099E800594B584A049306F48056584B05920893ED
:1099F800002E3FF47FAF00215848F7F7B5FC002848
:109A08007FF478AF0DF0FAFC74E774029ED4079ADD
:109A1800127802F00102524C002184F88C10002DBB
:109A2800A5D0524901200870002AAFD1554B1A78A9
:109A3800002A40F0BD800599049C488BB4F9007059
:109A4800898BB4F90240B842B4BF8026002646F09C
:109A58004003B942D8BF33469B0843F08006A04272
:109A6800B8BF3346049F43F04006A142C8BF3346FF
:109A78009B08B7F90440B7F9066043F08007A04295
:109A8800B8BF3B4643F04007A142C8BF3B469B08CE
:109A980043F08007324C8642C8BF3B4643F040073C
:109AA80094F88EE08E42B8BF3B469E4501F04A844A
:109AB800A4F8902084F892202E4984F88E300E78ED
:109AC800002E01F04B835F2B01F0BE836F2B01F05A
:109AD800FD83079B1B78DE076AD494F8921000294F
:109AE80066D1B4F99030322B62DD94F88E200120D3
:109AF800572A84F892004DD0069B1B685D0741F1F8
:109B080099825A2A41F0968294F89430002B42F0B8
:109B18005E8194F8963083F0010384F89630002B28
:109B280042F0D6810C200BF0EFFA174B174D099332
:109B380041E000BF585D0020605C0020545D0020BB
:109B48005C4C0020D8590020FA71002020340020F5
:109B5800C25C0020404B4C0003400020F86000200D
:109B68002C200020D443002008520020881F002009
:109B78007C520020CC1B002054610020546500203A
:109B8800BC3300208F340020D8430020D04300206D
:109B980068630020884B894A19684FF47A73B3FBCD
:109BA800F1F3C3EB431103EB8103DB00A2F8A83008
:109BB800834B844D0993069B1B685F0700F1B486AD
:109BC8000DF15009804E0A950022C9F80420344648
:109BD800149240F6330B4FF0190840F28337049D76
:109BE80002E00434544522D0A178E378994218FB66
:109BF8000170F6D294F801E00EF1040E18FB03711F
:109C080035F91E305B45A8BF5B46B3F5617FB8BF29
:109C18004FF461739842E4DA9942E2DB217827290C
:109C2800DFD848460434F7F78FFB5445DCD1674A40
:109C38000A9D1378664A99E8030082E80300002B1E
:109C480040F0F085634B1A78002A00F06A850121FC
:109C58005F48F7F789FB002840F0E782089BDB782C
:109C6800002B40F0E2825C4B0A932B881FB227F04E
:109C780001071FFA87F84345A5F8008001F0028024
:109C8800564F4FF002090E204FF0140A4FF0FF0B09
:109C980087F8009087F801A087F802B00BF034FA33
:109CA80049464B48B5F80080F7F75EFB002841F0BD
:109CB8009A8228F002039BB243452B800BD0474B76
:109CC80002201421FF2218700E2059709A700BF090
:109CD8001BFAB5F80080424B424A197850680B933A
:109CE80018F0030F08BF81F00201C1F340010C9284
:109CF80007F09CFC24213648F7F736FB30B9079A61
:109D080013785F0744BF23F0040313700A9B1B6892
:109D180013F00A0F11D006212D48F7F725FB00286C
:109D280001F0AD802B88580641F12582072128488B
:109D3800F7F71AFB002840F0C8870C212448F7F7EA
:109D480013FB2A88002800F0508342F480739A425B
:109D58002B8009D0214B022214211A700E20FF22D9
:109D680059709A700BF0D0F91F4B1B78082B00F034
:109D780048830E2B00F04583069BD3F8008018F427
:109D8800806F6BD0194B1B79002B00F030821421A7
:109D98000F48F7F7E9FA002840F02E8210F072FB1E
:109DA80001200BF0B9F8002855D0DFF844A00027AF
:109DB8004FF0CC0BA14620E04C4C0020D4490020A9
:109DC800D8430020D043002018630020804E002094
:109DD800F8600020C93300207C430020F4460020AE
:109DE8001C65002020650020705200209041002052
:109DF800046F0020DFB2022F2CD80BFB07F87B1C66
:109E08005AF80840002CF5D1032290F90230029448
:109E18000192C278E24951F822200092184622465F
:109E2800234601210AF0B6FC034607EB470000EB86
:109E380000100A9353B121460AEB8000CC2229F086
:109E480050F80A9B4AF808300137FFB21CF0BAFFF5
:109E58000028D0D14C46069BD3F80080079B93F886
:109E680000A0D04B1AF0010A00F0418201221A70BA
:109E7800099B04991B68B1F906105A89CA48012739
:109E88009142077080F21982C84B4FF07E521A60D7
:109E9800059BC74FB3F81890049B97F90420B3F9B2
:109EA8000030387897F801C0002AA3EB090714BFDF
:109EB80001224FF0FF32002FB8BF7F42B7F5FA7F7B
:109EC800A8BF4FF4FA77B84280F2F4813F1A07EE40
:109ED800907AF8EEE77AB74F4B45C7ED007A03DA88
:109EE800F1EE677AC7ED007A049BB3F902E0AEEBB6
:109EF8000903002BB8BF5B42B3F5FA7FA8BF4FF444
:109F0800FA73984280F2D3811B1A07EE903AF8EE62
:109F1800E77AF145C7ED017A03DDF1EE677AC7ED1F
:109F2800017A049BB3F90400A0EB0903002BB8BF26
:109F38005B42B3F5FA7FA8BF4FF4FA736345CCBF11
:109F4800A3EB0C03002302FB03F207EE902AF8EEC2
:109F5800E77A4845C7ED027ABCBFF1EE677AC7EDEC
:109F6800027A18F4805800F07F81B1F5FA6F924BAD
:109F7800A8BF4FF4FA61B1F57A7F1A78B8BF4FF4E9
:109F88007A71A1F57A71002A41F01D818B4ADFF8B8
:109F980044E282FB0130CB17C3EB6013581C6FF00F
:109FA800630C3EF910003EF913E00CFB0313A0EB21
:109FB8000E0003FB00F382FB0312DB17C3EB6213F3
:109FC8009E440FFA8EFE07EE90EAB8EEE78A87ED18
:109FD800038AB8F1000F40F066842B885A0640F1D6
:109FE800FB807749774A91ED018AD2ED019A92ED8B
:109FF800026A91ED034A92ED030A91ED029A92EDFD
:10A00800007AD1ED005AD7ED011A97ED002A6E4A71
:10A018006E4938EE445A79EEC63A77EE007A65EE24
:10A02800233A75EEC96A75EE890A37EE401A66EE6C
:10A03800A76AB0EE633AA0EE813A13F00303B0EEDC
:10A04800665A78EE044A79EE867AA0EE815AF0EEE6
:10A05800638AA4EEA73AD4EEA78AA4EEE75A33EEB1
:10A06800263AF0EE687AF0EE674AF6EE008A35EEA8
:10A0780088AAE0EEC14A28EEC33A35EE635A77EE75
:10A08800293A77EEE67AAAEE233A25EE285A76EEB2
:10A09800403A34EE49AAE0EE817A74EEA64AAAEE76
:10A0A800235A34EE094A37EE697A64EEA84A63EE19
:10A0B800036AE4EE074A75EEC85A36EE006A67EEA0
:10A0C800A87AB0EE667A95EE057AE5EE056AE5EED1
:10A0D800867AB1EE648AF0EE665AF0EE476AB1EE1F
:10A0E800674AE8EE246A63EE270A67EEA43AE4EECC
:10A0F800275AB1EE450AB0EE609AB0EE631AA4EEA4
:10A10800277A23EE244AE7EEA76AA5EE249AA0EE62
:10A11800031AE8EE245AB0EE448A31EEA16AE0EE62
:10A12800240AA5EE278A66EEA16A72EE028AE5EE97
:10A13800033A61EE211A26EE096AA4EEA47AA0EE8B
:10A14800274A0CBFD7ED022ADFED212A82ED005AFB
:10A15800A2EE256AE8EEA06AE2EE081A73EEA33AC8
:10A1680027EE227A34EE044AF0EE005AE3EEA26AB1
:10A17800A4EE226AA1EEA57AC7ED016AC1ED366A9E
:10A1880081ED356A87ED006A81ED377A82ED013A13
:10A19800C2ED027AC2ED034AF3B987ED027A1BE0F9
:10A1A8001C4A030804400020C01F00203C1F002058
:10A1B8002C610020A0410020EC2400201F85EB51D9
:10A1C800E0000020841B0020BC1B00202C20002065
:10A1D80000000000D4650020BAF1000F40F024818F
:10A1E80025F0E2FA17B0BDEC068BBDE8F08F079BAF
:10A1F8001B78D9077FF5D2AD4FF40F7026F0CEF853
:10A2080000283FF428AE0AF0ADFA4FF40F7026F09C
:10A2180067F800283FF41FAE0AF0A4FA4FF40F7055
:10A2280026F05EF80028EED115E69A4B0A931B68D3
:10A238009B077FF51AADB5F8008018F0010F7FF481
:10A2480038AD48F0010398452B803FF432AD924B6E
:10A25800022214211A700E20FF2259709A700AF0F7
:10A2680053FFB5F8008024E5059B5A8B9142C0F254
:10A278000685B1F5FA6FD4BFC2EB0101C2F5FA61E8
:10A288004FF47A7303FB01F184480378C2F5FA624C
:10A29800B1FBF2F1002B3FF479AE4378804A01FB21
:10A2A80003F182FB0123C917C1EB63116EE6DFEDF1
:10A2B8007D7A2EE6DFED7B7A0DE6B1F5FA6F80F256
:10A2C800D784187A8B1A03FB00F3C2F5FA6293FB62
:10A2D800F2F3C3F1640307EE903AF8EEE77A9FEDE4
:10A2E800727A724B67EE877AC3ED007AD0E51B78F5
:10A2F8000693002B7FF4BCAD6D4A1268002A3FF428
:10A30800B7AD6C4A079212F8030CDFF8E0B11146BA
:10A31800D71E24F0CDFF9BF80090079A002800F084
:10A328003086069BB9F1000F53D107F108017879FF
:10A3380024F0BEFF002841F02D855F49B87A24F04B
:10A34800B7FF002800F03086B9F1020F41F01E85F2
:10A358005A49F87B24F0ACFF002841F0138558498E
:10A36800387D24F0A5FF002800F03086B9F1040FED
:10A3780041F004855349787E24F09AFF002841F083
:10A38800F9845149B87F24F093FF002800F0308603
:10A39800B9F1060F41F0EA844C4997F8230024F0FC
:10A3A80087FF002841F0DE84494997F8280024F007
:10A3B8007FFF002800F03086B9F1080F41F0CE8405
:10A3C800444997F82D0024F073FF00283FF450AD5E
:10A3D80009231A4602EB820217443F4A7878B97873
:10A3E8008BF800301070517042E522F480739BB2F4
:10A3F8009A422B807FF4AEAC384B1B78082B7FF445
:10A40800B8AC2A8822F040039BB29A422B803FF4D2
:10A41800B3AC214B022214211A700E20FF2259706E
:10A428009A700AF071FEA7E40B9B19780C9B01F057
:10A438000101186807F0FAF817B0BDEC068BBDE803
:10A44800F08F13B9089A01239370254B089A1D7849
:10A4580092F8214007931B2024F054FF012C05F0AB
:10A468000108814600F0088705F00205089A1D4E8C
:10A4780092F82030DFF878A01B4F09959346052BFA
:10A4880000F29E87DFE813F0BE00B4003600FC003F
:10A49800FE00F1007C430020F4460020EC2400205C
:10A4A8001F85EB51000000000AD7233C3C1F002009
:10A4B80008400020AE460020B8460020BD460020D7
:10A4C800C2460020C7460020CC460020D1460020C6
:10A4D800D6460020DB4600200C40002070520020A9
:10A4E80003400020CC650020CC4300200800002059
:10A4F800CC1B0020012C04BF05238BF82030B8F1B9
:10A50800000F12D0059B3088B3F9181000221346AB
:10A5180061F30F0260F31F4261F30F03049861F3C4
:10A528001F430360032342600993BF4DDBF81410F7
:10A538002A68914280F0028647F230510322CBF814
:10A548001C108BF82020022008F098FB0CF056FF16
:10A558002968DBF81C200A440421CBF818208BF862
:10A568002010012C40F07D872A68DBF818109142F2
:10A5780080F026879AF8000020B924F0C3FE00284E
:10A5880040F01E873A6822F002023A602A6873880F
:10A59800642101FB03234FF480600022CBF81030C4
:10A5A8008BF820208BF8032008F038FB9BF820302C
:10A5B80065E724F0ADFE012807D19B4D72882B6812
:10A5C800642101FB0233CBF81030B9F1000F02D03F
:10A5D800B379002B4BD1012C00F0F286924DDBF8B9
:10A5E80010102A689142C0F0318701238BF820307F
:10A5F800012C3AD0F379012B46D024F017FE9BF8B2
:10A6080020303CE7B8F1000FD3D1099D4FF48060AA
:10A61800B9F1000F00F0568308F018FB089A0023E0
:10A628001361002D3FF47CA928460AF06DFD069BB6
:10A638001E6816F480573FF479A91D217B48F6F768
:10A6480093FE00287FF472A9794B03F1500A03E0C6
:10A6580004339A4500F0BA861A78262AF8D19978F0
:10A66800DA789142F4D2FFF763B96F4D8EE724F0A0
:10A67800DDFD03224FF47A738BF82020CBF81C30D1
:10A68800694D60E7684D6CE724F0D0FD032240F681
:10A69800B8338BF82020CBF81C30634D53E7654F57
:10A6A8003B78002B01F05782634BDFF89881DFF885
:10A6B80098B1DFF898A1059345465E4604909946FF
:10A6C8000EE019F804109847032C28DC88B93B7869
:10A6D8002AF8020F01349C4205F1040580F24981F1
:10A6E800072CE1B23046DBF80430EADD984700B2C7
:10A6F800EDE738F824206B88801A4FF47A719B1A9A
:10A7080001FB00F040F6CA0290FBF3F008449042C7
:10A7180040F2EE23A8BF10469842B8BF184600B2D0
:10A72800D5E7DFF82C91DFF82CA1444F0A9209F104
:10A738005A084FF0010B494619F8010C24F0B8FDEE
:10A7480000B399F8040099F8023099F803E000EB97
:10A75800400107EB8101013BD1F8A02003EB430343
:10A76800534493420ED097F8CC20C1F8A0300BFA8E
:10A7780000F022EA00000A9B81F89CE0C1F8A430AE
:10A7880087F8CC0009F10609C145D4D12C4B264ADB
:10A798001B780A93099BDFF8C0A012681B680B930B
:10A7A800AAF19C094FF0000B9046DAF8043083B305
:10A7B8001F7877B3DAF80820A8EB0202002A0CDB2E
:10A7C80099F8CC20012101FA0BF122EA010208F5DF
:10A7D800FA7189F8CC20CAF808100A9ACAB19AF80E
:10A7E800002059780432D2B2002940F0B583059987
:10A7F8000498098B30F9122001F1C800824240F315
:10A80800F78599F8CC109A7841FA0BF3D80740F1FC
:10A8180081860BF1010BBBF1040F0AF10C0AC4D1BC
:10A82800FFF715BA024B1DE054650020F8600020C0
:10A8380018630020DC630020D85900202C20002059
:10A848006D360020F4630020C04700202A20002035
:10A85800C5450020B4360308C820002004339C42B4
:10A868003FF4F0A919782329F8D19878DA7890423A
:10A87800F4D2AD48F6F778FD00283FF4E3A9AB4BD6
:10A888001B6813F4003341F013820022A84B1046D2
:10A89800995C142902F10C0201F0BC8001301828DF
:10A8A800F6D1FFF7CFB91D219F48F6F75DFD28B116
:10A8B80000F060BD0436B4423FF48FAB31782629EE
:10A8C800F8D1B278F3789A42F4D2089BDB78002B5F
:10A8D8007FF483AB9448F6F747FDDFED967A0028BE
:10A8E80001F0508138EE678A934A9449FDEEC87AA0
:10A8F800CDED047ABDF910301B0382FB0302DB1790
:10A90800C3EBA212C9F57A731BB203FB02F343F33C
:10A918000F334B4407EE903AF8EEE77A0123C7ED80
:10A92800037A0B70FFF759BB854C94F896305BB1EE
:10A93800079B1B78DE0707D5049BB3F90620059B08
:10A948005B8B9A4200F3D88511217748F6F70CFD06
:10A95800002800F0AB8294F89A302BB994F8943020
:10A9680013B93223A4F89830012384F89A30FFF7FA
:10A9780027B9DDF81090734A06926F49126842F2BF
:10A98800010AA1FB091B12EA0A0A4FEA9B1B00F005
:10A998008A826D4D6D486E4C6E492E78007826700F
:10A9A80008701EB16B490E7886F00106644C0F21C1
:10A9B80084F82410002B00F0E683059D664BB5F85B
:10A9C80026C0B5F824E0059D109318462D8B007815
:10A9D800624B129594F825500995614D0495A3FB97
:10A9E80000535B0803EB4303C31ADBB20F90CDF8A7
:10A9F80034C002F480520C9304F128000BF59673CE
:10AA0800CDF8449097F80080DDF82490DFF860C115
:10AA18000994534C0E91139200210A930896CDF88D
:10AA28001CE0089B002B00F02B83099B079D33F942
:10AA380011201FFA82FEAE454FEA410303D30D9D54
:10AA4800AE4540F262835CF82120934580F0228372
:10AA5800E25EBAF1000F40F0378301314145E2521E
:10AA680000F10600DDDB0E9A099C3E4B84F8242099
:10AA78000F2A49460CBF01220022DDF8449084F8D1
:10AA880025101A7000F08683374B3049314ADFF8B9
:10AA9800E4B008931C46042001230B70137008F0DF
:10AAA800EDF8DBF80030A1686268E3605B1A934256
:10AAB80084BF002384F82130069B3C781E68002C54
:10AAC80001F04D80059A294DB2F824E0178B2449EE
:10AAD80016F48056284640F0998332460EE04378B3
:10AAE80003EB830303EB830303F2EE239BB20132F0
:10AAF800A24221F8023B00F102000ED015F81230F4
:10AB0800002B00F00683022BE9D001320B8821F8D4
:10AB1800023BA24200F10200F0D1109A13780133EF
:10AB28001370FEF7E4BE00BFF8600020B8450020AF
:10AB3800884F030800007A44D34D6210B41F0020E8
:10AB48002C2000205C4C00203C5C0020A019002038
:10AB58006D360020A1190020CD620020ABAAAAAA58
:10AB6800FA710020AE340020203400202864002030
:10AB7800D062002054650020D84CD4F88830A9EB66
:10AB88000303002BFEF6C1AED54AD64B527C05997D
:10AB980033F812308A7DDFEDD46A9FEDD46AC97D1F
:10ABA8009BB207EE102A07EE903AB8EEC77AF8EE95
:10ABB800E77A27EE267A67EE867A0B9AC4F8882019
:10ABC800C7EE876A40F2FF32FCEEE67ACDED077AEF
:10ABD800BDF81C30934228BF134609B1D31A9BB263
:10ABE800C348C44D0178C44C35F81160226825F873
:10ABF8001130921B13440131C04D236001F00F0244
:10AC08001B0902702B80FEF780BE02F0ADFEBC4B24
:10AC1800BC4A1B68C31A93427EF777AEB74B002233
:10AC28001A80FEF772BE059A0499537DD27D013BC6
:10AC380031F913301AB1C3F53B6308331BB2A3F5DE
:10AC48007A7307EE903A9FEDB07AAC4AF8EEE77A5D
:10AC580040F2FF3167EE877AFCEEE77ACDED077AAE
:10AC6800BDF81C308B4228BF0B461380FEF74DBE43
:10AC78001B7AC3F1640307EE903AFFF72EBB4146F7
:10AC8800FFF702BB0221A148F6F76EFB00283FF44C
:10AC980010A82F8018F0020F7FF41DA848F00203B7
:10ACA80043452B803FF417A8994B022214211A70B0
:10ACB8000E20FF2259709A700AF026FAB5F8008023
:10ACC800FFF709B807F0AAFFA8E4924AB2F90030E2
:10ACD800002BB8BF5B42B3F5E17FBFF62EA8B2F9EF
:10ACE8000230002BB8BF5B42B3F5E17FBFF625A861
:10ACF800894B93ED096AD3ED076A93ED057AD3ED95
:10AD0800037A76EE866A77EE877A76EEA66AB7EEEB
:10AD1800007A37EE666A77EEA77AB0EEC66AF0EE8A
:10AD2800E75AB4EEE56AF1EE10FAB4BFB0EE655A30
:10AD3800B0EE465AB5EE405AF1EE10FA40F0AD8347
:10AD48009FED767AB4EEE56AF1EE10FA44BF9FED16
:10AD5800746A36EE477AB7EE006AF4EEC66AF1EE28
:10AD680010FAC8BFDFED6F6AF5EEC07AC8BF36EEDD
:10AD7800C77AF1EE10FA48BFB1EE477AF6EE007ADC
:10AD880027EE677ADFED667A77EE276ABDEEE66A28
:10AD980016EE103A2033402B40F25786DFED626AF8
:10ADA800624ADFED617AC2ED006AFDEEC76AC2ED64
:10ADB800017A16EE903A2033402BC2ED027A49D838
:10ADC800DFED587AB4EEE77AF1EE10FA40F3E8874F
:10ADD8009FED576ADFED576A01E0B0EE677AB4EE8F
:10ADE800E67AF1EE10FA77EE467AF6DC9FED527AC3
:10ADF800F4EEC77AF1EE10FA40F1E0879FED4C6A65
:10AE0800DFED4E6A01E0F0EE477AF4EEE67AF1EE15
:10AE180010FA37EE867AF6D4DFED417AB4EEE77AA7
:10AE2800F1EE10FA40F38186DFED3E7A37EEC77A0D
:10AE380027EE076ADFED425ADFED426ADFED427A1C
:10AE4800E6EE256A67EE065AE6EE267AA5EEA77ABA
:10AE5800F0EE477A3D4BC2ED037A1A6812F40032DD
:10AE680040F054863A4B1046995C0A2902F10C02CC
:10AE780000F0518501301828F6D1FEF75EBF2A8808
:10AE880022F040039BB29A422B803EF44FAF204BF6
:10AE9800022214211A700E20FF2259709A700AF0AB
:10AEA80033F9FEF743BF2B490E787AE594F89430CE
:10AEB800002B3EF485AE079B1B7813F001037EF44C
:10AEC8007FAE012284F8943084F89520FEF778BE8E
:10AED800024C012184F88C10FEF7A3BD2C20002021
:10AEE8009C640020BC6400200000C842000080442C
:10AEF800C35C0020C85C0020C45C00203037002000
:10AF0800001E002060E316006F12833FF8600020E7
:10AF1800F446002080430020941B0020A7DFA834BB
:10AF2800DB0FC93FDB0F494000000000E0000020B4
:10AF3800DB0FC940E4CB1641DB0F49C0E4CB16C197
:10AF480092E741B99730083C15A82ABEB8450020B9
:10AF5800884F03086D360020012900F0038599F811
:10AF6800CC20012303FA0BF30BF1010B1343BBF1C4
:10AF7800040F89F8CC300AF10C0A7FF416ACFEF7FE
:10AF880066BE511D787924F093F900283FF4D5A9BD
:10AF9800B9F1010F40F0FE8607F10D01B87A24F0EF
:10AFA80087F9002840F0F286B549F87B24F080F94B
:10AFB80000283FF4D4A9B9F1030F40F0E386B14962
:10AFC800387D24F075F9002840F0D886AE49787E9F
:10AFD80024F06EF900283FF4D4A9B9F1050F40F028
:10AFE800C986AA49B87F24F063F9002840F0BE86D4
:10AFF800A74997F8230024F05BF900283FF4D4A967
:10B00800B9F1070F40F0AE86A24997F8280024F05E
:10B018004FF9002840F0A2869F4997F82D0024F0A8
:10B0280047F900283EF424AFB9F1090F3EF420AFE8
:10B03800FFF7CEB95D2A00F065855B2A00F06F82C4
:10B048005E2A00F0F885562A00F00586972A00F057
:10B058007586A72A00F0E585904D2B889B0740F060
:10B06800B285A2F1B703072B00F28B82DFE813F059
:10B078007D028902890289027102890265026502DC
:10B08800079B002B3FD05CF8212093454FEA4103F2
:10B09800FFF4DEAC824A824DD25C05EB030E002A37
:10B0A80000F09480022A47D19EF8012002EB820228
:10B0B80002EB820202F2EE2292B2032933DD12B2CF
:10B0C800BAF1000F3FF4C9AC0C9D20F81520B9F176
:10B0D800000F03D10F9D022D7FF6BFACB0F8029090
:10B0E8000288B0F804E04A4496446E4A0FFA8EFE8D
:10B0F80082FB0E526C4DA2EBEE7225F803E012B201
:10B108004FF00109A9E41A464B000A9D4CF821505A
:10B118009FE4D3B2022B04D9032B7FF4F6AC734619
:10B12800E5E43B46E3E4012505FA01FE0E9D25EA28
:10B138000E0512B20E958CE4E25ABEE75B4A12780D
:10B14800002A7FF4F9A9B8F1000F3FF4F5A9012C02
:10B1580040F036819BF82030FFF791B931465448CA
:10B16800F6F702F9002800F0C98084F893600CF023
:10B1780073FDFEF7AEBC43F0400293422A807FF491
:10B1880086AEFEF7D3BD4B4B4B4A109201221A7084
:10B198004A4B04931B214648F6F7E6F800287FF44B
:10B1A80073AC474BDFF820B108931946DBF8003041
:10B1B800CA688B609B1AC82B00F2D584069B1E6850
:10B1C80006F48056A9E45B78FFF768B8CAB2022A89
:10B1D80040F2BC83032AAFD1129A139D079E002D1B
:10B1E80008BF324669E728F0010292B242452A8038
:10B1F8003FF450AD0E2087F8009087F801A087F83B
:10B2080002B009F081FFB5F8008043E500220FE0A5
:10B21800437803EB830303EB830303F2EE239BB230
:10B228000132A24221F8023B00F102003FF475AC62
:10B2380015F812301BB1022BEAD00B88F0E7D3B215
:10B24800032BFAD83B46EBE7B2F5FA7FFEF6B0AC33
:10B2580094F89230002B7EF4ABAC079B1B7801214D
:10B268000B4084F8921000F0BA830CF0C7F8154B25
:10B278000A4D0993FEF79FBC0025FFF7F7B800BFFA
:10B28800BD460020C2460020C7460020CC4600200C
:10B29800D1460020D6460020DB460020D0430020BF
:10B2A80028640020565555559C200020781F002002
:10B2B800F8600020AE340020CD620020FA71002032
:10B2C80020340020D843002054650020B2F5FA7FCE
:10B2D800FEF66EAC94F89230002B7EF469AC079AB7
:10B2E80012780121D70784F8921000F117840CF026
:10B2F800B3FCC24BC24D0993FEF75DBC079BC14A24
:10B308001B781060DB077EF5E8ABBF4B1B78002B82
:10B318003EF44EAC089BDB78002B7EF449AC94F8E5
:10B3280093300133DBB2032B84F893307EF640ACC4
:10B33800B64B5B7813B9002D7EF43AAC0CF05EF88E
:10B34800FEF7C7BBB24AB3491068B4F99020C66982
:10B3580081FB06018911F617701A00F5FF407F304E
:10B3680082423EF7A9AB891B0A4412B2A4F8902086
:10B37800FEF7A2BB089BDB78002B7FF49FAADFEDCA
:10B38800A67AA44938EE678AC9F5FA63FDEEC87A49
:10B398001BB2CDED047ABDF91020120381FB020126
:10B3A800D217C2EBA11203FB02F343F30F334B4452
:10B3B80007EE903AB8EEE78A87ED038AFFF77EBA80
:10B3C800099D002D3EF4ACAAFFF72EB9934A059BC0
:10B3D800D588049A1B8BB2F906105A1B914240F388
:10B3E80088802B449942B4BF00250125FEF7A9BAED
:10B3F800C8398A4242DA99F8CC109A7841FA0BF3A4
:10B40800D9073FF506AA524201200C9209F062FFC3
:10B418007B1E0C9A162B00F28281DFE813F00402DF
:10B428001802EC013D022C025102D701C201AD0104
:10B438009801830180013D0272015102D701C201C6
:10B448005D014901350166021F01DA0023F0EEFEB5
:10B45800032140F6B8328BF82010CBF81C20FFF7F8
:10B4680072B8AB460899DBF80020CB69099D1344F4
:10B478008B61002D3EF454AAFFF7D6B899F8CC306A
:10B48800012202FA0BF223EA020308F5FA7289F89C
:10B49800CC30CAF80820FFF7BCB9B4EEE56AF1EE83
:10B4A80010FA8CBFB0EE654AB0EE464AC4EE054AC3
:10B4B8009FED5B2A9FED5B5ADFED5B1ADFED5B2AA0
:10B4C8009FED5B3ADFED5B3A9FED5B4AA4EE825A53
:10B4D800E4EEE12AA4EE857AA4EEA23AB0EE475A49
:10B4E800B0EE637AA4EE837AA4EE874A84EE057AF6
:10B4F80028E40125FEF725BA00215048F5F734FF66
:10B5080000287FF421AA322384F89600A4F8983002
:10B51800FFF71ABA002A0CBF0120022075E7484B32
:10B52800012202204749484C0B60344B2270344DAD
:10B53800099309F0CFFEFEF73EBB304A424B099211
:10B548001146424A0A6002225A7023F03DFFFEF774
:10B5580032BB2A4A3C4B099211463D4A0A600022F6
:10B568005A7023F031FFFEF726BB244A364B099266
:10B578001146384A0A6001225A7023F025FFFEF767
:10B588001ABB792A00F082847A2A00F076849E2AEF
:10B5980000F06B849D2A00F06084AE2A00F0558488
:10B5A800AD2A00F04A84EF2A00F04484FD2A00F016
:10B5B8003E84FB2A00F02B84FE2A00F07084F72AD0
:10B5C80000F078847B2A00F01B840C4B0993FEF76B
:10B5D800F2BAD9F8D000204B90F836109B78114475
:10B5E8006429A8BF642121EAE17180F83610002B94
:10B5F80040F0998419F0B2F9B1E400BFD8430020B3
:10B60800D0430020C03300206D3600205461002054
:10B61800F43C0020D34D621000007A44905800207A
:10B6280099FB243F69A2163E39094E3DE3B59E3E7B
:10B6380088FA163E45FE7F3FA7DFA834F860002051
:10B648005E3D0020D4430020E4330020083400206D
:10B65800F0330020FC330020303E0020D9F8D00021
:10B66800BC4B90F837109B781144FE29A8BFFE21E7
:10B6780021EAE17180F83710002BBBD0162023F0A7
:10B6880089FED9F8D000B5E7D9F8D000B14B817858
:10B698001144C829A8BFC82121EAE17181709B78AB
:10B6A800002BA7D0142023F075FED9F8D000A1E70D
:10B6B800D9F8D000A74B41781144C829A8BFC821A0
:10B6C80021EAE17141709B78002B93D0132023F07D
:10B6D80061FED9F8D0008DE7D9F8D0009D4B0178EC
:10B6E8001144C829A8BFC82121EAE17101709B78DB
:10B6F800002B3FF47FAF122023F04CFED9F8D00086
:10B7080078E7944B0B989B78417911446429A8BF3A
:10B71800642121EAE1714171002B40F0F383D9F8EB
:10B72800D00067E7D9F8D0008A4B017A9B7811449A
:10B73800C829A8BFC82121EAE1710172002B3FF492
:10B7480059AF0B2023F026FED9F8D00052E7D9F8DC
:10B75800D000804BC1799B781144C829A8BFC82163
:10B7680021EAE171C171002B3FF444AF0A2023F0B4
:10B7780011FED9F8D0003DE7D9F8D000754B817992
:10B788009B781144C829A8BFC82121EAE1718171B9
:10B79800002B3FF42FAF092023F0FCFDD9F8D0008F
:10B7A80028E7D9F8D0006B4B417993F802E01144AF
:10B7B800C829A8BFC82121EAE1714171BEF1000F73
:10B7C80040F08E83112F7FF462AF13E7D9F8D000D1
:10B7D800604B017993F802E01144C829A8BFC82139
:10B7E80021EAE1710171BEF1000F40F09283102F40
:10B7F8007FF461AFFEE60B99564B0F790C93174413
:10B80800642FA8BF642727EAE7770F7123F0DCFDD0
:10B818000C9B9B78002B82D00320394623F0BAFD7D
:10B82800D9F8D000E6E60B984A4B01781144FA297A
:10B83800A8BFFA2121EAE17101709B78002B3FF43F
:10B848006EAF012023F0A6FDD9F8D000D2E60B9800
:10B85800404B817811446429A8BF642121EAE17131
:10B8680081709B78002B3FF45AAF022023F092FDA1
:10B87800D9F8D000BEE60B98364BC1799B781144B5
:10B8880081F30801C171002B3FF449AF052023F073
:10B8980081FDD9F8D000ADE60B982E4B817993F84D
:10B8A80002E011446429A8BF642121EAE171817191
:10B8B800BEF1000F40F01E830D2F7FF423AF2EE75B
:10B8C800D9F8D000234BC17893F802E01144C82975
:10B8D800A8BFC82121EAE171C170BEF1000F40F094
:10B8E80027830F2F7FF4FBAE84E60B98194B417822
:10B8F8001144B1F5967FA8BF4FF4967121EAE17122
:10B9080041709B78002B3FF40AAF152023F042FDCD
:10B91800D9F8D0006EE61049D1F800E04200BEF137
:10B92800000F08D0171803EB87079EF801E07F780F
:10B938007745BEF402AA1044084F094A03EB800376
:10B9480000200B6038801060FEF7F7B9129AFFF7F5
:10B95800B4BB00BF303E0020341F00202020002050
:10B968002420002004999B7831F91220B2F5617FD8
:10B978004FF4966191FBF3F3C0F2E48040F6330193
:10B988009142A8BF11460C2FA1F5617191FBF3F10B
:10B9980000F07781182F7FF4E2AAC9B2C8290B46B4
:10B9A800A8BFC823D9F8D020D77DD8B2B8423FF471
:10B9B800D6AADF1BC44BD07548BF0737FF109B784A
:10B9C8000137FFB23BB9002F3FF4C9AA384609F046
:10B9D80081FCFFF7C4BA182023F0DCFCF3E7BB496D
:10B9E800096811F4003140F04581B94B08465D5CA7
:10B9F8000F2D01F10C0170D001301828F7D1002368
:10BA0800FA3A84F89230B34BA4F89020B24D0993D7
:10BA1800FEF7D1B8B149D1F800E04200BEF1000FFD
:10BA280008D0171803EB87079EF801E07F78774561
:10BA3800BEF408A90244AA4FAA4803EB82030022D5
:10BA48000B603A800260FEF7FDB8B4EEE77AF1EEDB
:10BA580010FA40F3AC81DFEDA45A9FEDA46A01E02F
:10BA6800F0EE676AF4EEC66AF1EE10FA76EEE57A61
:10BA7800F6DCDFED9F6AF4EEE67AF1EE10FA40F1BB
:10BA88009381DFED995A9FED9B6A01E0F0EE667AAB
:10BA9800F4EEC67AF1EE10FA77EEA56AF6D4DFED89
:10BAA800967AF4EEE76AF1EE10FA40F3C880DFED1B
:10BAB800937A77EEE66A66EEA65A9FED915A9FED65
:10BAC800916ADFED917AA5EE856A26EEA55AE5EE34
:10BAD800867AE5EE276AFFF763B980490F68450063
:10BAE80037B12E1803EB86067F787678BE4286D269
:10BAF80005447B4E7B4803EB850300250B603580AE
:10BB080005607CE7814B002201200BE5804B1B7808
:10BB1800032B00F01F810022FFF7A4B97D4A6E4D68
:10BB280013606C4B0993FEF746B8DFED7B7AB4EEF1
:10BB3800E77AF1EE10FA44BFDFED6D7A37EEC77A97
:10BB4800FFF776B90C2F00F0BC80182F7FF407AAF6
:10BB580000210B4626E7714A0592FEF70CBF06F452
:10BB68008056FEF7DABF6E4A069B1E68136823F0FC
:10BB780004031360089A012306F4805682F82130E2
:10BB8800FEF7CBBF38EE678A664B67491870FDEE43
:10BB9800C87AC9F5FA63CDED047ABDF9102012030D
:10BBA80081FB0201D217C2EBA1121BB203FB02F305
:10BBB80043F30F334B4407EE903AF8EEE77AC7EDBC
:10BBC800037AFEF70ABA0023BB2A149300F0BF8059
:10BBD800B72A00F0EF80BE2A00F0E080BD2A7FF48B
:10BBE800D0AC4FF6FE71514A3A48D68909909089EF
:10BBF80033440144D38191811CF094FDF4F722FD74
:10BC08001CF078FD00F0B2FD012009F063FBB4F8E8
:10BC180090300022FA3BA4F8903084F89220FDF787
:10BC2800CABF434A2C4D137843F004031370294BC1
:10BC38000993FDF7C0BF3F4B0222032072E4DFEDFA
:10BC4800367AF4EEE76AF1EE10FA44BFDFED287AAF
:10BC580077EEE66A2FE71CF065FDF4F7F3FC1CF0BD
:10BC680049FD00F083FD012009F034FB94F88E2093
:10BC7800FFF7ECB926490978032900F0A380194693
:10BC8800B3E6CFB22C4B0D915B78BB423FF467A96A
:10BC98000D4B0C93384607F08DFC0C9B0D999B7847
:10BCA8001BB1C9B20C2023F075FB0137FFB28AE63D
:10BCB800174B1B78032B7EF4E8AD09F009FAFDF762
:10BCC800C1BF00273946DDE7303E0020B8450020D7
:10BCD800884F0308D8430020D0430020341F002099
:10BCE8002020002024200020DB0FC940E4CB16418F
:10BCF800DB0F49C0E4CB16C1DB0FC93FDB0F49405E
:10BD080092E741B99730083C15A82ABE103D00209B
:10BD180034370020C0330020DB0FC9BFD8590020BA
:10BD2800CC430020B41F0020D34D621034610020A2
:10BD38007C520020AC3D0020E4330020814B824D32
:10BD48004FF4C8721A80814B0993FDF734BF194626
:10BD5800022348E709F0BCF9FDF7EFBF08231A46AC
:10BD6800FEF738BB07231A46FEF734BB06231A46EC
:10BD7800FEF730BB05231A46FEF72CBB04231A46F0
:10BD8800FEF728BB03231A46FEF724BB02231A46F4
:10BD9800FEF720BB01231A46FEF71CBB022122E74F
:10BDA800F0EE477AFFF722B8F0EE676A77E6F0EE32
:10BDB800667A5EE619464FF6FE7314E7B0EE677AC8
:10BDC800FFF72AB809F084F9B4F9902017E65F4B19
:10BDD80084F8941084F895005B4D0993FEF7A5BD8F
:10BDE800002D3DF4F2AD5A4C94F88D30002B3DF403
:10BDF8001DAE09F06DF9002384F88D30FDF716BEED
:10BE08004FF4FA61022007F0FBFAFFF7DEBB0021CE
:10BE1800022007F0F5FAB4F890304C4A0992963BA4
:10BE28000022A4F8903084F89220FDF7C4BE0021C7
:10BE38000120EEE700210846EBE7FF21002010F083
:10BE4800FFFF94F88E20FFF7AEBB0121002010F011
:10BE5800F7FF94F88E20FFF7A3BB0021FF2010F016
:10BE6800EFFF94F88E20FFF798BB0021012010F017
:10BE7800E7FF94F88E20FFF78DBB364A334B0993C2
:10BE8800137A43F001031372FDF795BE314A2F4B25
:10BE98000993137A23F001031372FDF78CBE002176
:10BEA8000320B6E72A4C0BF0A9FA002384F88D305A
:10BEB800FDF7BCBD00210420ABE7002B93D0264939
:10BEC800264A09684FF47A7000FB031313608AE767
:10BED8000B2009F019F91D4B1B4D0993FDF76BBE9B
:10BEE80011200D930C9223F055FAD9F8D0000D9B30
:10BEF8000C9A67E40D200D930C9223F04BFA0D9BDE
:10BF08000C9AD9E40E2023F045FAD9F8D000FFF7AF
:10BF180071BB10200D930C9223F03CFAD9F8D00095
:10BF28000D9B0C9A63E4172023F034FAFFF7F7BB54
:10BF38000F200D930C9223F02DFAD9F8D0000D9B09
:10BF48000C9ACEE4EE650020D0430020D8430020B0
:10BF58002C2000209434002054650020BC3300209D
:10BF680038B50B4C23688BB15A68821A002A0546EB
:10BF780004DA0CE05A68AA1A002A07DB9A682260D9
:10BF880018461A6890472368002BF3D138BD38BD8E
:10BF98005C5D00200B4B002210B4027203F1B40464
:10BFA800042102E0072A09DC9979890702D5197961
:10BFB800815401329C4203F11403F3D15DF8044B20
:10BFC800704700BF7459030810B40D4C0423214670
:10BFD800002200E08B7913F0010301F1140106D16E
:10BFE80001320A2AF6D103705DF8044B704702EB60
:10BFF800820204EB82025DF8044B137903707047E8
:10C008007459030810B40123022415212222047252
:10C018004170C270037083705DF8044B704700BFB5
:10C028002C22022302704370704700BF2DE9F047AD
:10C038008C4B1B78DB07074644D58B4B8B4D1C7804
:10C048008B4E012C59D01CD3022C07D189498A4A1E
:10C0580009881288914201D901241C70EB7AE3B156
:10C068002B89D3B1854B1B78BBB107F0C5FA0028E3
:10C0780000F09B802B7B83422CBF01210021317073
:10C088000CE07C497E4A098810886A7B801A8842BD
:10C09800E2DAEB7A0024002BE2D131782A79632A9C
:10C0A80006D8022C774E00F0BA803378002B5DD189
:10C0B800754AAB7A8C4238BF0C461470002B4CD1B1
:10C0C800BDE8F0876B4B694D19885B88E878CB1A17
:10C0D80083EAE3728142A2EBE3721DD32B788B4291
:10C0E8001AD3614B1C78E01E012861D96749097889
:10C0F80002294FD0012C5E4EA5D15F4A5D491288B6
:10C10800687B0988121A914239DD5D4A12888A4291
:10C11800A4D200241C70A1E7B1EB400FE1DC524B24
:10C128001C78E11E012940F29480022ADEDC57497E
:10C138004F4E0878DFF84481DFF844C1DFF838E172
:10C1480000210324022834701C7088F80010ACF811
:10C158000010AEF8001081D11FE0012C71D0022C24
:10C168000BD10720BDE8F04708F0CEBF7068381A39
:10C17800474B984258DD72709AE7BDE8F087022471
:10C188001C706BE7022AD2DD4049097802294FF07A
:10C19800040464D13949364E09783E48022ACCBF96
:10C1A80000220122C28081804BE70221317075E7AD
:10C1B800022A9BDC95F800C091FBFCFC0CF1010CF9
:10C1C800BCF1080FDFF8B4A0304EA87895F801E06C
:10C1D80096F800802A4CDFF8A090254EA8BF4FF0B3
:10C1E800080C8AF800C01FFA8CFA10FB0AF01EFB34
:10C1F8000AFE80B2DFF88CA02080A9F800E00024B5
:10C208004FF0640EB8F1020F34701C70CAF8044085
:10C218008AF801E07FF439AF0FFA8CF1BDE7307886
:10C22800A0B9012377603370C2F164021A4B00FB96
:10C2380002F083FB0023C017A0EBA350643070709A
:10C2480036E70820BDE8F04708F05EBF7368F81AC3
:10C258008EE7032C96D10D49097802299AD0044E0D
:10C26800FCE600BF03400020E424002060430020D7
:10C27800F424002088410020E82400209E4100206A
:10C28800E6240020EC2400203437002088400020D9
:10C298007F9698008C4000206BCA5F6B2DE9F047B1
:10C2A8000569C3681D4028D00F4606464FF0004870
:10C2B8004FF00009B5FA85F328FA03F2D2431B3B85
:10C2C80032611540042B16D8DFE803F03129211913
:10C2D80003007B6A002B32D003F1FF3A1FFA8AFA77
:10C2E800C7F824903C6A34B12368204651469847E1
:10C2F8006468002CF8D1002DDCD1BDE8F0873868DF
:10C30800716B036889B29847002DD3D1F5E7786837
:10C31800B16B036889B29847002DCBD1EDE7B868B7
:10C32800F16B036889B29847002DC3D1E5E7F86837
:10C33800316C036889B29847002DBBD1DDE7F36AF9
:10C348001FFA83FACEE700BF08B50121022005F0E5
:10C35800A1F9094B1B7803F00503052B08D0002130
:10C36800012005F097F90021084605F093F9FEE74A
:10C3780018F038FDF3E700BFA42C0020022828BFDE
:10C38800022010B4084C094B207000EB8002C0EB6F
:10C39800C20207495DF8044B013003EB4203C0B207
:10C3A8000B6008F097BF00BFE4330020103D002069
:10C3B800D443002008B51CF0B5F9F4F743F9BDE8FB
:10C3C80008401CF097B900BF2DE9F04F013085B047
:10C3D800C3B203938E4D8F4F8F4C904E0A23029316
:10C3E8003220DFF8409219F0D7F84FF4FA7A4FF07C
:10C3F800100C4FF47A70D9F80430C3F30803002BFB
:10C4080040F0C880EFF31183002B40F0C380296807
:10C41800A26800BF2B689942F9D1D7F800E000FB69
:10C428000EF39B1AB3FBFEF300FB01314FF0010E34
:10C438000191D9F80430C3F30803002B40F08E8033
:10C44800EFF31183002B40F089802B68A16800BFAF
:10C458002A689342F9D1D7F800B000FB0BF2521AC0
:10C46800B2FBFBF200FB0323019A9B1AB3F57A7F18
:10C47800DFD3BAF1010ABED1039B002B40F0C48080
:10C488004FF47A7ADFF89C9150464FF0100CD9F8A7
:10C498000430C3F30803002B40F09980EFF31183B5
:10C4A800002B40F094802968A26800BF2B6899424D
:10C4B800F9D1D7F800E000FB0EF39B1AB3FBFEF3AB
:10C4C80000FB01314FF0010E0191D9F80430C3F39C
:10C4D80008033BBBEFF3118323BB2B68A16800BFA4
:10C4E8002A689342F9D1D7F800B000FB0BF2521A30
:10C4F800B2FBFBF200FB0323019A9B1AB3F57A7F88
:10C50800E3D3BAF1010AC2D1029B013B02937FF443
:10C5180067AF4349434B4448444A0860DA6005B072
:10C52800BDE8F08FEFF311888CF31288A1682368B7
:10C53800DB0344BFC6F800E0A1682B6832685FFAE5
:10C5480088F888F31188D7F800801A4400FB08F3AC
:10C558005B1AB3FBF8F300FB0233CDE7EFF3118866
:10C568008CF31288A1682368DB0344BFC6F800E097
:10C57800A1682B6832685FFA88F888F31188D7F8C1
:10C5880000801A4400FB08F35B1AB3FBF8F300FBC6
:10C59800023369E7EFF311828CF31288D4F808E0CC
:10C5A8002368D90303D501233360D4F808E02B6846
:10C5B8003168D2B282F311883A68194400FB02F359
:10C5C800A3EB0E03B3FBF2F300FB01312EE7EFF30D
:10C5D80011828CF31288D4F808E02368D90303D5B4
:10C5E80001233360D4F808E02B683168D2B282F3B3
:10C5F80011883A68194400FB02F3A3EB0E03B3FB5E
:10C60800F2F300FB01315DE7184621F0FFFE37E742
:10C61800546500205865002010E000E050650020B7
:10C62800FC9F002000ED00E0EFBEADDE0400FA053F
:10C6380038B5434B5A899989914224BF00225A81BF
:10C64800198ADA89914224BF0022DA81DA788AB31A
:10C65800072A2FD03B493C4D91F853000124002173
:10C668000A282C709C70D9713DD00C2865D0DFED5C
:10C67800377A8ABB364C9FED370AA278002918BF53
:10C68800F0EE407A062A04D8334901EB820191ED95
:10C69800000A217959B3013A032A4DD8F7EE007AF6
:10C6A80087EE800A25F060FC2388984228BF184648
:10C6B800208038BDD97921B198780428B8BF0420E2
:10C6C8009870204890F853000A280CD00C28CED136
:10C6D800DFED227A002ACDD0072ACBD00A282CD128
:10C6E800DFED1F7AC6E70A20DFED1E7AC1E79B78E7
:10C6F800154A07EE103A1178B8EEC77A27EE277A6E
:10C7080007EE901AF8EEE77A67EE877AB4EEE70A52
:10C71800F1EE10FA10DDC0EE077AFDEEE77A17EEBB
:10C72800903A102BA8BF1023012BB8BF0123DBB20E
:10C738008B4238BF0B46137038BDDFED0B7A99E793
:10C74800C0490020D4490020286100206F12033915
:10C758005C4E00206F120338FC3603080AD7A33951
:10C768000F506E3A5304E9386F12833A2DE9F047B7
:10C77800A84FA94E1BF0D6FFBE421ED2DFF8148385
:10C78800DFF814934446258862197DB14A450DD2D5
:10C79800052D0BD933886188C3F30B03994200F048
:10C7A800DE80144625886219002DEFD17168304665
:10C7B800143605F0FCF9BE42E4D3984A1378A3F185
:10C7C800170102290FD9964911F83300002840F0C3
:10C7D800F280D8000144497829B1924911F83330E0
:10C7E800002B00F01081904B5A78022A40F2DD802D
:10C7F80000228E495A701A788D48022A016000F288
:10C80800D08002EB82018B4BC2EBC10203EB4203E7
:10C81800998C5A8C884C9142236001D300225A8407
:10C82800864B9A78042A00F0E58032B91A88B2F566
:10C83800F07F84BF4FF4F0721A80814DFFF7F8FE45
:10C848002B68804A1A40002A00F0E080D80700F1DF
:10C85800CC80590400F1C4801A0700F1BC809B0405
:10C8680000F1B2801AF00AF810B9774807F034FDE1
:10C87800802005F0D3F94FF4007005F0CFF94FF49C
:10C88800802005F0CBF94FF4001005F0C7F94FF000
:10C89800007005F0C3F94FF0806005F0BFF922F091
:10C8A80093FD00213022694826F01BFB206817F011
:10C8B800FDFE674B276803F1500102E004339942FB
:10C8C8006DD01A78002AF9D19C78D8788442F5D2AC
:10C8D8006049614B0D79614961480A70614E624C4B
:10C8E8000460C822642111FB0521002259609A6066
:10C8F800DA601A615A619A61DA6183F8202083F854
:10C908002120376016F094FE584B9FED595A1B882A
:10C91800584A9FED596A5079584906EE903AF8EE10
:10C92800E66A1388C5EE265A07EE103A538812793C
:10C93800C1ED005A07EE903AB8EEC77A504BF8EEC0
:10C94800E77A18725A7227EE067A67EE867ABDE899
:10C95800F04783ED017AC3ED007A1BF0CBBE637913
:10C968009B077FF41EAF716894F804A0304605F069
:10C978001EF93388BAEB133F04D01436BE42FFF4D5
:10C9880001AF1AE773887068AA1FC3F30B039A42B2
:10C9980004F10601A8BF1A4625F0A6F9EDE7012221
:10C9A80096E700221A70234B32E7204902EB420235
:10C9B80001EB82011FE7D8000C186468002C7FF493
:10C9C80009AF1724147005E72E4805F027F9402011
:10C9D80005F024F946E72C4805F020F92B683EE7D6
:10C9E8002A4805F01BF92B6836E7294805F016F99F
:10C9F8002B682EE79A8AB2F57A7FBFF41EAF4FF400
:10CA08007A729A8219E718231370ECE643F40053FC
:10CA18002B601BE7D0910308708D0308705200202B
:10CA28003C5A03086C560308E4330020F033002016
:10CA3800D8430020103D0020D44300205C4E002045
:10CA4800443E002009600002045A0020C82000204B
:10CA580018630020CC65002020340020CC1B002067
:10CA68000C210020FC2000203A610020B81F002083
:10CA7800C0C9FB48EC1D002017B7D138BC1F0020E7
:10CA8800B065002009400002016000020920000290
:10CA98000860000202F003080000040808B51BF053
:10CAA80041FEF3F7CFFD1BF025FEFFF75FFE0120E7
:10CAB800BDE8084008F00EBC2DE9F047B54C82B03F
:10CAC800636820469847002800F0BF80B24B1B7867
:10CAD8000122042B84F83C2000F0BA80B4F9161027
:10CAE800B4F91820B4F91A3021636263A363AB4B1D
:10CAF8001B88002B69D0AA4DD4ED0C7AD5ED004ADD
:10CB080095ED050A95ED015A95ED067AD5ED035A8E
:10CB180095ED026AF8EEE76AD5ED047AA4EEA60A66
:10CB2800A5EE267A67EEC07AA5EEC07AE6EE267AFA
:10CB380085ED057AC5ED067A25F016FAD4ED0D6A6D
:10CB4800D5ED094A95ED0E0A95ED0A5A95ED0F7A3D
:10CB5800D5ED0D7AD5ED0C5A95ED0B6A2063F8EEFC
:10CB6800E66AA4EEA60AA5EE267A67EEC07AA5EED6
:10CB7800C07AE6EE267A85ED0E7AC5ED0F7A25F0B5
:10CB8800F3F9D4ED0E6AD5ED124A95ED170A95ED35
:10CB9800135A95ED187AD5ED167AD5ED155A95ED07
:10CBA800146A6063F8EEE66AA6EEA40AA6EE857A31
:10CBB80067EEC07AA0EE657AE6EE867A85ED177A9A
:10CBC800C5ED187A25F0D0F9A063764FA17F764895
:10CBD80016F0B0FC3B88002B7CD1744E3568744B42
:10CBE8001B685B0742D4B5F90070216B636BA06BBF
:10CBF800704A714E92ED026AD2ED006AD2ED015A86
:10CC0800C91B2163B5F90270DB1B6363B5F90470B6
:10CC18003568C01B07EE900AB8EEE75A07EE901A7F
:10CC2800B8EEE77A07EE903AF8EEE77A36EE056A5C
:10CC380036EE877A77EEA57A0135A06382ED026A2F
:10CC480082ED007AC2ED017A356002B0BDE8F08766
:10CC58005A4BB4F91600B4F91810B4F91A20188010
:10CC68002063598061639A80A26340E7544F3B88F0
:10CC7800322B7ED0002B5BD152480378002BB2D0E8
:10CC8800DFF848E1F169326A8EFB01730027C917A2
:10CC98000770C1EB23118EFB0203D217C2EB2312DC
:10CCA800736A29806A80A08A47498EFB03E2DB17F2
:10CCB800C3EB22131B1AAB80CF601BF033FDF3F7D5
:10CCC800C1FC1BF017FDFFF751FD012008F002FB26
:10CCD800356888E7354E226B3568B3F5C87F4FF065
:10CCE800000323632B80398818BF7068B7F8008069
:10CCF80008BF0020B1F5C87F18BFB368616B024454
:10CD08000B440020B8F5C87F60637260B360688028
:10CD18003AD0D4F838E0F168A0637144B8F1010F53
:10CD2800A880F16054D008F1FF38A7F8008056E7D2
:10CD3800F169226B002323632B80B7F800E00A44D3
:10CD4800BEF1320F616B63636B80F261A26B6BD0D3
:10CD5800706A0190306AA363014401983162024409
:10CD6800BEF1010FAB80726263D00EF1FF333B80DE
:10CD780082E7154B2988D8686A88AB883182B06108
:10CD88007282B3820021D4E7A36BF360A063A8800A
:10CD9800C9E700BF8843002088400020B85500201C
:10CDA800BC550020EE650020B84300200C2100206F
:10CDB8005C4C0020A4650020A06500208C40002069
:10CDC800C4200020C1200020346100201F85EB51C1
:10CDD800DFF80CC1DFF8F8E0C8328CFB02A9C833D1
:10CDE800D217C2EBE9128CFB03A9DB17C3EBE913DB
:10CDF800C8316B802A808CFB013CA28ACB17C3EB1D
:10CE0800EC139B1AAB80CEF80C001BF08BFCF3F7ED
:10CE180019FC1BF06FFCFFF7A9FC404608F05AFA12
:10CE2800B7F8008035687EE7A36331627262AB8031
:10CE38009BE7234A234812682349037012F40032FF
:10CE480081F800E032D113462049C85C0B2803F171
:10CE58000C030ED00132182AF7D1338A2B80728A3C
:10CE68001B4B6A80B18AB269A980B7F800E0DA6022
:10CE78007BE71848D0F800C05300BCF1000F09D078
:10CE880003EB020E01EB8E0E9CF801C09EF801E048
:10CE9800E645E2D21344DFF84CE00F4A01EB830188
:10CEA80000230160AEF800301360D6E70B4A127811
:10CEB800032A01D01A46C7E708F00AF93568CCE713
:10CEC800B8450020C6200020C0200020884F030855
:10CED80034610020341F0020242000203437002033
:10CEE8001F85EB5120200020F8B50F4C0F4DAC42A8
:10CEF80006D261682046143404F059FEAC42F8D3D7
:10CF08000B4A0C4B0C4C0D4D0D4E156001250022A3
:10CF180004270C4925701A705A700B48B770BDE881
:10CF2800F84008600CF09CB8708D0308D091030895
:10CF3800D4430020E433002028610020103D002065
:10CF4800C0490020D8430020F033002008B5FFF77F
:10CF5800CBFF1BF0E7FBF3F775FBBDE808401BF0C0
:10CF6800C9BB00BFF0B50C292BD8DFE801F06F2A48
:10CF78002A2A4C2A2A2A2B2A2A2A0700046AB2F8C3
:10CF88000CE097881668674D24F480540462036A9D
:10CF98004468C16923F4005343EA0E3321F4E6419F
:10CFA800A84243EA073341EA062100F0B58005F5B7
:10CFB8000065A84200F0B08092684460C1610264D4
:10CFC8000362F0BD046A96899588D2F800E0554F4F
:10CFD80024F480740462036A4468C16923F400730A
:10CFE80043EA062321F07301B84243EA052341EAE4
:10CFF8000E017ED04C4DA8427BD092684460C1613E
:10D00800C2630362F0BD046A96899588D2F800E08D
:10D01800444F24F010040462036A4468816923F0D1
:10D02800200321F0807143EA061321F4E641B84257
:10D0380043EA051341EA0E2148D03B4DA84245D0AA
:10D0480092684460816182630362F0BD046A9389D7
:10D05800B2F804E01768334E24F001040462056A4C
:10D068004468816943EA0E0321F4803125F0020502
:10D078009BB221F07301B04243EA050341EA07017C
:10D0880014D0294DA84211D005F54065A8420DD00D
:10D0980005F58065A84209D005F58065A84205D048
:10D0A80092684460816142630362F0BDD689158A43
:10D0B800578A23F0080333433D43D68824F4407449
:10D0C80023F00403ADB233432C43E9E7D589178A2B
:10D0D800D68823F0800343EA051324F44064558A74
:10D0E80023F0400344EA870443EA061344EA85042C
:10D0F800A6E7D589178AD68823F4006343EA05236F
:10D1080024F44054558A23F4806344EA071443EA1C
:10D11800062344EA051470E7158A24F4804444EA97
:10D12800851449E7002C0140003401402DE9F04FF7
:10D13800C822002183B07848784CDFF80492784DF3
:10D14800784E794FDFF8FC8125F0CBFE7748784997
:10D15800DFF8F4E1DFF8F4C100221359834200F04C
:10D16800C180B3F1804F00F0C980AB4200F0C880A5
:10D17800B34200F0C780BB4200F0C680734500F0A0
:10D18800C580634500F0C480434500F0C380DFF8E4
:10D19800C0A153457ED00AF5806A534508BF0923CC
:10D1A80079D01432C82AD8D15C4C624D624E604F97
:10D1B80004F1C80802E01434A04568D0A379002B14
:10D1C800F9D023794FEA131909F1FF39B9F1020FA0
:10D1D80003F00F03EFD835F8190040FA03F2D2072D
:10D1E800E9D54FF0010A0AFA03F3013B184024F08D
:10D1F80007FB16F809305149184411EBC002DAD080
:10D2080051F83000DFF84CE1217A00F138439B0AED
:10D218001EF8033003F01F0E5B09022B0AFA0EFA00
:10D2280062D0032B65D0012B03D17B694AEA030343
:10D238007B6193880093B3FA83F3C3F11F039BB216
:10D24800DA0800EB820203F00703D2F820E09B0023
:10D258004FF00F0C0CFA03FC2EEA0C0EC2F820E07B
:10D26800D2F820E001FA03F343EA0E031362694699
:10D278000023022214348DF804208DF805308DF82F
:10D2880006308DF807300FF035FBA04596D103B076
:10D29800BDE8F08F082309EBC3034FF0010B93F8A7
:10D2A80020A00AF01F034FEA5A1ABAF1020F0BFA2C
:10D2B80003F30BD0BAF1030F0ED0DA457FF471AF48
:10D2C800D1F814A043EA0A034B616AE7D1F818A021
:10D2D80043EA0A038B6164E7D1F81CA043EA0A0316
:10D2E800CB615EE70023D6E7BB694AEA0303BB616B
:10D2F8009FE7FB694AEA0303FB619AE70123CAE750
:10D308000223C8E70323C6E70423C4E70523C2E7CB
:10D318000623C0E70723BEE7105900207459030805
:10D32800000400400008004000100040002C0140AC
:10D3380000100240945403089C540308A848002095
:10D34800FC3603080040014000140040003401404E
:10D35800004401406C59030801490248FEF79EBF8A
:10D36800B05900200048014001490248FEF796BF25
:10D37800885900200040014001490248FEF78EBF4D
:10D38800605900200004004002494FF08040FEF739
:10D3980085BF00BF3859002001490248FEF77EBF0B
:10D3A80010590020002C014001490248FEF776BFC1
:10D3B80010590020002C01402DE9F04104684A4D25
:10D3C800A30AAB4272D009D8B3F5801F6AD04A3D90
:10D3D800AB425AD14FF0700E022608E0434DAB42E3
:10D3E80068D00235AB4252D14FF0C00E04264779BF
:10D3F8004FEA970C002961D0B000634685190227CF
:10D40800D4F80C809F400CEB4503BFB2384D03F1B4
:10D41800040C47EA080745F8231045F82C20E76074
:10D42800EFF31181502282F31288821905EBC202B0
:10D43800136973B313620433821905EBC202576987
:10D4480017B11F6053690433821905EBC20297694B
:10D4580017B11F6093690433821905EBC202D769BB
:10D4680017B11F60D36904330027CAB21F6082F363
:10D478001188304405EBC000036A6BB9E3684FF6C6
:10D48800FE721340E360BDE8F081BDE8F081BDE8BD
:10D49800F08105EB0E03CFE7E36843F00103E36097
:10D4A800BDE8F0814FF0480E0126A0E74FF0200EAE
:10D4B80000269CE74FF0980E032698E7BF08022342
:10D4C80006FA03F0BB40DB43E768094D9BB23B40DB
:10D4D80087190CEB470CE3600CF1040345F82C109A
:10D4E80045F823209CE700BF4B00100050001000B7
:10D4F8001059002030B503685C4D18885C4CB4FBAB
:10D50800F2F20139013AAB4294B283B089B282B2E5
:10D5180066D05848834263D0B3F1804F60D0A0F5FD
:10D52800983083425CD000F58060834258D05248DE
:10D5380083425BD000F5806083427DD022F4407244
:10D5480000F58C3092B283421A80D9621C850ED0C5
:10D55800484A93420BD002F54062934207D002F545
:10D568008062934203D002F58062934201D1002287
:10D578001A8601225A611A883C4992B242F0010285
:10D588008B421A8062D0B3F1804F61D03B4A9342FC
:10D5980060D002F5806293425ED002F50062934249
:10D5A8005CD002F5806293425AD002F590329342E1
:10D5B80058D002F54062934256D002F580629342F9
:10D5C8001ED002F58062934208BF092219D002A832
:10D5D8004FF0012340F8043D0FF056F903B030BD79
:10D5E800254822F07002834292B2A3D101201A800A
:10D5F800D9621C8558611A8892B202431A80C5E71D
:10D6080008221F4B03EBC20301A893F821408DF8B1
:10D618000440012300228DF805308DF807308DF87D
:10D6280006200FF031F91B2CD8D1164B019301A815
:10D638000FF02AF903B030BD01201A80D9621C8589
:10D6480058611A8892B202431A809CE70022D8E7F0
:10D658000122D6E70222D4E70322D2E70422D0E748
:10D668000522CEE70622CCE70722CAE7002C0140B4
:10D6780000A24A04003401400010004000040040A9
:10D68800FC36030819010001204B98422DD0B0F157
:10D69800804F2CD0A3F5943398422AD003F58063A9
:10D6A800984228D003F50063984226D003F580639A
:10D6B800984224D003F59033984222D003F5406372
:10D6C800984220D003F58063984207D003F5806321
:10D6D800984208BF092202D00020704708220C4B4C
:10D6E80003EBC20393F8200070470022F7E70122FA
:10D6F800F5E70222F3E70322F1E70422EFE7052228
:10D70800EDE70622EBE70722E9E700BF002C01401E
:10D71800FC3603082DE9F04F013085B0C3B20393FE
:10D728000B4602918B4C8C4E002B00F09A803220D5
:10D738008A4D8B4FDFF82C9217F02EFF4FF4FA7AB0
:10D748004FF0100C4FF47A70D9F80430C3F3080383
:10D75800002B40F0DE80EFF31183002B40F0D980DE
:10D768002968A26800BF2B689942F9D1D7F800E070
:10D7780000FB0EF39B1AB3FBFEF300FB01314FF0E5
:10D78800010E0191D9F80430C3F30803002B40F0CF
:10D798008780EFF31183002B40F082802B68A1680B
:10D7A80000BF2A689342F9D1D7F800B000FB0BF20A
:10D7B800521AB2FBFBF200FB0323019A9B1AB3F542
:10D7C8007A7FDFD3BAF1010ABED1039B002B40F068
:10D7D800BD804FF47A7ADFF88C9150464FF0100CE8
:10D7E800D9F80430C3F30803002B75D1EFF3118384
:10D7F800002B71D12968A26800BF2B689942F9D122
:10D80800D7F800E000FB0EF39B1AB3FBFEF300FB16
:10D8180001314FF0010E0191D9F80430C3F3080328
:10D8280013BBEFF31183FBB92B68A16800BF2A680B
:10D838009342F9D1D7F800B000FB0BF2521AB2FBB1
:10D84800FBF200FB0323019A9B1AB3F57A7FE3D31B
:10D85800BAF1010AC4D1029B013B0293002B7FF469
:10D8680066AF05B0BDE8F08FEFF311888CF312882E
:10D87800A1682368DB0344BFC6F800E0A1682B68F1
:10D8880032685FFA88F888F31188D7F800801A445C
:10D8980000FB08F35B1AB3FBF8F300FB0233D2E793
:10D8A800EFF311888CF31288A1682368DB0344BF67
:10D8B800C6F800E0A1682B6832685FFA88F888F338
:10D8C8001188D7F800801A4400FB08F35B1AB3FBF1
:10D8D800F8F300FB023370E7EFF311828CF3128840
:10D8E800D4F808E02368D90303D501233360D4F8BA
:10D8F80008E02B683168D2B282F311883A6819447B
:10D9080000FB02F3A3EB0E03B3FBF2F300FB0131C0
:10D918007FE7EFF311828CF31288D4F808E02368CC
:10D92800D90303D501233360D4F808E02B683168A4
:10D93800D2B282F311883A68194400FB02F3A3EBD0
:10D948000E03B3FBF2F300FB013118E7184620F091
:10D958005DFD3EE710E000E05065002054650020C2
:10D968005865002000ED00E0204B5B68C3F3080316
:10D9780030B4BBB9EFF31183A3B91D4B1D4C186824
:10D98800A16800BF1A689042F9D11B4B1C684FF47C
:10D998007A7202FB04F3591AB1FBF4F130BC02FBB2
:10D9A80000107047EFF31182102383F31288114996
:10D9B8008C680B6813F4803F104B02D0012018606C
:10D9C8008C680B49D2B20D68186882F311880A4B2B
:10D9D80019684FF47A72284402FB01F31B1B30BC10
:10D9E800B3FBF1F302FB0030704700BF00ED00E02D
:10D9F8005465002010E000E05865002050650020C4
:10DA08002DE9F84F8046FFF7AFFF254E2549DFF88F
:10DA1800A0E0254A254D844610274FF47A7401204A
:10DA2800DEF80430C3F30803D3B9EFF31183BBB9AD
:10DA38000B68D2F808A000BFD1F800904B45F7D189
:10DA4800D6F800B004FB0BF9A9EB0A09B9FBFBF9FE
:10DA580004FB0393A3EB0C034345E1D3BDE8F88F24
:10DA6800EFF3118A87F31288D2F808B01368DB0342
:10DA780044BF2860D2F808B00B68D5F800905FFA68
:10DA88008AFA8AF31188D6F800A0994404FB0AF3AD
:10DA9800A3EB0B03B3FBFAF304FB0933DAE700BF8C
:10DAA800586500205465002010E000E05065002013
:10DAB80000ED00E02DE9F04FDFF830C1474A484952
:10DAC800484E494D8046102718F1FF38C0F0848031
:10DAD800DCF80430C3F30803002B5CD1EFF31183A7
:10DAE800002B58D10B68946800BF08688342F9D1AD
:10DAF800D6F800904FF47A7000FB09FEAEEB040EE6
:10DB0800BEFBF9FE00FB03EEDCF80430C3F30803A8
:10DB18004FF47A740120FBB9EFF31183E3B90B6872
:10DB2800D2F808A000BFD1F800904B45F7D1D6F83D
:10DB380000B004FB0BF9A9EB0A09B9FBFBF904FBDC
:10DB48000393A3EB0E03B3F57A7FBDD2DCF8043060
:10DB5800C3F30803002BDFD0EFF3118A87F3128891
:10DB6800D2F808B01368DB0344BF2860D2F808B0C5
:10DB78000B68D5F800905FFA8AFA8AF31188D6F80C
:10DB880000A0994404FB0AF3A3EB0B03B3FBFAF3DD
:10DB980004FB0933D5E7EFF3118487F31288D2F831
:10DBA80008901368D80303D501232B60D2F8089096
:10DBB8000B682868E4B284F31188D6F800A04FF403
:10DBC8007A7400EB030E04FB0AF3A3EB0903B3FB1F
:10DBD800FAF304FB0E3E97E7BDE8F08F10E000E093
:10DBE80054650020586500205065002000ED00E0D5
:10DBF80030B4EFF31183102282F312880649074CE0
:10DC08000A680748013200250A602560DBB202680D
:10DC180083F3118830BC704754650020506500209C
:10DC280010E000E02DE9F04FC04B1E788BB0002EBD
:10DC380040F0BC80BE4BBF4C1D78DFF818A3DFF85E
:10DC48001893DFF8188305F00105A4F10A0B54F8BE
:10DC58000A3CBBB1CC2707FB06B7184602F0D6FC36
:10DC680080B154F80A0C02F0C9FC14F8023C8BB9D4
:10DC7800242831D0F5B154F80A3C184602F0C6FC05
:10DC88000028EED10136032E04F1CC04DFD10BB00D
:10DC9800BDE8F08F012B23D0022B2BD0032B37D0DC
:10DCA800042B67D0052B40D0062B4FD054F80A2CF4
:10DCB8001346D2E754F80A3C23281A4600F0898113
:10DCC8009D4991F832108142C7D19C4BCAF8009007
:10DCD800C3F80C801346C0E7012304F8023CCAE7E6
:10DCE8004D2854F80A2C0CBF0223002304F8023CE8
:10DCF8001346B2E700233C2804F8023C45D03E28EE
:10DD0800D4D10122032304F8012C04F8023CB2E721
:10DD1800C02814D80022042304F8050C04F8040CC5
:10DD280004F8062C04F8023CA5E714F8063C14F89D
:10DD3800052C9A422FD814F8043C834203D00023C0
:10DD480004F8023C97E7062304F8023C14F801ECB7
:10DD5800BEF1000F00F08281BEF1010F00F0C68114
:10DD680001360023032E04F8023C04F1CC047FF4AE
:10DD78006EAF8CE714F8043C04F8030C58400523F4
:10DD880004F8040C04F8023C75E7032204F8013C8B
:10DD980004F8022C6FE714F8042CF91842400133F8
:10DDA80004F8042C04F8063C887264E7644B18688D
:10DDB80000283FF46CAF03F031FEDFF8A4A1614DF9
:10DDC800DFF8A091DAF8000002F020FC00283FF408
:10DDD8005EAFDAF8000002F011FC09281BD03F28DA
:10DDE80019D02B68002B67D1042800F0A9810C28D2
:10DDF80000F0E8807F28E5D0A0F12002D2B25E2AA8
:10DE0800E0D80BB92028DDD05A1C09F803002A6095
:10DE18001BF06EF8D6E72C68002C5BD14A4FA3465E
:10DE280007F59878BBF1000F08BFBB460837474590
:10DE3800F8D1BBF1000F00F07881083FDBF8000053
:10DE48003A68065D135D9E42204402EB040140F0EF
:10DE58006A81661E4E4422460BB9FD2A5DD906F832
:10DE6800013F01322A6010F8013F11F801EF9E4589
:10DE7800F2D00AB15F4512D034481BF041F85F4533
:10DE880008D35BF8080B1BF03BF809201BF030F8AF
:10DE9800BB45F6D92E481BF033F82A680024944273
:10DEA80090D2661E4E4416F8010F1BF021F82B681D
:10DEB80001349C42F7D385E70C2800F083800A28B8
:10DEC80052D00D2850D07F2800F0FD80FF2B3FF660
:10DED80079AF91E71C4E002706F59878BB4602E01B
:10DEE800083646450DD0224631684846F2F7A8FE66
:10DEF8000028F5D1B346002FF2D1374608364645FB
:10DF0800F1D13B465F469B46002B97D1002F3FF44B
:10DF180059AF0E481AF0F4FFB3E7511C202009F856
:10DF28000200296009F801300A46A3E7C933002036
:10DF3800034000200E6F0020045A002000ED00E08E
:10DF4800AC320020B4330020F84B0308A05E03086D
:10DF5800A85E0308FC9F0020EFBEADDE0400FA05B2
:10DF6800B0320020B43200201BF04BF823217C484B
:10DF780024F0CEFF002800F0E180A0EB0900286023
:10DF880088B1431E19F80310202940F0E78009EBF7
:10DF9800030204E012F8011D202948D10346581E47
:10DFA800002BF7D12B604FF480720021484624F0F3
:10DFB80098FF6C4B1B78002B3FF469AE6A481AF047
:10DFC8009FFFFFE669481AF09BFF67481AF098FF21
:10DFD800F8E667496748C978674ADFF8CCE1936291
:10DFE800003118BF012101706449D16240211363D7
:10DFF80082F8341082F83550614962480B602C323F
:10E00800CEF80020574A012313701BF0DBFC56485A
:10E018001AF076FF4FF4006004F030FE5A4B93F884
:10E028003230232B00F0928014F8023C3CE62B603F
:10E03800564C002204F5987809F8032002E00834C9
:10E04800444577D02168484608F0A0FC0028F6D05F
:10E0580044456FD2636898470023A3E74C4BADF85B
:10E0680022E00FCB0DF1280C02AF87E80F004CF827
:10E0780024ED14F8051C14F8033C069404EB010E77
:10E08800624639464FF0010C06A8CDF81CE0ADF801
:10E0980020308DF824C0F4F735FFE8B9019F00233C
:10E0A80004F8023C002F3FF4EDAD54F80A0C06F0DA
:10E0B8008FFA013654F80A0CB847032E04F1CC0441
:10E0C8007FF4C5ADE3E5013B002232482B6009F837
:10E0D80003201AF015FF75E6029A2F4B0392394672
:10E0E800A4F10A00029306F0EDF9D7E714F8053C0D
:10E0F80014F8032C0694234407936E2A4FF0000368
:10E1080008930993ADF820207FF42AAE06A8F2F709
:10E1180019FE06A8F2F70AFE06A8F2F707FE06A8F7
:10E12800F2F704FE1CE62246A3E61C48083F1AF054
:10E13800E7FEA6E61A481AF0E3FE8DE728681FE70F
:10E14800074807F0B8FD0BB0BDE8F08F154A14F882
:10E15800023CC2F80C80CAF80090A5E5034667E7C0
:10E16800B4320020C9330020A85E0308B05E03085B
:10E17800E4330020702500200C210020D90101087B
:10E18800B0320020DC5E0308045A0020F84B030874
:10E1980068370308D85E030854730020A05E03089C
:10E1A800BC5E030800ED00E0AC3200202DE9F04F22
:10E1B8002DED028B95B005460CF064F9B24B1C7836
:10E1C80024B115B0BDEC028BBDE8F08FDFF824B3A5
:10E1D800DBF800305E05F4D5AC4F3A68002A00F051
:10E1E8001C81AB4ED6F8283103F5F43348339D42F1
:10E1F800C0F01381A74996F82C310968C6F8285150
:10E208000133DBB2880786F82C3101F10B8113F05A
:10E21800070801F05780282B9F4B039301F0AC812E
:10E228005E2090479D4B1B78002B6BD0984E9C4AE4
:10E23800D6F83031EB1A934200F2C887DFF8B8A25B
:10E248009AF80090B9F1000F33D1DFF86482D8F85A
:10E25800000002F0DBF9C0B201280ED90228914F64
:10E2680041F063823B78002B41F09483D6F8383133
:10E27800EB1AB3F57A6F81F03B848B480268002A69
:10E2880040D09AF80030BBB9884BD8F800001B681A
:10E298009B781E3B012B4FF0020141F2878304302B
:10E2A8000CF020F8012200238AF8002086F8443177
:10E2B80026E07D4802682AB3D6F8403140F6B731E7
:10E2C800EB1A8B421ED996F83C31002B01F02482C0
:10E2D800013BDBB286F83C31002B01F00D8112F8CE
:10E2E800011B96F84471026096F845317048CA19C6
:10E2F8000133006886F8442186F8453102F08AF92E
:10E30800C6F840516B4A039B12781B68012A03F137
:10E3180001030C9300F0A786674B1B786BB1674F1E
:10E328003B6853B1039B5A4ED3F80090D6F8583146
:10E33800A9EB0303632B00F23986DFF8C08198F854
:10E348000090B9F1020F01F0B380564F97F874307E
:10E35800032B00F081875A4B1B7873B1594C236803
:10E368005BB14B4EFFF700FBD6F86431049044F6DE
:10E378001F62C31A934200F2D380534B1B78002BC1
:10E388004ED1524B1B7843B1414ED6F8B43203F507
:10E398000043E8339D4280F0E0864D4B1B78002B0C
:10E3A8003FF40FAF3A4E4B4C4B4D06F2BD27206859
:10E3B80002F02CF900283FF404AF206802F01EF99F
:10E3C8002B7880465A1E33B120682A7002F01EF955
:10E3D8000028F2D1F5E603223946781E24F067FDBD
:10E3E80096F8BC3296F8BD2286F8BF8283F47F4344
:10E3F80083F0FF039B1A1FFA88F89BB2B8EB132F20
:10E40800D5D196F8BE22DBB29A42D0D1781E0FF051
:10E41800EBFB2B7818442870C9E71F4B039301E7DF
:10E428002E4C2278002A40F015862D4F3C78002C7F
:10E4380066D12C4E3078002841F03782144E2A4C91
:10E44800D6F8AC122278294B93FBF2F30B449D4289
:10E4580097D396F8B032264AC6F8AC52D75CFB0779
:10E4680001F1A883B90701F161837A0701F1F98203
:10E4780096F8B0322178013393FBF1F201FB1233A5
:10E4880086F8B0327DE700BFC93300204C37002042
:10E49800842100207C43002054650020DE370020C2
:10E4A8003F0D03000C0000204437002040370020B7
:10E4B8003C370020DF370020EC3700209C66002026
:10E4C800F4370020F8370020383800204938002079
:10E4D800FE3700200438002008380020D0370020FC
:10E4E800413800204038002048380020A08601002C
:10E4F800443800205C4C00204837002096620020F9
:10E50800054E306E002841F012808146034B87F893
:10E518000090C3F8AC5234E7503800208421002022
:10E5280096F86A31002B40F0F887DC4B1A6802F045
:10E538000803002B48F603414AF60B404BF60F43FD
:10E5480049F6074704BF03460F4612F0040F4FF081
:10E55800190118BF1F46920686F86A1103D547F4B9
:10E56800804747F0200705F039F8C7F30909002864
:10E5780041F04284CA4B9B79002B41F0AC84984609
:10E5880064204FF0FF3A4FF0000C0C970D97ADF850
:10E598003CC0CDF842C0CDF846C0CDF84AC0CDF851
:10E5A8003890ADF83E80ADF840A08DF84E000CAF25
:10E5B8000FCFDFF804E386F805C0AEE80F0097E850
:10E5C8000F00AEE807002EF8023B71464FF0010C31
:10E5D8001B0CFE271F20C82201F81E39B770B27124
:10E5E80086F807C0F07096F87A01307180F0F10370
:10E5F80083EA0313DAB2130983F0E70343EA022339
:10E6080083EAC2031BB283EA0312D2B2C3F307231D
:10E6180083EA121343EA022383EAC2031BB283F09C
:10E62800C80282EA0212D2B2C3F3072383EA1213A2
:10E6380043EA022383EAC2031BB283EA0C0787EA90
:10E648000717FFB2C3F3072282EA171242EA07222A
:10E6580000EB0C0382EAC7070EEB0C0086F87A3150
:10E66800378011F8013B7B4083EA0313DBB21A09B8
:10E6780082EA172242EA032282EAC3031BB29FB24C
:10E6880081423780EDD183F07C0383EA0313DBB248
:10E698004FEA131E8EEA172E8EEA032E8EEAC30E59
:10E6A8000FFA8EFE1FFA8EF9DFF810C2A6F8009056
:10E6B8005FFA8EFE4FEA192986F8289086F827E037
:10E6C8000CF5D17806F1220ADCF80000DCF8041019
:10E6D800DCF80820DCF80C3047460FC70CF1100CAA
:10E6E800D445B846F0D1DCF8000038606D4F9CF88E
:10E6F800043088F8043007F1270886F8C9E186F85D
:10E70800CA9117F8011F206801F084FFB845F8D1B5
:10E7180096F86B31002B40F005876349039A097816
:10E7280012680A2086F86B01002901F0AB805F4F60
:10E7380001293888089041F2BE830229B7F802E01F
:10E7480001F07483B8880790032901F0BD83F88825
:10E758000690042901F071840529388901F068843C
:10E768000629B7F80A9001F05F840729B7F80C80EA
:10E7780001F05784FB89059396F87A110C920B46A1
:10E7880083F0300282EA0212D2B21709484909938B
:10E7980087F07A0747EA02270988337187EAC202B5
:10E7A800444FC1EB012187FB013A089B4FF0000C55
:10E7B80063F30F0C079B6EF31F4C4FF0000E63F3CF
:10E7C8000F0E069BCDF834C012B28A440027C91731
:10E7D80063F31F4EC1EB6A2A059BCDF838E082EA45
:10E7E800021160F30F070020C9B268F30F00C2F3EB
:10E7F800072269F31F4782EA111263F31F404FF0A3
:10E8080000090F978DF845A010908DF8449042EAC2
:10E8180001220DF1300C82EAC107BCE80F003FB2BB
:10E8280087F0C80888EA0818DFF88CE086F80590B1
:10E838005FFA88F8C7F30727AEE80F0087EA1817CA
:10E8480047EA08239CE8030083EAC8031BB283F065
:10E8580023024EF8040B82EA0212D2B2C3F3072352
:10E86800099F83EA1213704643EA022383EAC2022D
:10E8780007F1010C20F814194FF023081621FE2780
:10E88800C82386F87AC1328086F807800EF1020E16
:10E89800B770F170B371114612E000BF7C430020DD
:10E8A8006043002027230020C0470020FA71002081
:10E8B80030370020030820808C210020862100208A
:10E8C80010F8013B4B4083EA0313DBB21A0982EAD2
:10E8D800112242EA032282EAC3031BB299B27045AD
:10E8E8003180EDD183F0F40383EA0313DBB24FEAFE
:10E8F800131E8EEA112E8EEA032E8EEAC30E0FFA2D
:10E908008EFE1FFA8EF8E64FA6F800804FEA182C04
:10E918005FFA8EFE86F81EE086F81FC07968BA682E
:10E928003868FB6807F5D178A8E80F003869796975
:10E93800BA6906F2A317A8E8070006F2C11886F814
:10E94800C1C186F8C0E117F8011F206801F062FE16
:10E95800B845F8D196F87271002F40F0D985D14B9F
:10E9680096F87AE1B3F90010B3F90220B3F904304C
:10E978009FEDCD6A777107EE103A039B1B680C93E5
:10E988008EF06A0383EA031306EE901AD9B20B09D4
:10E9980083F0D50343EA012383EAC1031BB283EA68
:10E9A80003115242C9B207EE902AC3F3072383EA40
:10E9B800111343EA0123F8EEE77AF8EEE66AB8EEB7
:10E9C800C77A83EAC1031BB267EE867A66EE866A67
:10E9D80027EE067A002083F0C808CDED0E7ACDED3B
:10E9E8000D6A8DED0F7A10901190129088EA081C2C
:10E9F8000DF130095FFA8CFCC3F30728B9E80F0062
:10EA080088EA1C1848EA0C2888EACC08DFF8A8C26B
:10EA18000FFA88F8ACE80F0088F01E0799E807009D
:10EA280087EA0717FFB2C8F3072383EA171343EAF5
:10EA380007238CE8070083EAC7071C20C8214FF08A
:10EA480005094FF01E08FE230EF10102F07086F84A
:10EA5800729186F80780B3700CF10C00B171ACF1BB
:10EA6800100186F804E0378086F87A2111F8013B16
:10EA78007B4083EA0313DBB21A0982EA172242EACF
:10EA8800032282EAC3031BB29FB281423780EDD1D1
:10EA980083F0270383EA0313DBB24FEA131E8EEADF
:10EAA800172E8EEA032E8EEAC30E0FFA8EFE1FFA79
:10EAB8008EF9DFF8ECC1A6F800905FFA8EFE4FEAF7
:10EAC800192986F8259086F824E00CF5D17806F106
:10EAD800220ADCF80000DCF80410DCF80820DCF876
:10EAE8000C3047460FC70CF1100CD445B846F0D18E
:10EAF8006E4FBCF80030A8F8003007F1240886F8FB
:10EB0800C6E186F8C79117F8011F206801F082FD59
:10EB1800B845F8D196F873310393002B40F0F4848C
:10EB280096F87AA15F4B624AB3F90410B2F906204D
:10EB3800604FDFF888C1DFF880E186F804A08AF02A
:10EB4800220080EA0010C0B2030983F0590343EAA7
:10EB5800002383EAC0031BB2B2F5FA6F83EA0310FD
:10EB6800C0B2A8BF4FF4FA62C3F30723B2F57A7FA5
:10EB780083EA101343EA0023B8BF4FF47A7283EA9A
:10EB8800C000A2F57A72642303FB02F28CFB029C9C
:10EB9800D31787FB0172C9174FF0000807B2C3EB00
:10EBA800AC13C1EBA2010DF13009CDF83080CDF8DE
:10EBB8003480CDF83880CDF83C8087F0C80CADF8AB
:10EBC8004230ADF84010C846B8E80F008CEA0C1C7B
:10EBD8005FFA8CFCC7F3072787EA1C1747EA0C275C
:10EBE80087EACC07AEE80F003FB287F04A0383EA12
:10EBF8000313DBB2C7F3072181EA131141EA0321AA
:10EC0800724681EAC303D8F800C09DF80C107171F0
:10EC18000AF1010705204A214FF0FE0886F87A71AB
:10EC280042F810C914274FF0C80C86F873013380D6
:10EC38000EF1040EF17186F80280F77086F806C0AE
:10EC4800184612F8011B414081EA0111C9B20B09AB
:10EC580083EA102343EA012383EAC10109B288B297
:10EC680072453080EDD181F0140181EA0111C9B2F9
:10EC78004FEA111E8EEA102E8EEA012E8EEAC10E80
:10EC88000FFA8EFE1FFA8EFC4FEA1C2A044B04482A
:10EC980086F81DA05FFA8EFE86F81CE010E000BF23
:10ECA800862100208043002088C3E43A27230020DF
:10ECB800FA710020676666668C210020D34D6210C9
:10ECC800DA4F59689A680068DB68A6F800C007F54B
:10ECD800D17CACE80F0038697969B7F81880ACE8DE
:10ECE800030006F2A317ACF8008086F8BFA1B84667
:10ECF80086F8BEE106F2BF1A18F8011F206801F075
:10ED080089FCC245F8D1CA4BCA4A1B781278013B24
:10ED180012F00100DBB214BFC0214021172B03D829
:10ED2800C54A13441B7B0393C44B1A8893071ABF25
:10ED3800002341F01001012312F4027F18BF0223BF
:10ED480012F0100F18BF062312F0200F18BF10235F
:10ED5800002840F0C3864FF0030C96F87AA10C9374
:10ED68008AF0460383EA0313DAB2130983F09203A5
:10ED780043EA022383EAC2031BB283EA0310C0B248
:10ED8800C3F3072282EA101242EA002282EAC00292
:10ED980012B282F0C80E8EEA0E1E00235FFA8EFEB3
:10EDA8009DF80C808DF834800320C2F307228DF87B
:10EDB80037C082EA1E128DF835308DF836108DF87E
:10EDC800380042EA0E2C99E807008CEACE0E0FFABA
:10EDD8008EFEDFF87482F3718EEA0E1CA8E8030039
:10EDE8005FFA8CFCCEF3072E8EEA1C1E4EEA0C212D
:10EDF80081EACC0C96F808E088F800200FFA8CFC21
:10EE08008EEA0C0E8EEA0E1E5FFA8EFECCF30722F7
:10EE180082EA1E1242EA0E22707AB17A96F80BC084
:10EE2800737182EACE0E0FFA8EFE80EA0E0080EA37
:10EE38000012D2B2CEF3072080EA121040EA022074
:10EE480080EAC20000B2414081EA0111C9B2C0F3B0
:10EE5800072282EA111242EA012282EAC10212B2B0
:10EE68008CEA020C8CEA0C1C5FFA8CFCC2F30722B9
:10EE780082EA1C1242EA0C2296F80CE0707BB17B05
:10EE880096F8109086F804A082EACC0212B28EEAB4
:10EE9800020E8EEA0E1E5FFA8EFEC2F3072282EA87
:10EEA8001E1242EA0E2282EACE0212B2504080EAD4
:10EEB8000010C0B2C2F3072282EA101242EA00220E
:10EEC80082EAC00212B2514081EA0111C9B2C2F30A
:10EED800072282EA111242EA012282EAC102F17B88
:10EEE80013B281EA030282EA0212D2B2C3F3072301
:10EEF80083EA121343EA022383EAC2031BB289EAB4
:10EF0800030282EA0212D2B2C3F3072383EA12137E
:10EF180043EA022383EAC2031BB283F0320282EA85
:10EF28000212D2B2C3F3072383EA121343EA02237D
:10EF380083EAC2031BB29AB24FF0FE0C0AF1010138
:10EF4800DBB232804FF0090EC82086F802C04FEAC3
:10EF5800122CA8F10E0286F803E0B07186F87A1137
:10EF680086F812C00393737458F80E0C51689268AF
:10EF780038F802AC9DF80C3008F5CA7EAEE80700F8
:10EF880008F5D2788EF80290AEF800A086F8B4C1E1
:10EF980086F8B33117F8011F206801F03BFBB8452C
:10EFA800F8D1049BC6F86431FFF7E7B9DFF89CA0F5
:10EFB800DFF89C8041200FF05DF8BAF9023088FB39
:10EFC8000320DB17C3EBA00080B20FF039F8BAF9C1
:10EFD800003088FB0320DB17C3EBA00080B20FF0E2
:10EFE8002FF8BAF9043088FB0320DB17C3EBA00025
:10EFF80080B20FF025F8124B3868197801F00AFB37
:10F0080096F85C3113F0010800F095830D4AC6F8B4
:10F0180058910133DBB2A2FB0312D20802EB820241
:10F02800A3EB420386F85C31FFF787B986210020FD
:10F03800705200200340002078370308D043002096
:10F0480048730020CDCCCCCC8C21002080430020FC
:10F05800676666668B4B8C49186801F0A7FA00232F
:10F068002370FFF7E2B9894F386800283FF454A9A4
:10F078004FF0000A2346DFF84882854E049554462F
:10F088009A4601F0C3FAF8B1F4B94FF001092546E0
:10F09800386801F0B3FA83B27E2B00F01E8298F82C
:10F0A8000120002A4BD196F84811C1B11B2B86F8D4
:10F0B800482100F0EC810D2B47D0386888F8019082
:10F0C80001F0A4FA0028E3D15346A24650460CAA00
:10F0D8007049049D1C460EF0E5FFFFF71DB97D2B16
:10F0E80000F0C78396F84C2122B180F02003DBB2F0
:10F0F80086F84C1196F84721062A10D8B6F84A1116
:10F1080038681944A6F84A11B118013281F850310B
:10F1180086F8472101F07AFA0028B9D1D4E7B6F881
:10F128004A2188F8019013449BB21A0A52FA83F3D1
:10F13800FF2BA6F84A31386802D1574CA1E7386846
:10F1480001F064FA0028A3D1BEE73868A6F84A217E
:10F1580001F05CFA00289BD1B6E796F8B832C6F8F9
:10F16800B452012B40F2DC8296F8B9224B49981828
:10F1780001EB8001013202F001024F6A86F8B922E0
:10F18800BFB1474C0D940DF15009123CA52349F825
:10F19800204D802286F8103115232946484686F8E6
:10F1A800112186F81231B847002840F03F8296F8BE
:10F1B800B8323C4A013382FB0312A2EBE37202EB42
:10F1C80042029B1A86F8B832FFF7E7B8364A374B3F
:10F1D80092F80BE0039A1B881168D6F8342134485A
:10F1E800891A4FF47A72DFB202FB0EF21B0A877794
:10F1F800077591424FF00007C37743758770077111
:10F2080080F07B822B4B2C491A689B68C6F83051DA
:10F2180081FB02E7D21781FB03E1C2EBA702DB17F0
:10F22800C3EBA10311124FEA232C4FF0F40E02771F
:10F238000127417780F8203030217522782380F823
:10F2480021C080F81AE0C77680F8221080F82320C1
:10F2580080F82430FEF7F2BF184B0493186801F0C9
:10F26800C9F900283FF477A8049B0121186801F028
:10F27800BDF90222002387F8742088F80030FFF7D0
:10F288006AB800BF3C38002090370020383700208B
:10F2980084210020CA220020D422002078370308C5
:10F2A800A92200205655555590410020884100203C
:10F2B8000C3800207043002067666666B46300203F
:10F2C8000C0000205E2090473B6802209847FF20F2
:10F2D8000EF010FC0378FF2B00F0668390F90130E4
:10F2E8004FEAE3785FFA88F8D8B20BF04FF8404657
:10F2F8000BF04CF83B685E2098473B680320984722
:10F30800FF200EF0F7FB0378FF2B00F04983B0F9DC
:10F318000830D8B2C3F307280BF038F840460BF092
:10F3280035F8B14B1B78042B77D0DFF8E8A2B6F894
:10F338002E119AF80020DFF8E09291FBF2F302FB1D
:10F3480013139BB2B9F80010A6F82E314FEA031830
:10F358001FFA88F8642303FB01235200B3FBF2F37E
:10F3680048EA0328C3F303225E203B681FFA88F8A3
:10F3780048EA020898473B68062098475FFA88F0F1
:10F388000BF004F84FEA18200BF000F89749B6F88C
:10F398002E214B7AB9F800900132012BA6F82E21C4
:10F3A80000F067854A7B09EB89031FFA83F9002A75
:10F3B80040F08F833B685E2098473B683A20984727
:10F3C8008B4BA3FB09384FEA58181FFA88FA5FFAE3
:10F3D8008AF00AF0DBFF4FEA1A200AF0D7FF3B68F1
:10F3E8005E2098473B683B209847642303FB1893AB
:10F3F8009BB28048053380FB0320DB17C3EBA000DA
:10F40800C0B20AF0C3FF00200AF0C0FFDFF80C8288
:10F4180098F80630002B40F0F38296F82C313A68C1
:10F42800FEF7F9BEDFF8F8819FED738A4FF0240AE2
:10F438005E20904750463B689847704BF8EC016A4D
:10F448009B8A07EE103AF8EEE66AB8EEC77A0AF138
:10F45800010AC6EE877A5FFA8AFA67EE887AFDEEC5
:10F46800E77ACDED037ABDF90C905FFA89F00AF0DE
:10F478008DFFC9F307200AF089FFBAF1270F01D0E1
:10F488003A68D5E796F82C313A68FEF7C0BE386876
:10F4980001F0BCF800287FF410AE386886F8469171
:10F4A80088F8019001F0B2F800287FF4F1AD0BE67E
:10F4B800FEF75AFA524B1B68A0EB030A40F6B83322
:10F4C8009A4500F2CB814F4A13793A2B00F0DA8340
:10F4D800002388F80030FEF73EBF386886F84651AA
:10F4E80086F8475186F8489188F8015001F08EF85F
:10F4F80000287FF4CDADE7E596F8441196F845313C
:10F5080041484A1CFEF7F4BE013B86F8733148E5D2
:10F51800013F86F87271FFF7FDBA013B86F86A3140
:10F52800FFF7F6B8013B86F86B31FFF713BA0024F2
:10F53800DFF8F080A1464FF0500A02E0DBB283F317
:10F54800118816F804B0601C594630440EF076FC59
:10F55800002840F0A1810BF101031C44EFF3118353
:10F568008AF31288326E9442E8DB0022DBB23266FC
:10F5780083F31188FEF7CABF4FF0000A5E20D3F864
:10F58800008086F82CA190473B68DFF89C901720F4
:10F59800984750460AF0FAFE1C4BA3FB08239B0B26
:10F5A800A9FB03125209C2EB0212A3EB8203D8B2E1
:10F5B8000AF0ECFE3B685E2098473B6818209847A5
:10F5C800134BA3FB08239B09A9FB03125209C2EBA7
:10F5D8000212A3EB8203D8B20AF0D8FE50460AF012
:10F5E800D5FE3A68FEF71CBE343700209041002053
:10F5F8001F85EB516766666600007A4488430020E1
:10F608009C620020846200203C37002073B2E745EA
:10F61800D34D62109E4100208841002060430020A5
:10F62800B84300200DA40108898888880C9DA5424C
:10F638004FF000014FD941F2210014F8013B81EA53
:10F648000323590013F4004F80EA010289B292B2F1
:10F6580008BF0A46530012F4004F80EA03019BB228
:10F6680089B208BF19464B0011F4004F80EA030223
:10F678009BB292B208BF1A46530012F4004F80EAB8
:10F6880003019BB289B208BF19464B0011F4004F21
:10F6980080EA03029BB292B208BF1A46530012F4E2
:10F6A800004F80EA03019BB289B208BF19464B009C
:10F6B80011F4004F80EA03029BB292B208BF1A46C7
:10F6C800510080EA010312F4004F9BB289B218BFBF
:10F6D8001946AC42B1D14846F1F76AFBB5490C9CD2
:10F6E800B548641A152CA8BF1524224622F0FCFA46
:10F6F800B24A96F8B83214705BE5B14B039A1B789E
:10F708001268C6F83421013B012B3FF67BAD10226D
:10F7180002238270037175E50AF01AFEFEF7F0BD48
:10F72800A84A02EB8302576A2AE50AF001FE012380
:10F738003B70FEF7A2BDA44B1B88DA0515D4D8068A
:10F7480000F17183990600F1A4835A0600F1A7839A
:10F75800180700F1A783D90700F1A78313F0020F58
:10F768000CBF4FF004084FF00C08984B984A1B78D0
:10F77800D27803F001030AB143F002035320049343
:10F788000EF078FC934A128802EB820202EB8202A6
:10F79800900080B20EF054FC00200EF051FC8E4A0E
:10F7A8008E4912883868C2EBC212520081FB0231BE
:10F7B80011444FEAE27ACAEB612A5FFA8AFA5146A3
:10F7C80000F028FF864B38681A78049B48EA03083B
:10F7D800834B8AEA020A002183F800A000F01AFF8E
:10F7E8004146386800F016FF7D4B7D4A1B78386823
:10F7F80088EA0303DBB21946137000F00BFF96F892
:10F808005C31002B7FF402AC4F200EF033FC20F06B
:10F818001FFE20F01DFE20F01BFE0121386800F0BD
:10F82800F9FE704A6E4B92F800801B786C4A386873
:10F8380008F0010883F001034146137000F0EAFE66
:10F84800674B674A1B78386888EA030319461370C0
:10F8580000F0E0FE96F85C31FFF7D8BB624AB2F8D8
:10F868005E3100210133A2F85E3188F80010FEF7FE
:10F8780072BD386886F84C9100F0C8FE00287FF405
:10F8880007AC21E4884689460846069107918E46CA
:10F8980008910591FEF770BF41463A200EF02AFA0A
:10F8A80040EA09095FFA89F955E65049504B009337
:10F8B800A1F13F074F4B504A0B9101F8404C0CA85F
:10F8C8004E490A97F1F74CFB0A9F7B1C0A933C7040
:10F8D8000A9B2922591C0A911A700A9BEA22591C70
:10F8E8000A911A700A9BC822591C0A910CA81A700E
:10F8F80021F08CFA00F101080CA942460A9822F07E
:10F90800F3F90A9A02EB080301330A9302F8084054
:10F918000A9B5A1C0A921C700A9B5A1C0A921C7059
:10F928000A9B5A1C0A921C700A9B5A1C0A921C7049
:10F938000A9B5A1C0A921C700A9B5A1C0A921C7039
:10F948000A9B5A1C0A921C700A9B5A1C0A921C7029
:10F958000A9B5A1C0A921C700A9B5A1C0A921C7019
:10F968000A9B5A1C0A921C700A9B5A1C0A921C7009
:10F978000A9B0122991814A80A911A7050F8283D78
:10F98800DB1B3B700AF024FD174B3470C3F8AC52F4
:10F99800FEF7F7BCC6F8385187F80090FEF76DBC43
:10F9A8004FF000084046B7E440469EE400F01EFED3
:10F9B800FEF778BC942200206C5B0020815B00205D
:10F9C8003437002078370308D04300200340002054
:10F9D8002034002088410020303700200308208090
:10F9E800487300207C52002084210020903700209A
:10F9F800EA330020005F0308085F0308145F030868
:10FA08003B68DFF87492DFF868A25E2098473B688D
:10FA180028209847D9F800308AFB032ADB17C3EB64
:10FA2800AA0A5FFA8AF00AF0B1FCCAF307200AF0C2
:10FA3800ADFC3B685E2098473B6804209847B8F8BF
:10FA48000830002B40F0FA81D9F8083083F3100809
:10FA58005FFA88F00AF09AFCC8F307200AF096FCCF
:10FA6800DBE47A4B7A4A0D93A3F14008126800212F
:10FA780003F8401C212388F80230D30040F1ED81BF
:10FA880074490327744B1B88580500F1E381DA0792
:10FA980000F1028203F00203704A002B1CBF032707
:10FAA8001146DFF8D8913A46484622F01DF907EB8F
:10FAB800090314A80133A9F1020140F8203D0022EE
:10FAC8005B1A07F8092088F801300AF081FCFEF774
:10FAD800CFBC9AF8003099FBF3F96BE4604AD2780E
:10FAE800002A0CBF4FF0040C4FF0050CFFF735B996
:10FAF8000123D8F800003B7000F080FD0746D8F8D5
:10FB0800000000F07BFD79067EF4B7AB8E287EF40A
:10FB1800B4AB9AF80030002B7EF4CBAB514B524A71
:10FB28001A602D2386F83C31FEF7AEBB474A4F4B8F
:10FB38000D920DF15008A2F13D0048F8200D1988EA
:10FB4800DFF83491A2F1400300204FF00A0E02F8CA
:10FB5800400C082283F801E040469A70F1F702F958
:10FB6800D9F800304249DA1781FB0313C2EBA3032B
:10FB780099B24046F1F7F6F803F03EFDD9F808903F
:10FB88000C9B4FEA1942591C0C911A700C9B4FEAB6
:10FB98001922591C0C911A700C9B5A1C0C9283F850
:10FBA80000900C9B5A1C0C92187040460AF010FCEE
:10FBB800FEF75BBCDFF8C8909FED2E8AB9F90230DA
:10FBC800224A0D9207EE903AF8EEE77A0DF15008C6
:10FBD80067EE887AA2F14003FDEEE77AA2F13D01D3
:10FBE80048F8201D02F8400C0822CDED037A5A701F
:10FBF8001E229A70BDF80C104046F1F7B3F8B9F917
:10FC0800003007EE903AF8EEE77A404667EE887AD9
:10FC1800FDEEE77ACDED037ABDF80C10F1F7A2F806
:10FC2800B9F9043007EE903AF8EEE77A404667EE05
:10FC3800887AFDEEE77ACDED037ABDF80C10F1F77E
:10FC480091F840460AF0C4FBFEF70CBC9037002040
:10FC5800F8600020EC5E0308D0430020FC5E030837
:10FC680020340020443700200C3800208841002030
:10FC78006766666658A08B417043002053370020A2
:10FC8800804300209178049210461DF0E7FC049A06
:10FC980000287FF41DAC9349934F944B944E0988E8
:10FCA8000592944AF961F863B6F85E1118689B6882
:10FCB800C7F86CA0F862FB641068F965049200F05C
:10FCC8005BFA824600287EF441AB049B49461868DB
:10FCD80000F08CFC059A96F86031D2780692642B75
:10FCE8004FF0040287F8742040F0168196F86131CD
:10FCF800072B08BF86F861A196F86131089307EBD6
:10FD08000319D9F804100591084621F07FF8D9F8AD
:10FD1800081007915FFA80F9084621F077F85FFA32
:10FD280080FA089B74480599059009EB0A02083285
:10FD3800C27123F00F0282726F4A03F00F035373EC
:10FD48006D4B0AEBC900987318464A460F3021F0EC
:10FD5800CBFF6A4B079909F109001844524621F074
:10FD6800C3FF0598C37903F10109CBB1013B5FFAE1
:10FD780083FC0CF1080CDFF89CE184440023073075
:10FD880010F8012B5A409300D10883EA420301F08E
:10FD9800180153404EFA01F253408445DBB2EFD1CB
:10FDA800564A069809F8023021F07AFF96F8613130
:10FDB8000022013386F8613186F86021059BDDF861
:10FDC80014909B785BB1049B19F80410186800F034
:10FDD80021FC013499F80230E4B2A342F3D896F832
:10FDE80060310322013386F8603187F8742088F87F
:10FDF8000020049BFFF732BA3A4B414A1B8892799C
:10FE080003EB830303EB83034FEA83081FFA88F8A5
:10FE1800002A4DD0354B1B680FFA83FA03F0ECFB30
:10FE280040B2FEF7B0BB4FF034089EE498469946BE
:10FE38001846069307930593FEF79EBC03F0DCFB78
:10FE48000AF0A4FA00200AF0A1FA96F82C313A68D0
:10FE5800FEF7E1B903272B4923E6DBF800302A4AED
:10FE68002A4903F48003002B16BF114604270327F1
:10FE780008E63B685E2098473B68392098475FFA58
:10FE880089F00AF083FA4FEA19200AF07FFAFFF79F
:10FE9800BDBA4FF0240868E41D49042701E64FF075
:10FEA800100862E44FF020085FE44FF008085CE4B3
:10FEB8004FF0FF33B0E798469946184606930793E4
:10FEC8009E460593FEF758BC9846994618460693F1
:10FED8000593FEF751BC054B8046B3F900A064209A
:10FEE800FEF751BB884100200C0000207043002021
:10FEF80084210020B4630020746600207A66002004
:10FF080060430020F05E0308EC5E0308E45E03082B
:10FF1800F45E03080007090E97F875904B494C4AA0
:10FF2800059219F00F0F04BF09F101095FFA89F969
:10FF3800B9F1070F28BF4FF001094FEA091A07EB7B
:10FF48000A035FFA8AFC187C0023095C937202F1A9
:10FF58000D0307EB0A024CEA000001291870D26869
:10FF680003F1010E0CD90239C9B2881C1844734632
:10FF780003F8012B83424FEA1222F9D101318E4452
:10FF8800BA4422F0600309F101099AF811205FFAD6
:10FF980089F91343B9F1080F8EF800300EF1010307
:10FFA80051D04FEA091A07EB0A012A4A087C274967
:10FFB800095C9A1A02EB010E0CF1100CBEF1130F3A
:10FFC8005FFA8CFCC5DDD2B2931DDBB20598DFF871
:10FFD8008CE043F04001C17103F1010CCBB1053253
:10FFE8005FFA82FA0AF1080A824400230EF101003E
:08FFF80010F8011B59408B00B9
:020000040801F1
:1000000083EA4103CA084B40154902F0180241FA3D
:1000100002F253408245DBB2EED106980CF80E3066
:1000200087F8759021F040FECCE60593FEF7A8BB5B
:1000300098460593FEF7A4BB984699460593FEF7AC
:100040009FBB9846994618460593FEF799BB034A0D
:100050009A1ABCE77837030874660020816600208E
:100060000007090E7A660020436A8269D154436A08
:100070000169826B01338B4228BF00234362002A4F
:100080002FD0EFF31181502383F31288836B1A680A
:10009000D2072CD470B45E686EB9456A826A954204
:1000A00017D084691444DC600ED9AA1A5A6085629C
:1000B000002280F854201A6842F00102C9B21A6086
:1000C00081F3118870BC70470469A21A5A60866275
:1000D000EEE7012380F85430C9B281F3118870BC77
:1000E0007047026D136843F0800313607047C9B214
:1000F00081F31188704700BF426B10B462B1436C4A
:10010000C2684469D11A013B615C5DF8044B08BFC9
:1001100013464364C8B27047016A4369C4685B5CB4
:100120000131A14228BF114601625DF8044BD8B2EB
:10013000704700BF836B13B190F854007047836A17
:10014000406A181AB0FA80F040097047416A836A21
:1001500099420AD3CB1A816B026961B14968501E7A
:100160000B4483420AD2C01A704702691144CB1A69
:10017000816B0029F2D1501EC01A704700207047D1
:10018000436B43B1426C5B6893422FBF981AC068BF
:100190009B1AC0187047C269036A9A422FBFD01ACF
:1001A000C0688018C01A70470A4B30B503F11404B8
:1001B00093F900205D78072AC8BF143A81180433E8
:1001C0000D7313F8025C855413F8012C0A76A342D0
:1001D000EED130BDAC37030803682DE9F041DF698B
:1001E0001FB13B46BDE8F0411847002A164611DD15
:1001F00004460D460E4400E023689B68204698475D
:100200000028F9D0236815F8011B1B682046984781
:10021000AE42F1D1BDE8F081002325220270437087
:100220008370C37070472D2343702E2303712F23D7
:10023000C371704730B50446006D61710368A268F0
:1002400023F00103036087B0A379009213F0040246
:100250003DD04FF4805213F00203019244D1029337
:100260004FF480630022039311F00103059237D10C
:10027000049308238D07694648BF04930CF088FD5A
:100280006079236DA17900F00202002A15BF4FF4B6
:1002900040324FF480324FF40034002410F0010F4C
:1002A000586808BF2246CC074CBF024320EA02022E
:1002B0005A609A6809074CBF42F0080222F008020F
:1002C0009A601A6842F001021A6007B030BD13F05C
:1002D000020301920BD04FF4005513460295C1E77B
:1002E000042304930C23C5E74FF40053B7E70293AC
:1002F000B8E700BF10B50446006DA160036823F0A5
:1003000001030360A37986B013F00402009141D089
:100310004FF4805213F00203019244D102934FF440
:10032000806362790393D1074FF000030493059330
:1003300045BF0423049308230C236946920748BF52
:1003400004930CF025FD6079236DA17900F0020281
:10035000002A15BF4FF440324FF480324FF400347E
:10036000002410F0010F586808BF2246CC074CBF8C
:10037000024320EA02025A609A6809074CBF42F021
:10038000080222F008029A601A6842F001021A601C
:1003900006B010BD13F00203019207D04FF40051D4
:1003A00013460291BDE74FF40053B7E70293B8E755
:1003B00000231922036042701A22C2700122436096
:1003C0004271C371704700BF1D4B70B59C68236DAF
:1003D000626BDD69C2B1A36B2BB12B0702D5236D14
:1003E00008221A6270BD2A06F7D5A26A616A8A429B
:1003F00020D0511CA069A162825C2069266D8142D7
:100400003285EAD3A362E8E7A906E4D5E26A22B11D
:10041000988C216B80B29047DDE7E1699B8C606925
:10042000DBB24E1CE6614354E169E368994228BFA0
:10043000E261D0E7226D136823F080031360CCE7FC
:10044000A82C00201D4B70B55C68236D626BDD69C4
:10045000C2B1A36B2BB12B0702D5236D08221A6200
:1004600070BD2A06F7D5A26A616A8A4220D0511C63
:10047000A069A162825C2069266D81423285EAD33F
:10048000A362E8E7A906E4D5E26A22B1988C216B61
:1004900080B29047DDE7E1699B8C6069DBB24E1C5E
:1004A000E6614354E169E368994228BFE261D0E71D
:1004B000226D136823F080031360CCE7A82C002082
:1004C0001D4B70B51C68236D626BDD69C2B1A36BF7
:1004D0002BB12B0702D5236D08221A6270BD2A06A4
:1004E000F7D5A26A616A8A4220D0511CA069A16234
:1004F000825C2069266D81423285EAD3A362E8E7F7
:10050000A906E4D5E26A22B1988C216B80B29047AB
:10051000DDE7E1699B8C6069DBB24E1CE661435408
:10052000E169E368994228BFE261D0E7226D136870
:1005300023F080031360CCE7A82C002070B4EFF305
:100540001186502383F31288836B1A68D20720D454
:100550005D686DB9446A826A944217D0816911441A
:10056000D9600ED9A21A5A608462002280F8542001
:100570001A6842F00102F1B21A6081F3118870BC6E
:10058000704701698A1A5A608562EEE7012380F894
:100590005430F1B281F3118870BC704703685B6A14
:1005A00003B11847704700BF03681B6A03B11847BF
:1005B000704700BF03682DE9F041DF691FB13B467A
:1005C000BDE8F0411847002A164611DD04460D46E5
:1005D0000E4400E023689B68204698470028F9D025
:1005E000236815F8011B1B6820469847AE42F1D1DD
:1005F000BDE8F08103689B69184700BF03685B6929
:10060000184700BF0368DB68184700BF03689B6892
:10061000184700BF03685B68184700BF03681B6882
:10062000184700BF054B53F8203033B11A689B8838
:10063000918A0B4218BF1B0493617047206500200C
:1006400003682DE9F04F03F13845644EAD0A0124EB
:10065000755D05F01F066D09022D04FA06F400F021
:10066000A280032D00F0A480012D52D08088B0FA22
:1006700080F4C4F11F04A4B2E50803EB850504F07F
:1006800007042E6AA4000F27A74026EA07062E6259
:100690002E6A01F0030702FA04F47A1E3443012A99
:1006A000C1F3810CC1F300182C62C1F3411135D99B
:1006B000C60700F19780850700F1A380440700F189
:1006C000B180020700F1BF80C60600F1CD8085062B
:1006D00000F1DB80440600F1E980020600F1F780BA
:1006E000C60500F10581850500F11381440500F17F
:1006F0002181020500F12F81C60400F13D818504AE
:1007000000F14B81440400F15981020455D4BDE845
:10071000F08F334D6E6934436C61A7E700242246A5
:100720004FF0010E4FF0030904E00132102A04F1EA
:100730000204ECD00EFA02F636EA0005F5D1D3F841
:1007400008A009FA04F5ED430AEA050AC3F808A06F
:10075000D3F808B00CFA04FA4AEA0B0AC3F808A066
:10076000B3F804A01FFA8AFA2AEA06069E80B3F8B4
:1007700004A008FA02F646EA0A06B6B29E801E688F
:100780002E401E60D3F800A007FA04F646EA0A06D7
:100790001E60D3F80CA001FA04F605EA0A0A46EA3C
:1007A0000A05DD60C1E70E4DAE693443AC615DE71B
:1007B0000B4DEE693443EC6158E71A6822F0404271
:1007C0001A601A6842EA87771F60DA6822F04042AE
:1007D00042EA8171D960BDE8F08F00BF6C5903080F
:1007E000001002401A6822F003021A601A683A43A5
:1007F0001A60DA6822F003020A438507DA607FF59F
:100800005DAF1A6822F00C021A601A6842EA870289
:100810001A60DA6822F00C0242EA81024407DA60C8
:100820007FF54FAF1A6822F030021A601A6842EA68
:1008300007121A60DA6822F0300242EA0112DA6026
:1008400002077FF541AF1A6822F0C0021A601A68E9
:1008500042EA87121A60DA6822F0C00242EA811284
:10086000C606DA607FF533AF1A6822F440721A6068
:100870001A6842EA07221A60DA6822F4407242EAF1
:1008800001228506DA607FF525AF1A6822F44062FE
:100890001A601A6842EA87221A60DA6822F4406213
:1008A00042EA81224406DA607FF517AF1A6822F423
:1008B00040521A601A6842EA07321A60DA6822F473
:1008C000405242EA0132DA6002067FF509AF1A6847
:1008D00022F440421A601A6842EA87321A60DA68E3
:1008E00022F4404242EA8132C605DA607FF5FBAE6F
:1008F0001A6822F440321A601A6842EA07421A6003
:10090000DA6822F4403242EA01428505DA607FF576
:10091000EDAE1A6822F440221A601A6842EA874251
:100920001A60DA6822F4402242EA81424405DA6021
:100930007FF5DFAE1A6822F440121A601A6842EAA4
:1009400007521A60DA6822F4401242EA0152DA6071
:1009500002057FF5D1AE1A6822F440021A601A68C7
:1009600042EA87521A60DA6822F4400242EA81526F
:10097000C604DA607FF5C3AE1A6822F040721A60CE
:100980001A6842EA07621A60DA6822F0407242EAA4
:1009900001628504DA607FF5B5AE1A6822F0406224
:1009A0001A601A6842EA87621A60DA6822F04062C6
:1009B00042EA81624404DA607FF5A7AE1A6822F049
:1009C00040521A601A6842EA07721A60DA6822F026
:1009D000405242EA0172DA6097E600BF036803F111
:1009E00038422DE9F04F920A584DAA5C02F01F05DB
:1009F00052090124022A04FA05F400F08C80032A2B
:100A000000F08E80012A3CD001F003077A1E012AF3
:100A1000C1F3810CC1F300188088C1F3411135D9AD
:100A2000C60700F19780850700F1A380440700F115
:100A3000B180020700F1BF80C60600F1CD808506B7
:100A400000F1DB80440600F1E980020600F1F78046
:100A5000C60500F10581850500F11381440500F10B
:100A60002181020500F12F81C60400F13D8185043A
:100A700000F14B81440400F15981020455D4BDE8D2
:100A8000F08F334A55692C435461BDE70024224658
:100A90004FF0010E4FF0030904E00132102A04F177
:100AA0000204ECD00EFA02F636EA0005F5D1D3F8CE
:100AB00008A009FA04F5ED430AEA050AC3F808A0FC
:100AC000D3F808B00CFA04FA4AEA0B0AC3F808A0F3
:100AD000B3F804A01FFA8AFA2AEA06069E80B3F841
:100AE00004A008FA02F646EA0A06B6B29E801E681C
:100AF0002E401E60D3F800A007FA04F646EA0A0664
:100B00001E60D3F80CA001FA04F605EA0A0A46EAC8
:100B10000A05DD60C1E70E4A95692C43946173E7CD
:100B20000B4AD5692C43D4616EE71A6822F0404223
:100B30001A601A6842EA87771F60DA6822F040423A
:100B400042EA8171D960BDE8F08F00BF6C5903089B
:100B5000001002401A6822F003021A601A683A4331
:100B60001A60DA6822F003020A438507DA607FF52B
:100B70005DAF1A6822F00C021A601A6842EA870216
:100B80001A60DA6822F00C0242EA81024407DA6055
:100B90007FF54FAF1A6822F030021A601A6842EAF5
:100BA00007121A60DA6822F0300242EA0112DA60B3
:100BB00002077FF541AF1A6822F0C0021A601A6876
:100BC00042EA87121A60DA6822F0C00242EA811211
:100BD000C606DA607FF533AF1A6822F440721A60F5
:100BE0001A6842EA07221A60DA6822F4407242EA7E
:100BF00001228506DA607FF525AF1A6822F440628B
:100C00001A601A6842EA87221A60DA6822F440629F
:100C100042EA81224406DA607FF517AF1A6822F4AF
:100C200040521A601A6842EA07321A60DA6822F4FF
:100C3000405242EA0132DA6002067FF509AF1A68D3
:100C400022F440421A601A6842EA87321A60DA686F
:100C500022F4404242EA8132C605DA607FF5FBAEFB
:100C60001A6822F440321A601A6842EA07421A608F
:100C7000DA6822F4403242EA01428505DA607FF503
:100C8000EDAE1A6822F440221A601A6842EA8742DE
:100C90001A60DA6822F4402242EA81424405DA60AE
:100CA0007FF5DFAE1A6822F440121A601A6842EA31
:100CB00007521A60DA6822F4401242EA0152DA60FE
:100CC00002057FF5D1AE1A6822F440021A601A6854
:100CD00042EA87521A60DA6822F4400242EA8152FC
:100CE000C604DA607FF5C3AE1A6822F040721A605B
:100CF0001A6842EA07621A60DA6822F0407242EA31
:100D000001628504DA607FF5B5AE1A6822F04062B0
:100D10001A601A6842EA87621A60DA6822F0406252
:100D200042EA81624404DA607FF5A7AE1A6822F0D5
:100D300040521A601A6842EA07721A60DA6822F0B2
:100D4000405242EA0172DA6097E600BF10B504092A
:100D5000013C022C17D80D4B33F8142000F00F0083
:100D600042FA00F313F001030DD0012303FA00F05F
:100D70000138104020F048FD054A064B125D104432
:100D800003EBC00010BD002010BD00BF9454030849
:100D90009C540308A8480020564B574A57482DE951
:100DA000F04F4FF080069E874FF48076A3F84460A2
:100DB0004FF40076A3F84C604FF48066A3F85460BB
:100DC0004FF400664FF09041A3F85C604FF48056FA
:100DD0004FF400554FF480444FF0010B4FF0020ADE
:100DE0004FF004094FF008084FF0100C4FF0200EA0
:100DF00040271960996019619961196299621963B4
:100E000099631964996419659965196699661967F2
:100E10009967A3F864604FF400414FF08006A3F88F
:100E200004B0A3F80CA0A3F81490A3F81C80A3F8B6
:100E300024C0A3F82CE09F86A3F86C50A3F874405C
:100E4000A3F87C10A3F8BC604FF48076A3F8C460CC
:100E50004FF40076A3F8CC604FF48066A3F8D4601A
:100E60004FF40066A3F8DC604FF48056C3F880208E
:100E7000A3F884B0C3F88820A3F88CA0C3F890200E
:100E8000A3F89490C3F89820A3F89C80C3F8A020FE
:100E9000A3F8A4C0C3F8A820A3F8ACE0C3F8B0201E
:100EA000A3F8B470C3F8B820C3F8C020C3F8C820B2
:100EB000C3F8D020C3F8D820C3F8E020A3F8E4603A
:100EC000C3F8E820A3F8EC50C3F8F020A3F8F440EE
:100ED000C3F8F820A3F8FC10C3F80001A3F80451EC
:100EE000C3F80801A3F80C41C3F81001A3F81411CA
:100EF000BDE8F08FA8480020000400480008004822
:100F0000002867D003682DE9F04F03F138445C4EA8
:100F1000A40A0125345D04F01F066409022C05FAB9
:100F200006F558D0032C00F0A580012C58D08088FD
:100F3000B0FA80F4C4F11F04A4B2E50803EB850500
:100F400004F007042E6AA4000F27A74026EA07062C
:100F50002E622E6A01F00307A2407C1E3243012C50
:100F6000C1F3810CC1F300182A62C1F341113CD9CD
:100F7000C60700F18980850700F19580440700F1DC
:100F8000A380020700F1B180C60600F1BF8085068C
:100F900000F1CD80440600F1DB80020600F1E9801B
:100FA000C60500F1F780850500F10581440500F1D3
:100FB0001381020500F12181C60400F12F8185040F
:100FC00000F13D81440400F14B81020400F159819C
:100FD000BDE8F08F70472B4CA6693543A561A6E7A5
:100FE000284C666935436561A1E7002422464FF02D
:100FF000010E4FF0030904E00132102A04F102044B
:10100000E6D00EFA02F636EA0005F5D1D3F808A0CC
:1010100009FA04F5ED430AEA050AC3F808A0D3F873
:1010200008B00CFA04FA4AEA0B0AC3F808A0B3F8AD
:1010300004A01FFA8AFA2AEA06069E80B3F804A0E2
:1010400008FA02F646EA0A06B6B29E801E682E40EC
:101050001E60D3F800A007FA04F646EA0A061E60EE
:10106000D3F80CA001FA04F605EA0A0A46EA0A05D2
:10107000DD60C1E7034CE6693543E56157E700BF32
:101080006C590308001002401A6822F003021A602B
:101090001A683A431A60DA6822F003020A438507A5
:1010A000DA607FF56BAF1A6822F00C021A601A68DA
:1010B00042EA87021A60DA6822F00C0242EA8102F0
:1010C0004407DA607FF55DAF1A6822F030021A60DB
:1010D0001A6842EA07121A60DA6822F0300242EA1D
:1010E0000112DA6002077FF54FAF1A6822F0C002E2
:1010F0001A601A6842EA87121A60DA6822F0C0029F
:1011000042EA8112C606DA607FF541AF1A6822F41E
:1011100040721A601A6842EA07221A60DA6822F4FA
:10112000407242EA01228506DA607FF533AF1A6821
:1011300022F440621A601A6842EA87221A60DA686A
:1011400022F4406242EA81224406DA607FF525AF4C
:101150001A6822F440521A601A6842EA07321A608A
:10116000DA6822F4405242EA0132DA6002067FF580
:1011700017AF1A6822F440421A601A6842EA8732AE
:101180001A60DA6822F4404242EA8132C605DA6027
:101190007FF509AF1A6822F440321A601A6842EAF1
:1011A00007421A60DA6822F4403242EA01428505B9
:1011B000DA607FF5FBAE1A6822F440221A601A68E2
:1011C00042EA87421A60DA6822F4402242EA814207
:1011D0004405DA607FF5EDAE1A6822F440121A6019
:1011E0001A6842EA07521A60DA6822F4401242EAA8
:1011F0000152DA6002057FF5DFAE1A6822F4400280
:101200001A601A6842EA87521A60DA6822F44002C9
:1012100042EA8152C604DA607FF5D1AE1A6822F044
:1012200040721A601A6842EA07621A60DA6822F0AD
:10123000407242EA01628504DA607FF5C3AE1A6843
:1012400022F040621A601A6842EA87621A60DA681D
:1012500022F0406242EA81624404DA607FF5B5AE72
:101260001A6822F040521A601A6842EA07721A603D
:10127000DA6822F0405242EA0172DA6002047FF535
:10128000A7AE1A6822F040421A601A6842EA8777CD
:101290001F60DA6822F0404242EA8171D960BDE8FD
:1012A000F08F00BF002852D0036803F138422DE9C7
:1012B000F04F920A504DAA5C02F01F05520901241A
:1012C000022A04FA05F443D0032A00F09080012A90
:1012D00043D001F003077A1E012AC1F3810CC1F348
:1012E00000188088C1F341113CD9C60700F18880FD
:1012F000850700F19480440700F1A280020700F105
:10130000B080C60600F1BE80850600F1CC804406A0
:1013100000F1DA80020600F1E880C60500F1F680EF
:10132000850500F10481440500F11281020500F1F8
:101330002081C60400F12E81850400F13C81440423
:1013400000F14A81020400F15881BDE8F08F704736
:101350002A4A95692C439461BBE7284A55692C4376
:101360005461B6E7002422464FF0010E4FF0030906
:1013700004E00132102A04F10204E6D00EFA02F66B
:1013800036EA0005F5D1D3F808A009FA04F5ED43D3
:101390000AEA050AC3F808A0D3F808B00CFA04FA60
:1013A0004AEA0B0AC3F808A0B3F804A01FFA8AFAA5
:1013B0002AEA06069E80B3F804A008FA02F646EA76
:1013C0000A06B6B29E801E682E401E60D3F800A0AA
:1013D00007FA04F646EA0A061E60D3F80CA001FAE2
:1013E00004F605EA0A0A46EA0A05DD60C1E7034A8F
:1013F000D5692C43D4616CE76C5903080010024096
:101400001A6822F003021A601A683A431A60DA680E
:1014100022F003020A438507DA607FF56CAF1A6891
:1014200022F00C021A601A6842EA87021A60DA682F
:1014300022F00C0242EA81024407DA607FF55EAFD7
:101440001A6822F030021A601A6842EA07121A601B
:10145000DA6822F0300242EA0112DA6002077FF510
:1014600050AF1A6822F0C0021A601A6842EA871266
:101470001A60DA6822F0C00242EA8112C606DA6017
:101480007FF542AF1A6822F440721A601A6842EA85
:1014900007221A60DA6822F4407242EA01228506C5
:1014A000DA607FF534AF1A6822F440621A601A6875
:1014B00042EA87221A60DA6822F4406242EA812214
:1014C0004406DA607FF526AF1A6822F440521A60AB
:1014D0001A6842EA07321A60DA6822F4405242EA95
:1014E0000132DA6002067FF518AF1A6822F4404232
:1014F0001A601A6842EA87321A60DA6822F44042B7
:1015000042EA8132C605DA607FF50AAF1A6822F432
:1015100040321A601A6842EA07421A60DA6822F416
:10152000403242EA01428505DA607FF5FCAE1A6876
:1015300022F440221A601A6842EA87421A60DA6886
:1015400022F4402242EA81424405DA607FF5EEAEA1
:101550001A6822F440121A601A6842EA07521A60A6
:10156000DA6822F4401242EA0152DA6002057FF59D
:10157000E0AE1A6822F440021A601A6842EA875202
:101580001A60DA6822F4400242EA8152C604DA6044
:101590007FF5D2AE1A6822F040721A601A6842EAE9
:1015A00007621A60DA6822F0407242EA016285043A
:1015B000DA607FF5C4AE1A6822F040621A601A68D9
:1015C00042EA87621A60DA6822F0406242EA816287
:1015D0004404DA607FF5B6AE1A6822F040521A6011
:1015E0001A6842EA07721A60DA6822F0405242EA48
:1015F0000172DA6002047FF5A8AE1A6822F0404258
:101600001A601A6842EA87771F60DA6822F040425F
:1016100042EA8171D960BDE8F08F00BF10B1036864
:1016200082881A85704700BF10B1036882889A616A
:10163000704700BF38B100298388026814BF0021B9
:1016400010218B40936170470E4B1B8801463BB9BC
:101650000D4B0E4A1B7810680BB981F00101E9E7C8
:101660000B4B5A691AB118B91A6810605874704750
:10167000084A18681188084A92FBF1F201210260B9
:10168000597470472C6500202E65002030650020BD
:10169000346500204C65002020A1070010B40A4BDF
:1016A0000A4A1C7801238340234052F8200029B9BC
:1016B000B3FA83F149095DF8044BBBE7191C18BF65
:1016C00001215DF8044BB5E71C6500202065002072
:1016D00030B1036882881B8A1A4214BF012000209F
:1016E000704700BF2DE9F0410B4E346873691C4010
:1016F0000FD0DFF828800127B4FA84F3C3F11F0369
:1017000007FA03F558F8230003689847AC4375615E
:10171000F2D1BDE8F08100BF00040140B4580020C0
:101720002DE9F0410B4E346873691C400FD0DFF88F
:1017300028800127B4FA84F3C3F11F0307FA03F5E5
:1017400058F8230003689847AC437561F2D1BDE8AF
:10175000F08100BF00040140B45800202DE9F041A1
:101760000B4E346873691C400FD0DFF828800127C6
:10177000B4FA84F3C3F11F0307FA03F558F8230002
:1017800003689847AC437561F2D1BDE8F08100BFB2
:1017900000040140B45800202DE9F0410B4E34689C
:1017A00073691C400FD0DFF828800127B4FA84F356
:1017B000C3F11F0307FA03F558F82300036898479D
:1017C000AC437561F2D1BDE8F08100BF0004014077
:1017D000B45800202DE9F0410B4E346873691C4069
:1017E0000FD0DFF828800127B4FA84F3C3F11F0378
:1017F00007FA03F558F8230003689847AC4375616E
:10180000F2D1BDE8F08100BF00040140B4580020CF
:101810002DE9F0410B4E346873691C400FD0DFF89E
:1018200028800127B4FA84F3C3F11F0307FA03F5F4
:1018300058F8230003689847AC437561F2D1BDE8BE
:10184000F08100BF00040140B45800202DE9F041B0
:101850000B4E346873691C400FD0DFF828800127D5
:10186000B4FA84F3C3F11F0307FA03F558F8230011
:1018700003689847AC437561F2D1BDE8F08100BFC1
:1018800000040140B4580020084A094808B593698B
:1018900043F0010393610021402221F026FB054B18
:1018A0004FF0FF321A60C3F8032008BD0010024059
:1018B000B4580020F458002003685B6A184700BF42
:1018C0002DE9F041044618460D46164698461FF08D
:1018D000A1FA2768E6722844A07229467D6943462A
:1018E00032462046AC46BDE8F0416047036810B57B
:1018F00004461B689847236820469B689847A37B4B
:101900000133A37310BD00BF10B5036804469B6884
:101910009847FF2301226373227310BD064B984240
:1019200002D04FF0FF307047044A538B01339BB213
:101930005383508B80B2704700380040EC64002025
:1019400038B583680446154613B11A689B88138519
:10195000606840F2E93300E07BB30289013B12F09A
:10196000020F9BB2F8D0017340F2E93300E023B3D9
:101970000289013B12F0010F9BB2F8D0037B606833
:1019800040F2E93300E0DBB10189013B11F0020FC5
:101990009BB2F8D0057340F2E93300E083B10289CD
:1019A000013B12F0010F9BB2F8D0037BA36813B187
:1019B0001A689B889361012038BDFFF7AFFFDEE70F
:1019C000FFF7ACFFF2E700BFF0B50D460178012943
:1019D00083B00446164618D0022902D0002003B076
:1019E000F0BD80681F46FFF719FE45F08001606872
:1019F000EFF7A4FD3B46324600216068EFF7EEFCAE
:101A0000A068FFF711FE0120E9E790F90400421CED
:101A1000E4D00228E2DC617900962A46F0F792FAD7
:101A2000DDE700BF427A02B9704710B5044603688B
:101A3000406804F10A0198470023637210BD00BF9B
:101A4000437A5A1C0344D2B242729972037A934287
:101A500000D802B9704710B504460368406804F125
:101A60000A0198470023637210BD00BF98B10B4B69
:101A7000012210B402FA01F103F1750402E003330C
:101A8000A34209D01A788242F9D15A780A42F6D094
:101A900001205DF8044B70470020FAE7C0370308C7
:101AA00030B40A4D002305F1140401E0272B09D0BE
:101AB00003EB43020133A15C8142F7D12A4430BCDD
:101AC000907D7047002030BC704700BFAC370308E2
:101AD0002DE9F341056906460F467DBBD0F800802D
:101AE000C8F30A0323B30023D6F80080019315F04E
:101AF00057F9042819D1224C236943F001032361CB
:101B0000BBB2A8F8003015F04BF904282ED108F12B
:101B100002030193019B3F0C1F8015F041F92369DB
:101B2000042823F00103236125D06FF0010505E0AF
:101B300015F036F9042805D04FF0FF35284602B0DD
:101B4000BDE8F0810E4C236943F002032361C4F821
:101B50001480236943F04003236115F021F92369C0
:101B6000042823F002032361BDD0E5E7236923F0B5
:101B700001032361D9E7336804333360DEE700BF34
:101B800000200240F8B504460D468E180027B542E5
:101B900001D12069F8BDE368591CE160234415F8C0
:101BA000012B1A720429F2D1A1682046FFF790FF99
:101BB000E7602061EBE770B5448806460D46C4F344
:101BC0000B0422460021284621F08FF933690A4A86
:101BD000934209D3094A934206D22246284619461F
:101BE000BDE8704020F084B823B121462846BDE806
:101BF0007040184770BD00BFD0910308BE92030823
